:020000040800F2
:100000000080012095450008C9450008C945000841
:10001000C9450008C9450008C9450008000000009E
:10002000000000000000000000000000C9450008BA
:10003000C945000800000000C94500089D020008ED
:10004000C9450008C9450008C9450008C945000858
:10005000C9450008C9450008C9450008C945000848
:10006000C9450008C9450008C9450008C945000838
:10007000C9450008C9450008C9450008C945000828
:10008000C9450008C9450008C9450008000000002E
:10009000000000000000000000000000C94500084A
:1000A000C9450008C9450008C9450008C9450008F8
:1000B000C9450008C9450008C9450008C9450008E8
:1000C000C9450008C9450008C9450008C9450008D8
:1000D000C9450008C9450008C945000800000000DE
:1000E000C9450008C9450008C945000800000000CE
:1000F000000000000000000000000000C9450008EA
:1001000000000000C9450008C9450008C9450008AD
:1001100000000000000000000000000000000000DF
:10012000C9450008C9450008C9450008C945000877
:10013000C9450008000000000000000000000000A9
:10014000000000000000000000000000C945000899
:10015000C9450008C9450008C9450008C945000847
:10016000C9450008C9450008000000000000000063
:10017000000000000000000000000000000000007F
:1001800000000000C9450008000000000000000059
:10019000C945000810B5054C237833B9044B13B199
:1001A0000448AFF300800123237010BDD00B002062
:1001B00000000000B8510108084B10B51BB10849F8
:1001C0000848AFF300800848036803B910BD074B27
:1001D000002BFBD0BDE81040184700BF0000000016
:1001E000D40B0020B8510108C80B0020000000000B
:1001F000154B002B08BF134B9D46A3F5803A0021F9
:100200008B460F461348144A121A08F051FC0F4B44
:10021000002B00D098470E4B002B00D098470020B1
:10022000002104000D000D48002802D00C4803F006
:10023000E8FD07F01FFE2000290003F0A2FD03F0F7
:10024000DDFD00BF0000080000800120000000006C
:10025000753D0008D00B0020E41A0020033E000882
:10026000000000000A4B4FF47A721B68B3FBF2F3F4
:10027000013BB3F1807F09D2064A5360064BF0215F
:1002800083F823100023936007231360704700BF97
:10029000A801002010E000E000ED00E0024A136831
:1002A00001331360704700BFEC0B0020014B18684E
:1002B000704700BFEC0B002070B5037A032B044697
:1002C00004D0042B14BF00250A2500E00C2504F1FE
:1002D0000C0393E8070000F047FAE37E0230054480
:1002E0007BB104F1240393E8070000F03DFA04F128
:1002F0003003064693E8070000F036FA3044043035
:100300000544236C0BB9A36C3BB104F1400393E8A3
:10031000070000F029FA02300544E36C0BB9636D65
:1003200033B14C3494E8070000F01EFA0230054463
:10033000284670BDF7B50646019010460F46144694
:10034000FFF7BAFF054600F075F9B8426DDC1021E1
:1003500001A800F099F92946019800F02FF9019BB6
:10036000257A1844042D019005D1324901A800F0E6
:10037000ABF9294604E0304901A800F0A5F90321B2
:1003800001A800F081F9A37E00216FF3070163F358
:100390004101E37E003318BF012363F38201480764
:1003A00041BF94F83D3063F3C40194F83C3063F3EB
:1003B0004511236C0BB9A36C0BB141F08001E36CC8
:1003C0000BB9636D0BB141F04001CDB2294601A8D4
:1003D00000F05AF9218B01A800F05CF904F10C033C
:1003E0000ECB01A800F084F9E37E5BB104F1240395
:1003F0000ECB01A800F07CF904F130030ECB01A86C
:1004000000F076F92A0605D504F140030ECB01A8C9
:1004100000F06EF96B0605D54C3494E80E0001A887
:1004200000F066F90198801B01E06FF0010003B055
:10043000F0BD00BF943C0108993C010873B502ACC3
:10044000064644F8082D20460D4600F017F900F046
:10045000F000202815D101A9009800F0FDF8009BBC
:1004600003440093019B012B0CDD204600F006F9AC
:10047000C0F3C0103070204600F000F92870012051
:1004800000E0002002B070BD13B5012904464FF012
:10049000000301900DDD62F30713194601A800F077
:1004A000F3F80021019800F089F8019B1844001B23
:1004B00001E06FF0010002B010BD0C22FFF7E4BFB5
:1004C0002DE9F341002480461F4668460B9B0093AC
:1004D00015460E46019400F0D1F8234660F3070359
:1004E00003F0F002302A2BD1C3F3C00288F80020B9
:1004F000C3F34102C3F30003326001A92B700098DB
:1005000000F0AAF8009D019B054400951D44044697
:100510002A466946089800F00DF988B1009BEB1A4D
:10052000002B0DDB3368002B03DD684600F09EF8DE
:100530003880009B0A9AED1A1560099A012413600D
:10054000204602B0BDE8F081F7B502AC064644F89B
:10055000083D20460F46154600F090F8002360F352
:100560000703C3F3C002C3F303133A7001A9337046
:10057000009800F071F8009B03440093019B012B4D
:1005800004DD204600F072F82880012003B0F0BDA1
:10059000094A136870B51C460025E61AB14204DD0D
:1005A00014F8015B05700125F7E70029A8BF5B1867
:1005B00005B11360084670BDF00B002010B5421E57
:1005C000802400200B4B0B40002BBEBF03F1FF33F8
:1005D00063F07F030133DBB291FBF4F10029C8BF64
:1005E00043F08003002900F1010002F8013FE9DC3B
:1005F00010BD00BF7F000080F7B5002407460E46FF
:100600000C6001250134052C11D001210DF10700EA
:10061000B84701280BD19DF80720316802F07F030D
:1006200005FB0313336013064FEAC515EAD42046D1
:1006300003B0F0BD431C7F2B01DC02307047B3F5E3
:10064000804F01DA03307047024A9342D4BF04302E
:1006500005307047FEFF1F00024B18600248FFF78D
:10066000CBBF00BFF00B002091050008036819788C
:100670005A780233036002EB012070470368024698
:1006800013F8010B13607047036819700368013396
:100690000360704702684FF4807391FBF3F31370AB
:1006A0000268531C0360074B0B40002BBEBF03F1D5
:1006B000FF3363F0FF0301335370036801330360BA
:1006C000704700BFFF00008070B5054608460E4623
:1006D00009F0F6FB044601462846FFF7DBFF2246F9
:1006E0003146286808F0E6F82B681C442C6070BD81
:1006F00030B585B004AC04E90E00029C002C054620
:100700000CDD2146FFF7C6FF22460399006808F07A
:10071000D1F82B681C442C6005B030BD019921B183
:1007200005B0BDE83040FFF7CFBF05B0BDE83040B1
:10073000FFF7B0BF0B68D31A012B70B505460C4606
:10074000164601DC00200CE00846FFF78FFF236807
:1007500068601A189642F5D3AB602368184420608D
:10076000012000232B6070BD84B004AB03E90700B7
:10077000019810B104B009F0A3BB029804B070470F
:1007800070B504680E4624B1204609F099FB054671
:1007900001E084684568304609F092FB854208D143
:1007A0002A463146204609F0F9FBB0FA80F04009AC
:1007B00070BD002070BD1FB5044601A880E80E0082
:1007C00007C8FFF7D1FF069B02301844002CC8BFB2
:1007D000023004B010BD2DE9F04F85B01F46149CC7
:1007E000009410AD8B46039080469246384695E8BB
:1007F0000E00FFF7E0FF8146FFF71CFF58454FF062
:1008000000062BDC032363F307166AF3C3069DF887
:10081000383067F3420663F30006F1B203A8FFF72E
:1008200033FF49460398FFF7C9FE039B1844039022
:1008300095E80E0003A8FFF75BFF002F04DDBDF86D
:100840003C1003A8FFF726FF22461399039808F0EF
:1008500031F803982044C8EB000001E06FF001007C
:1008600005B0BDE8F08F13B50329044601944FF09D
:10087000000016DD62F3071063F3C300C1B201A8E4
:10088000FFF702FF02210198FFF798FE019BBDF8D8
:1008900010101844019001A8FFF7FCFE0198001BFE
:1008A00001E06FF0010002B010BD2DE9F0410646F5
:1008B0000F46022500244FF00C08B44209DA08FB69
:1008C000047393E80700FFF74FFF0330054401343A
:1008D000F3E72846BDE8F0812DE9F74F0C9F0D9D09
:1008E00001908B4606462946384690469946FFF7C2
:1008F000DCFF8246FFF79EFE58454FF000042CDCDB
:10090000082363F3071468F3C304012363F3420469
:10091000E1B201A8FFF7B8FE51460198FFF74EFE7D
:10092000019B18440190494601A8FFF7B3FE00243B
:100930004FF00C09BC420DDA09FB04530ECB01A8A1
:10094000FFF7D6FE0E9B01A813F82410FFF79CFEBC
:100950000134EFE70198801B01E06FF0010003B064
:10096000BDE8F08F2DE9F34702AC99460A9B44F8A5
:10097000083D8246204688461746FFF77FFE00F076
:10098000F000902821D101A90098FFF765FE009D95
:100990002E18019D0096012D1BDD2046FFF766FEF7
:1009A0000023AAF8000035443B60009BAB420AD20A
:1009B0003E6846450BDC731C3B602046FFF75EFE3D
:1009C00049F82600F1E7012003E0002001E04FF0A4
:1009D000FF3002B0BDE8F08738B504460D4605F09B
:1009E000AAFB2046256105F0CBFB2046BDE8384038
:1009F00005F082BB7FB504460E4605F0CFFB684686
:100A000005F0CCFB9DE80F0084E80F00204631463E
:100A1000FFF7E2FF204604B070BD10B5046905F091
:100A2000A7FB201A10BD70B504460D4616460021DE
:100A30001A46006801F090F8324629462068BDE861
:100A4000704001F00AB9092805DD1428B4BF3C2024
:100A50004FF416707047032070472DE9F8430446A1
:100A60008946174600254D451DDA384605F080FBBE
:100A70003B69984224DA3846D4F80080FFF7CDFF6E
:100A800005F1080602460021D8F80000264401F0CE
:100A900063F84A463146D8F8000001F0BBF8002858
:100AA0000EDB0544DFE70BD1D4F810324FF47A7136
:100AB00004F5FE705943FFF78FFF0020BDE8F8836F
:100AC0004FF0FF30BDE8F8832DE9F347056800F5E6
:100AD0008179044608460F46FFF79FFF012203462F
:100AE00049462846FFF79FFF0128054602D04FF0F0
:100AF000FF3034E03846FFF790FF4FF0050882469C
:100B00000026B8F1010812D0534601220DF1070169
:100B10002068FFF788FF012809D19DF8073003F00E
:100B20007F021B0605FB02664FEAC515E9D4314674
:100B300004F20310FFF742FD013009EB00053846CF
:100B4000D4F80080FFF769FF324603462946404645
:100B5000FFF769FFB042CAD194F80201000902B060
:100B6000BDE8F08710B50446D0F8100286B008B38F
:100B700004F5FE7005F0FCFAD4F80C32984217DB4D
:100B800094F81432A3B94FF47A7101A8FFF732FF39
:100B9000FA2104F10800FFF790FC011E08DD01AA0C
:100BA0002046FFF75AFF28B9012384F8143201E0E8
:100BB0004FF0FF3006B010BD10B443688BB104682D
:100BC0005CB18268501012F0010F18BF2258204407
:100BD00018BFD3585DF8044B184708465DF8044B1E
:100BE00018475DF8044B70472DE9F74381460E46E0
:100BF000174600F5087400F51C784FF0FF3554F8DF
:100C0000041C89B33046FFF7BBFD48BBB36872686C
:100C100054F8041C1A44013902F1FF3C11F8010F89
:100C2000E0B19A4220D993F800E0BEF12F0F01D134
:100C30002F2804E02B2804D023280CD070450BD09B
:100C400012E018468445034606D010F801EFBEF1C5
:100C50002F0FF7D100E0531E0133DFE79A4203D193
:100C60002368A3B9636893B910344445C7D165B10B
:100C7000D9F86C3213B9D9F8703283B1694609F5E5
:100C80001B7000970196FFF797FF002507E0694664
:100C90002046009701960025FFF78EFFE4E72846DF
:100CA00003B0BDE8F0832DE9F0418EB005460F4654
:100CB000FFF70AFF86B2B31E0B2B68D8DFE803F0FC
:100CC00067066745676767676767676305F58173E9
:100CD00003930DAB0293FA240CAB0DF11C080193A6
:100CE0000494CDF800800BAB0DF129020AA90DF197
:100CF0002A00FFF7E5FB01284ED10AAA4146284603
:100D0000FFF772FF9DF82830002B40D0012B05D152
:100D1000BDF82C3000930422002306E0022B3DD1C5
:100D2000BDF82C30009305220023214605F1080070
:100D3000FFF799FD002831DD01463A462846FFF7C6
:100D40008CFE431C044623D128E0FA24009405F5C8
:100D500081730AAA0DF11B0107A8FFF7F5FB012813
:100D60001CD1BDF82830009321460023062205F14E
:100D70000800FFF778FD011E10DD3A462846FFF710
:100D80006CFE58B903E0002485F8144200E000240A
:100D90002846FFF7E7FE1CB9344601E04FF0FF3468
:100DA00020460EB0BDE8F081F8B507460E46154660
:100DB0004FF0FF34284605F0DBF92B69984206DA3C
:100DC00029463846FFF76FFFB0420446F2D120466D
:100DD000F8BD000030B59DB004460D46416801A83D
:100DE000FFF708FE06AB58222149184607F062FDBE
:100DF00094F87822BABB002D08BF05464FF47A71EB
:100E00002B8BC4F81032594304F5FE70FFF7E4FD54
:100E1000FA212A4604F10800FFF78CFA011E22DDB0
:100E200001AA2046FFF719FE0546F0B901AA0221E2
:100E30002046FFF7B9FF022815D1FF238DF80230B5
:100E400004F58172FA230DF102010DF103008DF812
:100E50000350FFF7F3FA012805D19DF8025025B998
:100E600084F8780201E04FF0FF3528461DB030BD10
:100E7000A03C01082DE9F04397B0804600AF7D48C3
:100E80007D4C0D4609F01CF8083020F00700ADEB52
:100E9000000D784A7949684608F010FD2068784AC4
:100EA00078498068142306F053FB236876499868D4
:100EB00006F04EFB2368986806F006FA2068704A30
:100EC00070498068152306F043FB23686F499868D2
:100ED00006F03EFB2368986806F0F6F92068684A39
:100EE00068498068162306F033FB2E1D23683046C0
:100EF000D3F8089000F0BEFA65490246484606F06D
:100F000027FB2368986806F0DFF920685C4A5D4992
:100F10008068172306F01CFB23683046D3F808903E
:100F200000F002FA5B490246484606F011FB2368CE
:100F3000DFF89091986806F0C7F92068504A514947
:100F40008068182306F004FB2068534980686A46CD
:100F500040F25B7306F0FCFA2368986806F0B4F977
:100F60002068474A47498068192306F0F1FA236848
:100F70004549986806F0ECFA2368986806F0A4F9E9
:100F80000126286889F800604FF47A72002100F089
:100F9000E3FD286840F25B72694600F001FE0546F9
:100FA000206885B12123364A3C49806806F0D0FA92
:100FB00023683B4998682A4606F0CAFA236898686D
:100FC00006F082F950E02E4A2E498068242306F06C
:100FD000BFFA23683349986806F0BAFA236898681C
:100FE00006F072F989F800502F4BDFF8DC902F499A
:100FF0001E705822384689F8006007F05BFC032316
:101000003B7239462A4B7D604046FB60FFF7E2FEAB
:101010000546A0B9274B2068194A1E7019498068F7
:10102000312306F095FA23682349986806F090FA70
:101030002368986806F048F989F8005012E02068A3
:101040000F4A16498068342306F082FA23681B4948
:1010500098682A4606F07CFA2368986806F034F906
:10106000002D01DB164B1D6028465C37BD46BDE8F0
:10107000F08300BF913D0108E8050020D941010837
:10108000483D01089B3D0108AB3D0108D23D0108E8
:10109000E83D0108FF3D0108173E0108353E010803
:1010A000453E0108643E0108F40B0020A03C010805
:1010B000773E0108050C0020843E0108983E010897
:1010C000000C0020040C0020FC0B00202DE9F04354
:1010D000304BDFF8D490304D304C002285B00746BD
:1010E00088461A7041463846FFF7C4FE00284ED0A5
:1010F000D9F80030284E043B012B17D83068284A15
:1011000028498068462306F023FA274B30681B687D
:101110000093264A26498068462306F019FA336868
:10112000986805B0BDE8F04306F0CEB820680130FD
:101130002060FFF788FC03902868194A19498068E5
:101140004A2306F005FA2868039B2268194980683B
:1011500006F0FEF92B68986806F0B6F82368052BB0
:101160000CD1BFF34F8F1449144BCA6802F4E062EC
:101170001343CB60BFF34F8F00BFFDE7DDED037A74
:10118000F8EEE77A17EE900A05F06EFDAAE705B0D3
:10119000BDE8F083050C0020E8050020F80B0020D6
:1011A000F83C0108353E0108000C0020B23E010861
:1011B000CA3E0108E83E010800ED00E00400FA051F
:1011C00070B592B004460E4641680DA81546FFF76B
:1011D00011FC0AA900234B608B6094F878320A96C0
:1011E00013B94FF0FF304AE02B785A1E012A0AD873
:1011F000D4F818224FF6FF70824214BF0132012248
:10120000C4F81822AA80EA680692AA68059207C95B
:1012100002AE86E80700AA8801926A780092FA2155
:10122000002204F10800FFF7D6FA011ED9DD0DAA4D
:101230002046FFF712FC10BB2B78012B06D10DAA1C
:1012400004212046FFF7B0FD042807E0022B16D149
:101250000DAA07212046FFF7A7FD0728C1D1FA23D1
:1012600000930DF1260204F5817309A90DF1250003
:10127000FFF76AF910F1FF3018BF4FF0FF3012B0DE
:1012800070BD000070B5D0B005AC054616460C49DF
:101290001A46204608F012FB002320468DF8043041
:1012A0008DF805308DF80630039408F009FE01AA88
:1012B000049031462846FFF783FF50B070BD00BF51
:1012C000D941010810B5044600F0FCF8002384F869
:1012D000A830204610BDF8B51F4600230446164628
:1012E0000376421E4D1E481D15F8013F02F8013FCE
:1012F0008542F9D1304600F08CF93146A06004F106
:10130000580008F06BFD012384F8A830384600F03F
:1013100080F9E060069800F07CF92061204600F03A
:10132000BFF90020F8BD000010B588B006AA06235A
:101330000921044600F017F99DF81D2004929DF83C
:101340001C2003929DF81B2002929DF81A20019206
:1013500094349DF8192000929DF81830034A142106
:10136000204608F05DFA204608B010BD0C3F010889
:1013700030B5ADF52D7D0D460446684600F096FF6C
:101380002946684600F008FF431C3DD09DF8073011
:101390009DF806201B0443EA02639DF809201343CD
:1013A0009DF8082043EA0223A3609DF80F309DF8C2
:1013B0000E201B0443EA02639DF8112013439DF89D
:1013C000102043EA022323619DF813309DF8122078
:1013D0001B0443EA02639DF8152013439DF8142073
:1013E00043EA0223E3609DF80B309DF80A201B04BA
:1013F00043EA02639DF80D2013439DF80C2043EA55
:1014000002236361002400E0044608A800F05AFBB0
:1014100020460DF52D7D30BD037E10B504463BB949
:10142000204600F021F980F00100C0B2404210BD1A
:1014300043F69821FFF79CFF0028F1DA10BD07B5AD
:1014400004230DEB030200F08EF89DF804309DF8A4
:1014500007208DF804208DF807309DF806209DF8B0
:1014600005308DF806308DF80520019803B05DF841
:1014700004FB00001FB50F210446FFF7E0FFC3B2D5
:101480000293C0F3072358340193C0F3074300933A
:10149000044A030E1421204608F0C2F9204604B085
:1014A00010BD00BF2A3F010838B51C2204460D4676
:1014B000002107F0FDFA2046294605F095F8204660
:1014C00038BD000070B504461E460D46203011465A
:1014D000FFF7EAFF314604F13C00FFF7E5FF002289
:1014E0002846E561082105F099FAE069064905F00A
:1014F000AFFAA36A226A1A60636CE26B1A60034B4C
:1015000020461C6070BD00BF80841E00080C0020B7
:101510002DE9F8430446884617469946002508EB0E
:1015200005064D45B6B21CDAE069226AE16A036835
:1015300012040A601B68F0219847E0690368310AC9
:101540001B689847E0690368F1B21B689847E06937
:10155000795D03681B689847A36A226A1A6001359F
:10156000DDE7BDE8F8832DE9F843044688461746D1
:101570009946002508EB05064D45B6B21DDAE0692F
:10158000216AE26A0368090411601B680F21984709
:10159000E0690368310A1B689847E0690368F1B2A3
:1015A0001B689847E069036800211B6898477855D5
:1015B000A36A226A1A600135DCE7BDE8F88307B543
:1015C000090201F20341012301AA89B2FFF7CBFF0F
:1015D0009DF80400A0F117035842584103B05DF88C
:1015E00004FB37B505460024210201F20341012323
:1015F00001AA89B22846FFF7B6FF9DF804302BB147
:101600000134042CF0D14FF0FF3000E0204603B04D
:1016100030BD70B5044604260025204605F046FD81
:101620002E210543204608F001FA28B1013E4FEA79
:10163000052500F10104F0D1284670BD07B5130E51
:101640008DF80430C2F307238DF807208DF806309B
:10165000C2F3074204238DF805200DEB0302FFF7C8
:1016600057FF03B05DF804FB10B5044682680F21F4
:10167000FFF7E4FF226920460121FFF7DFFF204644
:10168000E2680521FFF7DAFF012010BD13B502ACB7
:10169000012304F8042D2246FFF73AFF02B010BDE3
:1016A000436CC26B10B51A60C36B826C04461B049A
:1016B0001360022005F0CCFA636CE26B1A6096208E
:1016C00005F0E0FA204680220021FFF7DFFF2246E6
:1016D000204606230921BDE81040FFF719BF37B5A2
:1016E000090201F20144A4B221460546FFF7CEFFEC
:1016F000012301AA21462846FFF735FF9DF8043053
:10170000002BF5D103B030BD73B50E1E054618DBB6
:101710003402A4B204F20341012301AA89B2FFF703
:1017200022FF9DF8043073B1314628461022FFF79E
:10173000D6FF04F2024189B2FF222846FFF7A6FF36
:1017400001E0002000E0012002B070BD002908B5D2
:1017500008DB090201F5806101F47F41FFF796FF84
:10176000012008BD002008BD07B5130A8DF804301C
:101770008DF80520022301AAFFF7CAFE03B05DF829
:1017800004FB2DE9F04F85B0B1F10008064617467D
:101790009A460E9D01DA002059E04FEA0824A4B2CF
:1017A00004F58061012201F47F41FFF76FFF012200
:1017B00041463046FFF793FF04F20C4B1FFA8BFBB8
:1017C0004FF00009384605F071FC2E210DF8090094
:1017D000384608F02BF930B109F10109B9F1040FCD
:1017E00000F10107EED104236A4659463046FFF75F
:1017F0008FFE04F5826189B21FFA8AF23046FFF744
:10180000B3FF07F0A7FC6FEA80426FEA924204F24E
:10181000044189B292B23046FFF7A6FF0422414646
:101820003046FFF75CFF684604F0B8FC684604F0F9
:10183000A7FC684604F060FC41463046FFF7BFFE57
:1018400028B9684604F094FCA842F5DDA3E705B08A
:10185000BDE8F08F07B5022301AAFFF784FE9DF8CB
:1018600004309DF805208DF804208DF80530BDF872
:10187000040003B05DF804FB2DE9F74FB1F1000A55
:10188000074693461C4638DB4FEA0A2606F585666E
:10189000B6B23146FFF7DEFF0AF10C05ED02ADB23C
:1018A000C0F30A01294489B205F500630A199A4276
:1018B00080460FDD5B1A0193BDF804905A464B46F3
:1018C0003846FFF750FE019AC9EB04039BB25A4415
:1018D000294601E0A3B25A463846FFF744FE08EB1A
:1018E000040292B231463846FFF73EFF38464022A6
:1018F0005146FFF7F4FE204601E04FF0FF3003B001
:10190000BDE8F08F2DE9FF410C1E074616469846AC
:1019100002DA4FF0FF3022E0684604F03FFC6846F0
:1019200004F02EFC6846240204F0E6FB04F584640F
:10193000A4B221463846FFF78DFF214605463846BA
:10194000FFF788FF8542F4D1454507DC731CF0D0D2
:10195000684604F00DFC8642EBDADAE7284604B06C
:10196000BDE8F0812DE9F0430C1E85B00746164610
:10197000984602DA4FF0FF3025E0684604F00EFC8E
:10198000684604F0FDFB6846240204F0B5FB04F24F
:101990002644A4B2002521463846FFF75BFF814666
:1019A00020B121463846FFF755FF05464D45F2D197
:1019B000454507DC731CEDD0684604F0D9FB864230
:1019C000E8DAD7E7284605B0BDE8F0832DE9F74F00
:1019D000B1F1000A074693461C4638DB4FEA0A2657
:1019E00006F22446B6B23146FFF734FF0AF1080585
:1019F000ED02ADB2C0F30A01294489B205F50063D6
:101A00000A199A4280460FDD5B1A0193BDF80490D3
:101A10005A464B463846FFF77BFD019AC9EB040353
:101A20009BB25A44294601E0A3B25A463846FFF712
:101A30006FFD08EB040292B231463846FFF794FE80
:101A4000384620225146FFF74AFE204601E04FF07B
:101A5000FF3003B0BDE8F08F70B5084694B00D4676
:101A60001646FFF7D6FDC3B20293C0F307230193D6
:101A7000C0F3074300931121030E04460E4A04A845
:101A800007F0CEFE294604A808F03EF810B93460ED
:101A900001240EE0002109A800F092FC294609A8C3
:101AA00000F0E6FD044608B10A9B336009A800F087
:101AB00009FC204614B070BD2A3F010800220270C4
:101AC000026170477047000030B5124B0446186839
:101AD00087B0154618B9104804F04AFF15E005AA6A
:101AE000FFF7BAFF88B1059BDAB20292C3F307226F
:101AF0000192C3F3074200921B0E084A10212046B0
:101B000007F08EFE2561002001E04FF0FF3007B0A6
:101B100030BD00BF080C0020433F01082A3F0108E8
:101B200070470069704700004FF0FF3310B5036045
:101B30000123037140F2DC538360054B1B68C360D3
:101B4000044613B9034804F013FF204610BD00BF3C
:101B5000080C0020843F010801718260704710B5B5
:101B600001680446C068FFF7CFFD80F001004FF028
:101B7000FF33C0B22360404210BD10B50446FFF7EA
:101B8000EEFF204610BD10B50446FFF7CDFF04F16F
:101B90001000FFF793FF002384F82430204610BD87
:101BA0000368002B2DE9F74304460D46164609DB72
:101BB00004F11007294632463846FFF785FF0546EF
:101BC00048B105E0C068FFF70CFD00282060EFDA9F
:101BD0004FF0FF351AE03846D4F80C80D4F8009066
:101BE000FFF79EFF42F210730093024633464946C8
:101BF0004046FFF7C6FD0028EAD040F2DC522946F5
:101C00002046FFF7A9FF012384F82430284603B0BB
:101C1000BDE8F08370B50D460168002904461646FC
:101C200018DB90F82430ABB12379C0680BB9A268F7
:101C300001E04FF0FF320023FFF764FE031E09DBD3
:101C4000B342A8BF33462A462168E068BDE8704029
:101C5000FFF7BCBE4FF0FF3070BD70B50D46016898
:101C600000290446164618DB90F82430ABB12379DE
:101C7000C0680BB9A26801E04FF0FF320023FFF704
:101C800071FE031E09DBB342A8BF33462A46216812
:101C9000E068BDE87040FFF7EFBD4FF0FF3070BD6A
:101CA00010B50446FFF740FF204610BD0368002B27
:101CB00010B5044603DAC068FFF793FC20600222E7
:101CC0002168E068FFF742FD80F00100C0B24042A9
:101CD00010BD000030B514468BB01378D278029254
:101CE000A2780192627800920D46074A112105A858
:101CF00007F096FD2279637905A943EA0222284676
:101D0000FFF7E2FE0BB030BD2A3F01082DE9F34199
:101D100004461F462379C0688846164621680BB9D9
:101D2000A26801E04FF0FF320823FFF71BFE051EFB
:101D300002DA4FF0FF3018E008236A462168E068B5
:101D4000FFF79AFD6A4641462046FFF7C3FFBDF8FC
:101D500006305BBA9BB2083D9D42EAD3BB42E8DC49
:101D600032462168E068FFF787FD02B0BDE8F081E8
:101D70002DE9F347064608460F46FFF7D1FE3468C3
:101D8000D6F80C80240204F20C440546A4B24FF0AD
:101D900000090DF1040A284605F088F92E210AF8F9
:101DA0000900284607F042FE30B109F10109B9F1F6
:101DB000040F00F10105EED10423524621464046AE
:101DC000FFF7A6FB3468F5683846FFF7AAFE210244
:101DD00001F5826182B289B22846FFF7C5FC02B0E4
:101DE000BDE8F0872DE9F04104461D462379C0681F
:101DF0000F46164621680BB9A26801E04FF0FF328A
:101E00006B1EFFF77FFD00280BDB39462046FFF7EE
:101E1000AFFF2B4632462168E068BDE8F041FFF78E
:101E2000D5BD4FF0FF30BDE8F081000038B5036844
:101E3000002B04460D4607DB236875B11B0203F235
:101E4000044399B2AAB211E0C068FFF7CAFB0028A8
:101E50002060F1DA4FF0FF3038BD0C490A680132DA
:101E60000A60190201F2044189B292B2E068FFF7F8
:101E70007BFC2168E0680222FFF768FCE0682168CB
:101E80000122FFF72CFC002038BD00BF0C0C002005
:101E90002DE9F04705460C4616461031042206305F
:101EA00005F1160806F006FD042204F1140140466F
:101EB00006F000FD4FF0FF3704F1F003264405F172
:101EC0000A0A1A78FF2A2CD0B3422AD2591C0AB91E
:101ED0000B46F6E7062A03F1020493F8019018D0A6
:101EE00008D8012A10D0032A18D10422214605F16E
:101EF0000E0011E0352A05D0362A0FD104222146E2
:101F0000404609E09F7809E00422214605F11200CD
:101F100002E004222146504606F0CCFC04EB090303
:101F2000CFE73846BDE8F087EF2A08B50B460CDD51
:101F30000A78022A09D1042200F13401981806F027
:101F400087FCB0FA80F0400908BD002008BD70B5DC
:101F50000C46631A9A420ADDD0F8A83214F8015BE5
:101F60005E1C0344C0F8A86283F85050F1E770BDCE
:101F700010B5002909DDD0F8A8325C1C0344C0F874
:101F8000A842013983F85020F3E710BD2DE9F04154
:101F9000284F3D4686B04FF0000804460422C0F8A2
:101FA000A88255F8040B01900DEB02012046FFF7C3
:101FB000CEFF404604F084FE064607F0CBF83044DE
:101FC000030E84F83430030C84F83530030A84F8A7
:101FD000363084F83700042204F134012046FFF73C
:101FE000B6FF424614212046FFF7C2FF06222146D3
:101FF0002046FFF7ACFF4246CA212046FFF7B8FF54
:1020000002AB0C371E46286869681A4603C20835B9
:10201000BD421346F7D128681060AA889A802046EE
:102020000E223146FFF793FFD4F8A80206B0BDE8B0
:10203000F08100BFBD3F0108F0B4D0F8A8521746A8
:1020400042196E1CC0F8A86282F850101A1E04468D
:1020500009DD34440235C0F8A85284F850203946CE
:10206000F0BCFFF774BFF0BC704700002DE9F041F1
:102070002E4E354686B000270446C0F8A8720422CA
:1020800055F8120B01900DEB02012046FFF75FFFA0
:10209000042204F134012046FFF759FF04F1160829
:1020A0003A460C212046FFF763FF042241462046B2
:1020B000FFF74DFF3A4604212046FFF759FF06225D
:1020C00021462046FFF743FF3A46CA212046FFF744
:1020D0004FFF02AB1A361F46286869681A4603C2CA
:1020E0000835B5421346F7D1286810602A791A716D
:1020F000394620460D22FFF72AFFA21D2046042361
:102100003221FFF799FF2046042342463621FFF78C
:1021100093FFD4F8A832581CC4F8A8021C44FF232B
:1021200084F8503006B0BDE8F08100BFBD3F010823
:1021300070B5044686B001A804F15005FFF7BEFC57
:102140004FF416732A4601A9E069FFF7DFFD061E6A
:102150001CDB324629462046FFF7E6FEB0B1324688
:1021600029462046FFF794FE02280AD12046FFF7B1
:102170007DFF2A46034604F12001E069FFF732FEA5
:1021800004E0052804BF012384F8383001A8FFF7D4
:1021900099FC06B070BD0000424B2DE9F74F044694
:1021A0001868C4F8AC028846002873D0224609217A
:1021B0000623FFF7D8F941F2873741F28833102020
:1021C000B845D4BF47461F4601F034FE0546FFF729
:1021D00067FDE5612846FFF769FD40F2DC5200210A
:1021E000E069FFF7B9FC02AA002542F8045D042368
:1021F0000F21D4F8AC02FFF78BF904F1200A442137
:10220000E069FFF713FE432227495046FFF75CFCC5
:102210002E4684F8385004F1500B04F13C0994F830
:10222000383073BB012D05D0022D14D0002DF9D10B
:10223000E56424E02046FFF7A9FE5A4603465146CE
:10224000E069FFF7CFFD484603F09AFF484603F0E8
:1022500053FF0225E3E72046FFF76AFF484603F0F5
:1022600087FF8742DBDA98FBF7F2E36C0133934296
:10227000E364A2BF012384F838304FF0FF36012514
:10228000CDE7E4694CB12046FFF777FC204601F02A
:10229000E1FD02E04FF0FF3000E0304603B0BDE862
:1022A000F08F00BF080C0020DC3F010810B5044689
:1022B0002030FFF703FC04F13C0003F06FFF2046E1
:1022C00010BD000038B5856A054B036004462DB18A
:1022D0002846FFF752FC284601F0BCFD204638BDD9
:1022E0000040010810B50446FFF7ECFF204601F05E
:1022F000B1FD204610BD38B50025044645600120DB
:1023000005F088FF206000B10570204638BD10B58B
:102310000446006808B105F085FF204610BDF8B5F9
:10232000036804460F461546C3B1406810440130A7
:1023300005F070FF064688B194E8060006F0BAFA88
:1023400060682A463946304406F0B4FA354463687A
:102350000022EA54206805F065FF2660F8BD000001
:102360002DE9F04106460F4600F104083368DC5DB4
:102370007D1C04B304F0C002C02A0AD1595D2402B6
:1023800004F47C5421433046FFF7EAFFB81CBDE853
:10239000F081B3683BB1094807F092FD0749024656
:1023A0004046FFF7BCFF3168224629444046FFF70C
:1023B000B6FF2F19DAE72846BDE8F0814547010846
:1023C00038B5074B044640F80C3B0D4603F0E6FEDB
:1023D000002384F82430A3622562204638BD00BF64
:1023E000004001082DE9F043CF7817F00F0785B0C2
:1023F00080460C4645D14B7991F804908E7943EA9A
:102400000929CB790C2543EA062619F1FF3935D382
:1024100002A8FFF770FF294601A80194FFF7A0FF6B
:10242000051D02A8FFF773FFEFE702A8FFF763FFA0
:10243000294601A80194FFF793FF00F1080300F17A
:102440000A02E55C215C234420445B7843EA0525CD
:10245000437843EA0123012B15440CD1A15C2244AB
:10246000D37843EA01635178927843EA014343EA1F
:102470000223C8F8043002A8FFF749FF16F1FF361F
:10248000D3D2384605B0BDE8F08330B50446ADF58B
:10249000077D01A8FFF712FB4FF4007306AA01A9FC
:1024A000A06AFFF733FC051E11DB022204F10801CC
:1024B00006A806F0CDF950B92A4606A92046FFF72E
:1024C00091FF08B9042300E0022384F8243001A816
:1024D000FFF7F8FA0DF5077D30BD00002DE9F04358
:1024E00089B01D46002302930393049301238DF8C2
:1024F0000A308DF80D30294B04460E4618680190BD
:102500000C2202A9304606F0D5F906F023FE03128C
:102510002372607204F108010222304606F0CAF903
:1025200006A8FFF7E8FE0C2405962B782BB32E2186
:10253000284607F07BFA671C814670B9284607F0E9
:10254000BFFC059B1855804602460598294638442D
:1025500006F0B0F908EB07040FE0059BC5EB000897
:1025600003F80480059829464246384406F0A2F94B
:1025700009F1010508EB0704D7E7059B00221A556E
:10258000601C04220DEB0201304406F093F906A80A
:10259000FFF7BDFE601D09B0BDE8F083EC3F010808
:1025A00070B5836AC6B004460D4633B9102001F0F9
:1025B00041FC0646FFF774FBA662A06AFFF776FBB4
:1025C000A06A40F2DC520021FFF7C6FA01A8FFF72B
:1025D00075FA3522124901A8FFF776FAA66A06F0C5
:1025E000B9FDC0F30E013046FFF720FC2B4606A9CB
:1025F0004FF480722046FFF771FF0C34034606AAA1
:1026000001A9E069FFF7EEFB204603F0B9FD204683
:1026100003F072FD01A8FFF755FA46B070BD00BF88
:10262000F03F010838B590F82430044633B9C3614F
:10263000016AFFF7B5FF012384F8243004F10C058B
:10264000284603F095FDB0F57A7F10DD284603F0AB
:1026500072FDE3690133012BE36101DD032304E033
:10266000216A2046FFF79CFF012384F8243038BDFF
:10267000002310B50446016280F824302046FFF79D
:10268000D1FF2046FFF701FF94F824000128F5D080
:10269000031F5842584110BD38B51C2204460D4650
:1026A000002106F005FA2046294603F08AFF0023A0
:1026B00084F89C3084F89D30204638BD7FB50C46A8
:1026C0002046184915461E4607F0F8F8164B174ADB
:1026D0001749002D08BF1A4601A807F0EFF801A915
:1026E000204607F083F99DF820203146284600F067
:1026F000D9F807EE900AB8EE677AF2EE047AC7EEE0
:10270000276A16EE900A10F091FD02460B4601A8CA
:10271000084907F0D3F801A9204607F067F904B08B
:1027200070BD00BFAF4101082549010808400108FC
:10273000D94101080A40010830B5044685B000EBD4
:10274000C2000D460DF10F030DF10E020DF10D014A
:102750001C3000F072F89DF80F1000919DF80E30BB
:102760009DF80D2029462046FFF7A8FF05B030BD93
:1027700010B500F11C0104469C3000F0E9F901237A
:1027800084F89D3094F89C0010BD38B501200D46AA
:10279000002100F009F8044620B91DB140F2EE20F6
:1027A00004F070FA204638BD38B50D46044600F0F6
:1027B000EBF800F0E1F840B12946442000F089F937
:1027C000012C04D000F0A0F901E0022038BD002067
:1027D00038BD70B54D780C78102844EA052408D12E
:1027E000E5008C794FF6F0762E40C4F10C043444A9
:1027F000A4B2250445BF01256442002515704CBFD5
:10280000A4B21570282810D10A7902F0600160295D
:102810000BD0510602D524F0010405E092064CBF0E
:1028200024F0030424F00704A4B222111A70049BBC
:1028300004F00F041C70002070BD2DE9F043064623
:1028400087B00F469046994600F09EF83146BE206C
:1028500000F03FF9002400F0EFF803AD28550134F3
:10286000092CF8D12146284600F042F8044650B120
:102870009DF81430FF2B0FD19DF81330FF2B14BFA0
:102880000324012409E03078CDF8009043463A460D
:102890002946FFF79EFF00E00324204607B0BDE86D
:1028A000F083000037B50D461049044608684968B2
:1028B0006B4603C340F271234FF47A70534393FB8A
:1028C000F0F305EB8500400010FA83F080B254B9B4
:1028D00023461DF80310914202D1013080B202E07C
:1028E0000133082BF5D103B030BD00BF1040010803
:1028F00070B5064604460020A31B9BB2994215D032
:1029000014F8015B082280EA050313F0010318BFE5
:1029100080F01800400813B160F07F03D8B2531E56
:1029200013F0FF024FEA5505EDD1E5E770BD000059
:10293000044B5A681B6812681A4214BF0120002019
:10294000704700BF100C002010B5044604F036F9A3
:102950002046012101F016F8BDE8104004F05AB9F4
:1029600010B5044604F02AF92046002101F00AF8C7
:10297000BDE8104004F04EB908B5FFF7D9FF0030AC
:1029800018BF012008BD000010B50F4C2046FFF70E
:10299000DBFF2368E2681B0413604FF4FA7004F055
:1029A00057F92046FFF7DCFF3C2004F051F9FFF710
:1029B000BFFF0446F02004F04BF9FFF7B9FF08B160
:1029C000E0B210BDFF2010BD100C002038B5104D36
:1029D00004462846FFF7B8FF2B68EA681B0413601B
:1029E000012004F035F914B12846FFF7B9FF0E2095
:1029F00004F02EF9FFF79CFF00284FF02D0008BFD0
:102A0000002404F025F90248FFF7AAFF204638BD4C
:102A1000100C002038B50446082504F00100FFF72B
:102A2000D5FF640810B164F07F04E4B2013D15F0F5
:102A3000FF05F2D1204638BDFF20FFF7EBBF2DE99F
:102A4000F84380460E46FFF79FFF044600283AD120
:102A5000F020FFF7DFFF4025A5F10807FFB20120B6
:102A6000FFF7B4FF81460120FFF7B0FF18B1B9F1BD
:102A7000000F13D02AE0B9F1000F0FD1A8450AD8F2
:102A80003378DB070AD5A8451ABF2C464FF0010959
:102A90004FF0000902E02C464FF001094846FFF7CD
:102AA00095FF33785B08B9F1000F01D063F07F0325
:102AB000013DEDB2BD423370D1D10136002DCBD1F5
:102AC0002046BDE8F8830120BDE8F883FE20BDE87C
:102AD000F88370B50C460546FFF756FF5CB15520EC
:102AE000FFF798FF04F1080614F8010BFFF792FFB7
:102AF000B442F9D102E0CC20FFF78CFF2846FFF763
:102B000089FF002070BD000010B5044C2046FFF77F
:102B10001BFFA36822681A60002010BD100C002063
:102B200038B504460D4629462078FFF788FF01286E
:102B300020700BD0FE2806D040B12B78282B04D073
:102B4000102BF0D101E0012038BD002038BD00007D
:102B5000F0B5044685B01A480D4606F0E7FAFF23A3
:102B60008DF807300023237002AE08279DF8070078
:102B700018B323780F2B1FD831460DF10700FFF74C
:102B8000CFFF9DF80730012B01D10E4802E0FE2B4C
:102B900005D10D4806F0CAFA9DF807000DE00023A4
:102BA0002278F15C17FB02320133082BA954F7D1CC
:102BB000237801332370D9E7002005B0F0BD00BFB2
:102BC00043400108514001086240010810B5064C1D
:102BD000002120461C2205F06BFF20460921BDE89C
:102BE000104003F0EEBC00BF100C0020704710B581
:102BF000044601F02FF9204610BD38B505460446BD
:102C000055F8043B9B689847284600F0E7FD236889
:102C10000546DB6820469847284638BD81627047E4
:102C20002DE9F84F00220023C0E928230D46044671
:102C3000FDF73CFB4FF47A7A0AFB05FA8346002540
:102C4000FDF734FBCBEB000050452FD2606BFFF754
:102C5000D4FF606510F0C8FAD4E91E6732463B46DF
:102C60008046894610F082F90022214B10F032FB99
:102C700032463B4610F07CF902460B46C4E91E235F
:102C80004046494610F072F902460B46C4E91A2341
:102C900010F020FB02460B46C4E92623D4E92801A4
:102CA00010F066F90135C4E92801C9E70EA3D3E99C
:102CB0000023D4E9100110F00DFB064628460F460C
:102CC00010F092FA02460B46D4E9280110F02CFCD1
:102CD00004F0CCF802460B463046394610F0FAFABA
:102CE000C4E90801BDE8F88FB81E85EB51B80A3F6A
:102CF0000000503F034610B553F8042B044602B9B8
:102D0000036022689A4204D059220349034803F021
:102D100013FE206810BD00BF88400108AA400108CA
:102D200008B50248FFF7E6FF08BD00BF14190020F0
:102D300008B50248FFF7DEFF08BD00BF14190020E8
:102D4000F8B50446084B094E44F8043B05460F46C7
:102D50003046FFF7CFFF3946204600F0CBFC304627
:102D6000FFF7C8FF2846F8BD784001081419002075
:102D700038B5C0E91023084BC18500220446C0E9DC
:102D80001E230C2001F056F8B4F92E100546FFF76B
:102D9000D7FF656338BD00BF0000E040014B012252
:102DA0001A7070472C150020014B01221A707047D1
:102DB0009D0100200368184708B10B680360704745
:102DC000704738B5046805464CB104F11000FEF7B1
:102DD00079FE2046FEF7D1FE204601F03BF828465A
:102DE00038BD000038B503680C4CDA6899680546B0
:102DF000204607F023F92B68DB680022E254084BD9
:102E000001221A70074B1B7833B122460649074846
:102E1000BDE8384003F014BB38BD00BF590C00209A
:102E2000841500209C010020CC400108641400207F
:102E300030B585B0044603F0B1F9684603F0AEF949
:102E40009DE80F0084E80F00204605B030BD10B5A6
:102E5000044603F08DF923699842B4BF0020012095
:102E600010BD0000094B1B7870B505460C4623B118
:102E70000A460748074903F0E3FA23462A4606496B
:102E80000648BDE87040FEF7FDB900BF9C01002078
:102E900064140020DA4001087C140020C40E0020D5
:102EA00008B50B490B4803F0CBFA0B490B48FEF76A
:102EB0000DF90B4B1B68043B012B08D84FF07E50DB
:102EC00003F0D2FE0749034803F0BAFAF6E708BD5B
:102ED000E4400108641400207C140020C40E00208B
:102EE000000C0020F8400108C36810B504460BB17F
:102EF0009B689847204610BD10B5044B044640F827
:102F0000B83BFFF7F1FF204610BD00BF844B01081E
:102F100010B50446FFF7F0FF204600F09BFF204667
:102F200010BDC36810B504460BB19B689847204696
:102F300010BD000038B50546064B45F8183B044661
:102F400003F0CCFA2846FFF7ECFF204603F088F99F
:102F5000204638BDDC49010810B50446FFF7EAFFFA
:102F6000204600F077FF204610BD000070B50646F1
:102F70000B4B46F8983B044646B100F1B805B54204
:102F800004D0103D2846FFF7CCFFF8E704F13800E5
:102F9000FFF7AAFF04F12800FFF7A6FF204670BD47
:102FA0002C4C010810B50446FFF7E0FF204600F066
:102FB00051FF204610BD000010B5064B03602033C2
:102FC000044640F8BC3F03F029FA2046FFF7CEFF45
:102FD000204610BDF0490108A0F1BC00ECE700BF9D
:102FE00038B5CB6804460D460BB15B689847EB6873
:102FF000E360204638BDF0B593B005460E46416803
:103000008DF817200DA81F46FDF7F4FC0AAA00232F
:103010005360936095F878320A9613B94FF0FF30F9
:1030200051E0D5F8183201924FF6FF718B4214BF70
:10303000013301230DF117010122C5F81832029165
:103040000092FA2105F108009BB20022FDF744FC32
:10305000011EE3DD0DAA2846FDF7FFFC98BB0DA875
:10306000FFF7F5FE04460028D8D10DA92846FDF744
:103070001AFE0928F3D112AB4FF0FF3243F8242D8A
:10308000FA22019205F581720092012108AA0DF140
:103090001E000894FDF766FC012812D109988028CB
:1030A00011D000231A01AC18D4F81C1229B9C4F8A5
:1030B0001C62C4F82472084605E00133052BF1D1E7
:1030C00001E02046EDE713B0F0BD30B587B00D4606
:1030D000044601A8FFF7ACFE294601A8FDF77CFCD9
:1030E00001A8FFF7B4FE30B901A92046FDF7DBFDCA
:1030F000431CF5D100E0002007B030BD0000000007
:1031000070B59D4C9D4D8AB0FDF7ACF89C499D4B28
:103110009D481B2203F094F9A36822681A604FF0BF
:10312000804003F0A1FDFFF7BBFE984B98499948FA
:103130000122FFF760FF964A97490346924803F041
:103140007FF9964B029302A906A80595FFF748FF61
:103150009348FFF7E6FE06A99148FFF741FF914922
:10316000914803F0A7F906A8FFF7DBFE02A8FFF7D6
:10317000D8FE8E4B029302A906A80595FFF730FFF3
:103180008B48FFF7CEFE06A98948FFF729FF85493E
:10319000884803F08FF906A8FFF7C3FE02A8FFF7DF
:1031A000C0FE8548FFF7E4FAFF21844803F055FB91
:1031B0000022834B83480021FFF7DAFD0A2175487E
:1031C000FFF783FF63686C4A19682368194202D0CD
:1031D000D2681B0400E0926813607B4B1A78002AC7
:1031E0007CD0002275481A7003F019FB774D784E99
:1031F000784B7949C04328603246784806F084FB12
:10320000012804DC7649774806F058FB62E0337801
:10321000483B0C2B5ED8DFE803F0575D5D5D5D5DDC
:103220005D5D075D22373B006A4B6F4E1A78531E77
:10323000D9B2032907D82968012201F0700102FAE6
:1032400003F30B4303E01AB92B6803F070033360F8
:1032500066493268634806F031FB31680FE05D4B28
:103260001B78072B36D82A685F4D60495D4802F00D
:103270000F0242EA03122A6006F020FB29684F4839
:10328000C94303F0EAFA25E0574B58491A681EE093
:10329000574D49480121FFF778FA29460022464850
:1032A000FFF74AFA012253494348FFF745FA022241
:1032B00051494148FFF740FA00954F4B4D4A4F495D
:1032C000484806F0FBFA05E04D4B4E491A68454860
:1032D00006F0F4FA43494C48FFF7C4FD4B4B1A780B
:1032E0008AB100221A704A4B3E481A68511C196074
:1032F000484906F0E3FA3B494348FFF7B3FD0A218A
:103300002448FFF7E2FE444B1A783AB30022022128
:103310002C481A70FFF784FC13A3D3E900230FF0A5
:1033200025FE13A3D3E900230FF0D4FF10F082FA97
:103330003A4B334D1B78286083B102212148FFF7B7
:103340006FFC09A3D3E900230FF010FE2B68009354
:1033500002460B460C48324903F072F84FF07E509B
:1033600003F082FC2AE700BF7B14AE47E17AB43F4A
:103370000000000000606D40EC120020C040010819
:103380002E4101082A41010864140020E52D00089F
:103390007D410108C40E0020974101089D2D0008C1
:1033A000480C0020404B4C00300C0020A92D000898
:1033B000A0150020881500200813002038150020D3
:1033C00000004440201200208415002040110020FD
:1033D000580C0020E8120020B0410108590C0020D0
:1033E000B6410108850D00202C0C0020BA410108CF
:1033F0002D150020B10E0020B90E0020C441010897
:10340000E0120020DC410108E44101082C150020F5
:10341000E4120020014201089D0100209C010020CF
:103420000B42010810B50446FFF7C6FD204600F028
:1034300011FD204610BDA0F1BC00F3E72DE9F047D7
:10344000694EDFF8F091694CDFF8ECA194B04FF0D1
:10345000FF381323CDF8008014221521304603F0E5
:1034600021FB251D4A466249304600F0C5FC314625
:1034700008231A222846FDF725FF4FF07E5003F05F
:10348000F3FB282000F0D6FC0646FEF77CFB594BE8
:103490002660594A00935949594B2846FDF71BFFAE
:1034A0002846584DFDF7B8FF05F5FE764A465649C1
:1034B000204600F0A1FC2C6030460024FFF7B8FC49
:1034C0000FAFC5F81842C5F82042C5F82442C5F828
:1034D0003042C5F83442C5F84042C5F84442C5F808
:1034E0005042C5F85442C5F86042C5F86442C5F878
:1034F0006C42C5F870420FA8FFF79AFC0FCF0FC6B9
:103500003B683360414E85F8144247F230536B609C
:103510004FF41653C5F81C42C5F82C42C5F83C427E
:10352000C5F84C42C5F85C4285F878420322009306
:10353000374D384F23460221304603F005F84A46FE
:103540003549304600F058FC1C222146284605F03B
:10355000AFFA2846314D052103F046F8284602F01F
:1035600061FEC5F800A06C6228462D4D4A463946DA
:1035700000F042FC284602F055FE6C624A4639468D
:103580002846284CC5F800A000F036FC0B23049315
:103590002920182119220C238DE80F00CDF8308046
:1035A0002523CDF82C80CDF82880CDF82480CDF8C7
:1035B0002080CDF81C80CDF81880CDF8148026220C
:1035C0002821204603F0A2F84A461749204600F079
:1035D00013FC09211548FFF75FF831461448FFF73F
:1035E0001DFB14B0BDE8F087441100207C140020BE
:1035F000F92E00083D420108324201089E010020D8
:1036000024420108C40E0020C32D0008A813002086
:10361000EC120020352F0008B92F0008300C0020D4
:103620008815002038150020D166000808130020F6
:103630002012002098010020DC4901081FB5044633
:1036400010220021684605F033FA284B22681A60E0
:10365000A279012301930293122A44D8DFE802F0F1
:103660000C0B0A232527292B2D2F31333537393BD6
:103670003D3F4100022300931D4A1C48536823F438
:1036800040036946536001F027F9184801F070F8CB
:103690000A21164801F0CCF828BB144801F018F9AB
:1036A00080B204B010BD0323E5E70423E3E705235C
:1036B000E1E70623DFE70723DDE70823DBE709234C
:1036C000D9E70A23D7E70B23D5E70C23D3E70D234C
:1036D000D1E70E23CFE70F23CDE71023CBE711234C
:1036E000C9E71223C7E70020DBE700BF0C1A002060
:1036F000002301404FF0FF33EF2973B504460D4618
:1037000003604CDC2B49284603F0EAF82949206085
:10371000284603F001F927490646284603F0A4F895
:103720002368013304D148222349244803F004F9D3
:10373000731C04D149222049214803F0FDF8216877
:10374000204BA580C6F304369942A6710FD11E48BE
:10375000036813BB01931D4B5A6C42F480725A6488
:103760005B6C03F480730193019B01230360184891
:10377000002301220160436083600361836103626F
:103780004362C3628362C360C2610363436100F04A
:1037900045FF10B10F4803F0EBF802B070BD0E49C1
:1037A000284603F09DF80C492060284603F0B4F841
:1037B0000646B5E748420108D044010839450108EA
:1037C0005145010800200140B0150020003802409A
:1037D0000C1A00206A450108FC42010808B5FFF7F1
:1037E0002DFFC0F3032343EA001080B208BD0000A0
:1037F00030B50C4CA268A468B4F1006F13460CD12C
:10380000131F094C094A53F8045F42F8045FA242AF
:10381000F9D1044A4FF000539360103043F8201060
:1038200030BD00BF00ED00E090010020FCFFFF1F55
:103830007FB50023072855D8DFE800F00413202DBA
:103840003A54544700932A4B2A481A6B42F001021B
:103850001A631B6B03F001030093009B07B05DF834
:1038600004FB0193224B24481A6B42F002021A63B4
:103870001B6B03F002030193019BEFE702931C4BC8
:103880001E481A6B42F004021A631B6B03F0040318
:103890000293029BE2E70393154B19481A6B42F01F
:1038A00008021A631B6B03F008030393039BD5E71D
:1038B00004930F4B13481A6B42F010021A631B6BF0
:1038C00003F010030493049BC8E70593084B0E48CC
:1038D0001A6B42F080021A631B6B03F0800305939E
:1038E000059BBBE7094803F043F80020B6E700BF9B
:1038F000003802400000024000040240000802407C
:10390000000C024000100240001C024081450108EA
:10391000431C10B5044604D174220649064803F03E
:103920000BF82046002100F047FB04F00F040120B3
:10393000A04010BDA2450108F845010870B5044635
:103940004B1C0E46218216D0C1F30310FFF770FF07
:1039500005463046FFF7DCFF238A074A656103F01E
:103960000F03206052F82330A36105F110031835CE
:103970006360A560E56070BD44460108B0F91000C1
:1039800000F0B2BB10B58369446971B9216893FA3C
:10399000A3F2B2FA82F20320520000FA02F221EA04
:1039A000020293FAA3F3226010BD226893FAA3F1F6
:1039B000B1FA81F193FAA3F30320490000FA01F16F
:1039C000B3FA83F322EA01025B00012101FA03F357
:1039D0001343236010BD000070B5134C23681A69AF
:1039E000950707D5DA68900704D56FF002021A61CF
:1039F00002F0B8FF23681A69510713D5DA68520735
:103A000010D56FF00402094E1A615D6A3368EB1A33
:103A1000B3F57A7F06D300F0F1FD236805F57A72DD
:103A20009A63356070BD00BFA41A0020B415002051
:103A300030B589B001A903A801F084FA01F052FA67
:103A400000230293244B01901A6C244C42F008028C
:103A50001A641A6C02F008020292029A1A6A42F080
:103A600008021A621A6A22F008021A62069AA3F57C
:103A70000B3323604FF0FF33E360194B4ABBB0FBBD
:103A8000F3F001380025606014482561A560656188
:103A900001F01AFF13493220FFF7AAFE124B0F481C
:103AA0004FF480225A60294601F04AFF04210B4856
:103AB00001F046FF23680D4A596A1160126802F549
:103AC0007A729A63DA68284642F00402DA6009B032
:103AD00030BD4000D3E700BF00380240A41A0020E8
:103AE00040420F00D939000800E100E0B415002081
:103AF00000B589B003F062F8052101A802F074FD59
:103B0000039B019A1A60962003F0BCF8019B049A6B
:103B10001B041360962003F0B5F8F1E770B50D466D
:103B2000A0B0044603F04AF82B462246802168469E
:103B30000AF0B6FC051E03DC03F06CF820B070BD83
:103B4000094B1B6823B903220221084800F00CFC32
:103B5000064E00241DF804103046013400F0E4FC49
:103B6000A542F7D1E8E700BF0C170020541A002047
:103B70000FB407B504A951F8040B0191FFF7CEFF6C
:103B800003B05DF804EB04B0704708B502F072F9B9
:103B9000BDE8084000F01ABD08B5084B1B685BB9CA
:103BA00002210748032200F0DFFB4FF416510448BE
:103BB000BDE8084000F082BC08BD00BF0C17002023
:103BC000541A0020022810B5044601DC002010BD64
:103BD00003F070FA09230360033C094B53F82400F7
:103BE000002243F8242040B103681B699847041E53
:103BF000ECDA03F05FFA644204604FF0FF3010BD6E
:103C0000B8150020F8B505460E46144603F052FAE2
:103C10000923022D03600FDC124B1B680BB9FFF761
:103C2000BBFF35463719104EBD4215D015F8011BA4
:103C3000304600F079FCF7E7033D0C4B53F82500C4
:103C400060B103682246DB6831469847041E03DAF8
:103C500003F030FA634203602046F8BD4FF0FF34B2
:103C6000FAE700BF0C170020541A0020B8150020F6
:103C700070B504460D46164603F01CFA0923022CC3
:103C800003600BDC0F4B1B680BB9FFF785FF0E4879
:103C900000F02EFC01242870204670BD033C0B4B25
:103CA00053F8240058B1036832469B682946984768
:103CB000041EF1DA03F0FEF963420360ECE74FF013
:103CC000FF34E9E70C170020541A0020B815002033
:103CD00010B5044603F0EEF90923022C036010DD51
:103CE000033C0A4B53F8240040B103689B69984792
:103CF000041E08DA03F0DEF9644204604FF0FF307E
:103D000010BD012010BD002010BD00BFB81500205F
:103D100070B504460D46164603F0CCF90923022C73
:103D200003600BDD033C084B53F8240040B10368EB
:103D300032462946DB69BDE870401847002070BD57
:103D40004FF0FF3070BD00BFB8150020022808B545
:103D500004DC4FF400534B60002008BD03F0AAF9C7
:103D6000092303604FF0FF3008BD08B5012000F0C3
:103D700045F8704708B5FFF708FFFFF7FAFF08BDE1
:103D8000704708B5FFF7FCFFBDE80840FFF7B8B97A
:103D90000C4A136810B51844EFF30881884205D324
:103DA000094B0C221A604FF0FF3010BD07490C6818
:103DB00024B10749096821448842F1D210601846AD
:103DC00010BD00BFA4010020E01A0020C016002092
:103DD000C4160020074C08B523680546986803F010
:103DE00073FA2368D86803F06FFA0DB1FFF780FE0D
:103DF000FEE700BFE80500200120704708B5FFF787
:103E0000E9FF01207047002105F05ABC7047704758
:103E10007047704708B5FFF7F9FF08BD08B5FFF711
:103E2000F6FF08BD08B5FFF7F3FF08BD08B5FFF7BB
:103E3000F0FF08BD10B504F0EDF9044610B90248D2
:103E400002F096FD204610BD0B46010808B104F0B3
:103E5000E9B97047FFF7FABF10B504460948FEF705
:103E600049FF0023084A194652F82300A04208BF20
:103E700042F823100133402BF6D10248FEF73AFFF7
:103E800010BD00BFB8160020B81500202DE9F7437B
:103E90003449074605F038FE044628B9FFF77CFE92
:103EA000204603B0BDE8F0832F49384605F02CFECC
:103EB00018B9FFF771FE0124F2E72C49384605F0E6
:103EC00023FE18B9FFF768FE0224E9E703F0F2F8D1
:103ED000092303602648DFF8A080FEF70BFF0025CA
:103EE000C14658F8256036B30135402DF9D103F0AD
:103EF000E1F8182303601E48FEF7FCFE2FE0394668
:103F0000684602F059F9684602F084F930B948F879
:103F1000250003F0CFF802230360C1E7684602F0F2
:103F200069F9D0B1684602F06EF9064613E049F827
:103F30002560EC1CB4E74FF0FF340D4848F82540ED
:103F4000FEF7D8FE3B783A2BD9D16A460949384664
:103F500005F0DAFC009E002EE9D149F825604FF00B
:103F6000FF349DE73046010837460108284601081E
:103F7000B81600203F460108B815002030B5C368C8
:103F800091FAA1F4B4FA84F491FAA1F10325B1FAFB
:103F900081F1640005FA04F4490023EA040302FAFB
:103FA00001F11943C16030BD012A02D0022A18BFB5
:103FB0000022FFF7E3BF00002DE9F0410E46411C4F
:103FC000044604D13E224449444802F0B5FC04F0C2
:103FD0000F08434BC4F3031053F82850FFF728FC95
:103FE00006F007070446836895FAA5F1B1FA81F156
:103FF00095FAA5F20320490000FA01F1B2FA82F223
:1040000023EA01035200022101FA02F21343A360E2
:1040100087425AD8DFE807F05E1D021DB8F1070F8E
:10402000C6F303203BD9626A2B0A93FAA3F1B1FAD3
:1040300081F193FAA3F34FF00F0EB3FA83F38900E3
:104040000EFA01F19B0022EA010200FA03F3134386
:1040500063623B46226895FAA5F0B0FA80F095FAC3
:10406000A5F14FF0030EB1FA81F140000EFA00F015
:10407000490022EA00028B40013F1343012F2360D5
:1040800005D8636832074CBF2B43AB436360C6F36C
:10409000011229462046BDE8F041FFF785BF226A9C
:1040A00095FAA5F3B3FA83F395FAA5F14FF00F0E45
:1040B000B1FA81F19B000EFA03F3890022EA0302B0
:1040C00000FA01F313432362C3E76422024905485F
:1040D00002F032FC0023BDE784460108F8450108E0
:1040E0004446010830420108431C70B506460D469F
:1040F00004D185221B491C4802F01EFC06F00F0269
:104100001A4BC6F3031053F82240FFF791FB04FB50
:1041100004F2016802EB42030B40B3FBF2F3013BF4
:10412000012B05D8EB1E022B436809D823434360BB
:10413000032D08D101222146BDE87040FFF734BFAE
:1041400023EA04034360012DF4D0052D01D0022D94
:1041500001D10222EFE721460022BDE87040FFF7BF
:104160000DBF00BF84460108F84501084446010818
:1041700010B5224C92B000F046FC214B2360042382
:1041800006930122002306A80C9308920B9300F0DB
:1041900049FC00282DD11B4B9A6822F4F8129A6032
:1041A0009A6822F4F8129A601A6F42F480721A67C1
:1041B0000223019301A84FF48073049300F0E0FE02
:1041C00010B1114802F0D4FB104B0C4801221A60C8
:1041D0007F220023A260FF226360E26023616361AB
:1041E000A36100F0AAFF10B1094802F0C1FB12B0B0
:1041F00010BD084802F0BCFBDAE700BFC81600207B
:104200000028004000380240F84601083C0E4742B2
:1042100021470108D846010810B5154C154B2360FD
:1042200090B002A90022204601F0ADF8002201A9B9
:10423000204601F0D0F89DF80530013B0B939DF826
:1042400006300A939DF8073044330C939DF80830EC
:1042500009939DF8093008939DF80A30079307A841
:104260004FF0FF330F9304F075FD10B010BD00BF89
:10427000C81600200028004010B588B008AB194AC5
:1042800043F81C0D18491160184603F01BFE8369A2
:1042900003B907238DF80830036901338DF809301D
:1042A000C3688DF80A304369443B8DF80B3083684E
:1042B0008DF80C3043688DF80D30002403680948F0
:1042C0008DF80E30224602A98DF80F40069407940F
:1042D00000F0F0FF224603A9024800F07BFF08B07F
:1042E00010BD00BFC816002000280040044BD8684D
:1042F00010F010001CBFD868C0F34010704700BF1A
:104300000028004042681649920110B58B180468D5
:104310008C5082685A60C2689A600269DA604269A9
:104320001A61026A9A610022DA61DA849A84DA8573
:104330009A85B0F91A2001320AD108225A6118462A
:1043400001F01BFC58B10748BDE8104002F010BB5B
:10435000B0F9182001320CBF04220C22EEE710BD88
:104360001017002047470108F0B50E4685B00446F7
:1043700049493046154602F0B3FA484907462846EF
:1043800002F0AEFA0146384602F08CFA20600130A5
:1043900004D166224249434802F0CEFA2368424AD9
:1043A00093421ED002F5806293425ED0A2F5504245
:1043B00093422BD13D4B1A6A42F400321A621A6AB8
:1043C00022F400321A62002202921A6C42F4003285
:1043D0001A641B6C03F400330293029B0123636095
:1043E00014E0324B5A6A42F010025A625A6A0021B3
:1043F00022F010025A6201915A6C42F010025A6483
:104400005B6C616003F010030193019B224930460D
:1044100002F02AFA2149284602F026FA721C03D03B
:1044200001213046FFF760FE6B1C03D001212846B6
:10443000FFF75AFE4FF41653A3600023E360236195
:1044400063612362268365832046FFF75BFF226852
:10445000174B9A4207D1174B174801221A60214681
:104460004C2204F027FA05B0F0BD104B5A6A42F016
:1044700020025A625A6A22F020025A6200220392F3
:104480005A6C42F020025A645B6C03F020030393E1
:10449000039B0523A3E700BF8844010840440108AB
:1044A0005F470108C647010800100140003802407C
:1044B000004400400C170020541A00208160FFF7D0
:1044C00021BF0000034B19604168034B43F82120D2
:1044D000704700BFE8160020EC1600204368034A2E
:1044E0009B01D3581868C0F3401070471017002084
:1044F000416810B504462046FFF7F0FF0028FAD0C7
:104500008901034B5B585868C0F3080010BD00BF19
:10451000101700204368034A9B01D3581868C0F362
:10452000C01070471017002038B54468054628466B
:10453000FFF7F0FF0028FAD0A401034B1B59C1F389
:104540000801596038BD00BF1017002008B50E4A99
:10455000C36D934214D008D8A2F5806293420FD065
:104560000A4802F005FA002008BD094A934203D028
:1045700002F580629342F3D1BDE8084000F0CABC66
:10458000BDE8084000F0AEBC003C0040E247010836
:1045900000300140DFF820D0002103E0074B5B58DA
:1045A000435004310648074B42189A42F6D301F0B3
:1045B00023FDFBF71DFE704700800120C451010858
:1045C00098010020CC0B0020FEE7000008B50A4B44
:1045D0001A6842F400721A601A6842F480621A6023
:1045E0001A6842F480721A600F20FFF721FA00F077
:1045F00009FA002008BD00BF003C0240024A1368CF
:1046000001331360704700BFA01A0020014B1868E7
:10461000704700BFA01A00207047000010B5044684
:10462000002800F09F80036C23B9436480F83C307D
:10463000FFF7F2FF236CDB0600F19280236C23F47A
:10464000885323F0020343F002032364464B5A6865
:1046500022F440325A605A6861680A435A602368FB
:1046600021695A6822F480725A605A6842EA01222B
:104670005A605A68A16822F040725A605A680A4328
:104680005A609A68E16822F400629A609A680A4364
:104690009A603649A26A8A4256D0996821F07061C0
:1046A000996099680A439A609A68E16A22F04052D8
:1046B0009A609A680A439A609A68A16922F0020295
:1046C0009A609A6842EA41029A60226A002A43D0BC
:1046D0005A6842F400625A605A6822F460425A6092
:1046E0004FF4604292FAA2F2B2FA82F1626A58681A
:1046F000013A8A4002435A60DA6AE16922F47002A0
:10470000DA62DA6A013942EA0152DA629A68216BA6
:1047100022F400729A609A6842EA41229A609A688A
:10472000616922F480629A609A68002042EA8122DC
:104730009A606064236C23F0030343F00103236455
:10474000002384F83C3010BD9A6822F070629A60B1
:104750009A6822F04052AEE75A6822F40062CAE733
:104760000120EDE7012010BD002301400100000FF2
:1047700082B00023019390F83C30012B4ED00123EE
:1047800080F83C3003689A68D10705D59A68D2074B
:1047900014D4002002B070479A68214942F0010207
:1047A0009A60204A1268B2FBF1F202EB42020192D7
:1047B000019A002AEAD0019A013AF8E7026C22F441
:1047C000E06222F0010242F4807202645A685105EC
:1047D00041BF026C22F4405242F480520264026CE7
:1047E00012F480521CBF426C22F006024264002286
:1047F00080F83C206FF022021A600B4A5268D20601
:1048000008D1986810F04050C3D19A6842F08042B5
:104810009A60BFE7054A9342BBD1F2E70220B9E7AD
:1048200040420F00A8010020002301400020014069
:1048300003689A6870B5560504460D460BD59B680B
:10484000D80508D5236C43F020032364002384F8A3
:104850003C30012070BDFFF7D9FE064623681A6878
:1048600092070CD56FF012021A60226C42F40072AB
:1048700022649A6812F0405F13D0002070BD691C5A
:10488000EDD045B9236C43F004032364002384F87E
:104890003C30032070BDFFF7B9FE801B8542DDD29E
:1048A000F0E7A269002AE8D1DA6A12F4700F02D0A8
:1048B0009B685B05E1D4236C23F480732364206C34
:1048C00010F48050D9D1236C43F00103236470BDF0
:1048D0000368D86C70470000F7B50023019390F887
:1048E0003C30012B00F083800D6804688A68012346
:1048F000092D80F83C30AEB22AD906EB4603E768B2
:104900001E3B4FF0070E0EFA03FE27EA0E07E76084
:10491000E76802FA03F33B43E3604A68062A4FEA7A
:10492000820325D81344676B591F1F238B4027EA46
:1049300003036363626B06FA01F1114361632D4B5C
:104940009C4234D0002380F83C30184603B0F0BDC0
:10495000276905EB45034FF0070E0EFA03FE27EA21
:104960000E072761276902FA03F33B432361D4E76B
:104970000C2A0ED81344216BA3F123021F2393406A
:1049800021EA03032363236B06FA02F21A4322632C
:10499000D5E71344E16A413B1F229A4021EA020213
:1049A000E262E26A06FA03F11143E162C7E7122DFF
:1049B00004D1114A536843F480035360A5F11003F6
:1049C000012BBFD80C4A5368102D43F400035360E9
:1049D000B8D10A4B0A4A1B68B3FBF2F20A235343CD
:1049E0000193019B002BADD0019B013BF8E7022016
:1049F000ACE700BF0020014000230140A8010020D7
:104A000040420F0070474FF4807393FAA3F3B3FA58
:104A100083F303F1845303F560339B0001221A6092
:104A2000704700000368F7B5DD07044638D42368F3
:104A3000980771D423681E0700F1BD8023685D07C5
:104A400028D500230193A84BA84D1A6C42F0805240
:104A50001A641B6C03F080530193019B2B6843F491
:104A600080732B60FFF7D2FD06462B68DA0540F114
:104A7000C4809F4B227A1A70A368002B00F0CB8071
:104A8000FFF7C4FD984D064641F288372B6F9B0710
:104A900040F1BA80A269002A40F0CD80002015E0E4
:104AA000914B9A6802F00C02042A07D09A6802F02F
:104AB0000C02082A0CD15B68590209D58A4B1B6885
:104AC0009A03B4D56368002BB1D1012003B0F0BDC7
:104AD000884B22791A7063687BB1FFF797FD824D8E
:104AE000064641F288372B689B03A0D4FFF78EFD62
:104AF000801BB842F7D90320E8E7FFF787FD7A4D1E
:104B0000064641F288372B68980390D5FFF77EFD63
:104B1000801BB842F7D9EEE7734B9A6812F00C0F7E
:104B200007D09A6802F00C02082A16D15B68590275
:104B300013D46D4B1A68920702D5E268012AC4D1DA
:104B40001868F82292FAA2F2B2FA82F122698A4037
:104B500020F0F8010A431A606CE7E268664BDAB1AC
:104B600001221A60FFF752FD5F4D06462B689B0736
:104B70000CD52968F82393FAA3F3B3FA83F22369D7
:104B8000934021F0F80213432B6053E7FFF73EFDFB
:104B9000801B0228EAD9AEE71A60FFF737FD524DB5
:104BA00006462B689F077FF545AFFFF72FFD801B5B
:104BB0000228F6D99FE76269504B7AB101221A6048
:104BC000FFF724FD484D06466B6F98073FF536AF5B
:104BD000FFF71CFD801B0228F6D98CE71A60FFF74F
:104BE00015FD414D06466B6F99077FF527AFFFF71F
:104BF0000DFD801B0228F6D97DE7FFF707FD801B1E
:104C000002287FF632AF76E7FFF700FD801BB8423F
:104C10007FF63CAF6FE7FFF7F9FC334D064641F2F4
:104C200088372B6F98077FF535AFFFF7EFFC801BB8
:104C3000B842F6D95FE72C4DAB6803F00C03082BA4
:104C40003FF443AF2E4E0023022A33603ED1FFF7DC
:104C5000DDFC07462B68990132D447F6C07797FAF6
:104C6000A7F74FF44032B7FA87F792FAA2F24FF063
:104C70007061B2FA82F091FAA1F1226AE3691343FA
:104C8000626A02FA07F7A26A5208013A82403B437D
:104C90001343E26A144CB1FA81F102FA01F10B43B9
:104CA0006B6001233360FFF7B1FC054623689A016E
:104CB0003FF5F4AEFFF7AAFC401B0228F6D91AE72D
:104CC000FFF7A4FCC01B0228C4D914E7FFF79EFC21
:104CD00004462B689B017FF5E1AEFFF797FC001BB4
:104CE0000228F6D907E700BF0038024000700040F4
:104CF000703802400238024000004742800E4742AE
:104D000060004742194A936803F00C03042B10B566
:104D100003D0082B03D0164810BD164810BD5168AB
:104D2000536801F03F0113F4800F47F6C0745368D5
:104D300094FAA4F0B0FA80F003EA040323FA00F333
:104D400014BF0C480A48B0FBF1F05843074B4FF42E
:104D500040325B6892FAA2F2B2FA82F203F4403374
:104D6000D34001335B00B0FBF3F010BD00380240CC
:104D70000024F40000127A00564B1A6802F00F0269
:104D80008A422DE9F04105460E4630D32A68940741
:104D900037D4D0073DD44F4B1A6802F00F02964229
:104DA000C0F088802A68510700F18C80130707D56E
:104DB000494A2969936823F4604343EAC103936035
:104DC000FFF7A0FF444BF0229B6892FAA2F2B2FADE
:104DD00082F203F0F003D340404AD35CD840404B0A
:104DE00018600F20FEF724FE0020BDE8F081CAB253
:104DF0001A701B6803F00F039942C7D00120BDE869
:104E0000F0813549A8688B6823F0F00303438B6079
:104E1000BFE76A68304B012A1ED11B6813F4003FBC
:104E2000ECD02D4CA36823F003031343A360FFF7DA
:104E3000EDFB6B68012B074641F2883816D1A36859
:104E400003F00C03042BA6D0FFF7E0FBC01B40458A
:104E5000F5D90320BDE8F081911E01291B6802D815
:104E600013F0007FDCE713F0020FD9E7022B0AD121
:104E7000A36803F00C03082B8DD0FFF7C7FBC01B02
:104E80004045F5D9E5E7032B0FD1A36803F00C03E8
:104E90000C2B80D0FFF7BAFBC01B4045F5D9D8E7F3
:104EA000FFF7B4FBC01B4045D3D8A36813F00C0F29
:104EB000F6D170E7F2B21A701B6803F00F039E423E
:104EC0009CD16FE70449E8688B6823F4E0530343FF
:104ED0008B606BE7003C024000380240FC47010851
:104EE000A8010020084B4FF4E0529B6892FAA2F20E
:104EF000B2FA82F203F4E053D340044AD35C044A8A
:104F00001068D840704700BF00380240FC470108D5
:104F1000A8010020084B4FF460429B6892FAA2F26D
:104F2000B2FA82F203F46043D340044AD35C044AE9
:104F30001068D840704700BF00380240FC470108A5
:104F4000A80100200F2303600B4B9A6802F00302B4
:104F500042609A6802F0F00282609A6802F4E052BD
:104F6000C2609B68DB0803F4E0530361034B1B68DA
:104F700003F00F030B60704700380240003C024012
:104F80000368F7B5D90704463CD423689A0730D59F
:104F9000002301934A4B4B4D1A6C42F080521A6425
:104FA0001B6C03F080530193019B2B6843F48073C7
:104FB0002B60FFF72BFB06462B68D90557D5404DD4
:104FC0002B6F13F4407358D1E36803F44072B2F5C9
:104FD000407F3B4A70D1916823F0704021F4F81172
:104FE00020F4407001439160116FC3F30B030B4336
:104FF0001367206810F008001FBF334B227C1A6033
:10500000002032E0314D2E4E00232B60FFF7FEFAD8
:10501000074633681B0122D447F6C07393FAA3F303
:105020004FF0E042B3FA83F192FAA2F263688B4048
:10503000A168B2FA82F201FA02F21343C6F8843090
:1050400001232B60FFF7E2FA1D4D06462B6818017D
:105050009BD4FFF7DBFA801B0228F7D904E0FFF7A7
:10506000D5FAC01B0228D4D9032003B0F0BDFFF746
:10507000CDFA801B02289FD9F6E7E26802F440725D
:105080009342A1D02B6F124A0121116023F4407387
:10509000002111602B672B6FDA0795D5FFF7B6FA61
:1050A00041F2883706462B6F9B078DD4FFF7AEFA87
:1050B000801BB842F7D9D7E7916821F4F81192E73D
:1050C0000038024000700040E0114742680047424B
:1050D000400E47427047026838B5D36823F0A003FA
:1050E000D3600446FFF792FA05462368DB689B0607
:1050F00001D5002038BDFFF789FA401BB0F57A7F53
:10510000F3D9032038BD38B50368DA68520604467F
:1051100001D5002038BD4FF0FF32DA60FFF776FA94
:1051200005462368DB685B06F3D4FFF76FFA401B84
:10513000B0F57A7FF5D9032038BD38B50446B0B153
:10514000437F03F0FF0213B90277FFF7C3FF022387
:1051500063772368CA225A6253225A622046FFF7B5
:10516000D2FF236828B1FF225A620423637701200B
:1051700038BD9A68256922F4E00222F040029A6064
:10518000626899682A4365692A430A439A60E2681B
:105190001A611A69A16842EA01421A61DA68A169D2
:1051A00022F08002DA601A6C22F480221A641A6CEF
:1051B0000A431A64FF225A620123637738BD002331
:1051C000092803D840EA0310C0B270470A380133F7
:1051D000C0B2F5E7F8B5037F012B06460F464FF046
:1051E00002052FD0012303770368457708784D78AF
:1051F0008C789B6842BB13F0400308BFCB70FFF76D
:10520000DEFF01462846FFF7DAFF02462046FFF799
:10521000D6FFFB7840EA034040EA014040EA02241E
:105220003368CA225A6253225A623046FFF76BFF34
:1052300033680546A8B1FF225A620423737700231E
:10524000337701252846F8BD13F040034FEA0525C2
:1052500008BFCB7045EA00402043CC7840EA0444C4
:10526000DEE704F07F3424F0FE441C609A6838695D
:1052700022F480229A60FA68996802430A439A608D
:10528000DA6822F08002DA609B689B060AD4304616
:10529000FFF721FF30B13368FF225A62042373778E
:1052A0003577CEE73368FF225A62012373770023F4
:1052B0003377C7E7F8B5037F012B05464FF00206A9
:1052C00030D00123037746774B78C8788E780C78F6
:1052D000002A48D1DA0603D523F010030A334B70B5
:1052E000FFF76DFF07464878FFF769FF0246304633
:1052F000FFF765FF40EA443040EA074040EA0224F5
:105300002B68CA225A6253225A622846FFF7FBFED4
:105310002B68064640B1FF225A6204236B770023B4
:105320002B7701263046F8BD24F07F4424F0C004DA
:105330005C60DA6822F08002DA609B689B060AD41F
:105340002846FFF7C8FE30B12B68FF225A620423BB
:105350006B772E77E5E72B68FF225A6201236B7784
:1053600000232B77DEE71B0243EA0040304340EA8C
:105370004434C5E7030903EB830300F00F0000EB9F
:105380004300C0B270470368986A486070B51869F6
:105390001D6805F07F3323F0FE43C0F30E001E0CA2
:1053A0008860C3F3062406F03F0005F07F0506F091
:1053B000400608704C708D70CE7052B9FFF7DAFF5E
:1053C00008702046FFF7D6FF48702846FFF7D2FF47
:1053D0008870002070BD38B503685C6824F07F4396
:1053E00023F0C003180CC3F3042504F03F04C3F3F7
:1053F0004233C8704D708C700B7052B9FFF7BAFF12
:10540000C8702846FFF7B6FF48702046FFF7B2FF86
:105410008870002038BD03685A6822F0E0025A60A4
:105420004268B2F5827F0AD18268B2F5004F02D09D
:10543000B2F5806F03D11A6822F040021A60826AC6
:10544000B2F5005F09D11A6822F400521204120C5E
:105450001A601A6842F400521A60012380F8513031
:10546000002380F850300320704770B505460C4685
:10547000164629688B689B0701D5002070BD621C09
:10548000F8D024B92846BDE87040FFF7C4BFFFF745
:10549000BDF8801B8442ECD8F4E72DE9F041DDF83B
:1054A000188005460F4616461C462B6898683840FB
:1054B000B04202D10020BDE8F081621CF6D024B9D0
:1054C0002846BDE8F041FFF7A6BFFFF79FF8A0EB25
:1054D00008008442E9D8F3E713B50B460092802117
:1054E00000220446FFF7D9FF20B1636D43F020038B
:1054F0006365032002B010BD704738B5044600282C
:105500003BD090F8513003F0FF021BB980F85020D7
:10551000FFF7F2FF2168A568A06AA269022384F858
:1055200051300B6823F040030B6063682B43E56840
:105530002B4325692B4365692B43E5692B43256A7A
:105540002B43034302F400752B430B60120C636A78
:10555000B0F5005F02F0040242EA030208BFE36A0A
:105560004A6008BF0B61CB6923F40063CB61002064
:105570000123606584F8513038BD012038BD2DE924
:10558000F04385B099460023ADF80A3090F85030CA
:105590000C9E012B04460D46904600F045810123E8
:1055A00080F85030FFF732F894F851306168DBB280
:1055B000012B07460AD0B1F5827F40F03381A26803
:1055C000002A40F02F81042B40F02C81002D00F0A8
:1055D0001B81B8F1000F00F01781B9F1000F00F046
:1055E000138194F85130C4F83880012B04BF05238F
:1055F00084F851300023636523646364A36AA4F8CC
:105600003E90B3F5005FA4F83C902563A4F8369073
:10561000A4F83490236809D11A6822F400521204C5
:10562000120C1A601A6842F400521A601A68500686
:105630005EBF1A6842F040021A60E268B2F5006F7D
:105640006BD119B1E28E92B2012A06D135F8022B44
:10565000DA60E38E013B9BB2E3864FF00109E38EF3
:105660009BB2B3B9E38F9BB29BB9A36AB3F5005F5A
:1056700040F0AE8001220097334611462046FFF7E6
:105680000CFF002800F09D80636D43F0020363650A
:1056900035E0B9F1000F1BD0E38E9BB2C3B1226895
:1056A0009368990714D535F8023BD360E38E013B2C
:1056B0009BB2E386E38E1FFA83F9B9F1000F29D17B
:1056C000A16AB1F5005F03D1116841F48051116006
:1056D000E38F9BB263B123689A68D20708D5DB6871
:1056E00028F8023BE38F013B9BB2E3874FF00109AF
:1056F000701CB4D0FEF78AFFC01B8642AFD80325CA
:10570000012384F85130002384F85030284605B036
:10571000BDE8F0834FF00009DAE719B1E28E92B2EA
:10572000012A06D115F8012B1A73E38E013B9BB2B7
:10573000E3864FF00109E38E9BB21BB9E38F9BB266
:10574000002B92D0B9F1000F21D0E38E9BB2F3B1C0
:1057500023689A6891071AD529781973E38E013B5B
:105760009BB2E386E38E1FFA83F96A1CB9F1000F3E
:105770000AD1A16AB1F5005F04D12068016841F443
:1057800080510160154602E015464FF00009E38F95
:105790009BB273B123689A68D2070AD5DB6888F890
:1057A0000030E38F013B9BB2E38708F101084FF023
:1057B0000109731CBFD0FEF729FFC01B8642BAD86F
:1057C0009DE72368DB689BB2ADF80A30BDF80A306C
:1057D0002268956815F0100507D0636D43F0020349
:1057E00063654FF6EF73936001253A4631462046D4
:1057F000FFF73BFE002882D13A4631462046FFF7AC
:105800006BFE18B120236365012579E7A368002B9F
:105810007FF476AF03932368DA6803929B6803935F
:10582000039B6DE702256BE702256FE770470000D9
:10583000224A036890420ED0B0F1804F0BD0A2F5FF
:105840007C42904207D002F58062904203D002F57C
:105850008062904219D14A6823F070031343174ABB
:10586000904204D1CA6823F44073134318E0B0F1A6
:10587000804FF7D0124A9042F4D002F580629042F5
:10588000F0D002F580629042ECD00E4A9042E9D00E
:1058900002F580629042E5D002F580629042E1D04C
:1058A00003608B68C3620B688362044B984204BF39
:1058B0000B69036301234361704700BF000001408F
:1058C000000400400040014010B50446A0B190F82B
:1058D000393003F0FF021BB980F83820FFF7A6FF2C
:1058E000022384F839302068211DFFF7A1FF01232E
:1058F00084F83930002010BD012010BD036A10B5B6
:1059000001248C4023EA04030362036A8A401A4399
:10591000026210BD10B5044601220068FFF7EEFFD9
:105920002368064A934202BF5A6C42F400425A640A
:105930001A6842F001021A60002010BD0000014008
:10594000FFF7E8BF2DE9F0470668C2683369C1690F
:1059500023F4405313433361044683680069F268BB
:105960000343606922F41642034322F00C020B4306
:105970001343F3607369A26923F440731343B1F5D1
:10598000004F73617A4B7CD19E4203D003F5806354
:105990009E4244D1FFF7BEFA192505FB00F360686B
:1059A0004FF064094000B3FBF0F3B3FBF9F34FEAA7
:1059B0000318FFF7AFFA636868435B00B0FBF3F7C7
:1059C000FFF7A8FA636868435B00B0FBF3F3B3FB2F
:1059D000F9F309FB1373DB003233B3FBF9F35B001C
:1059E00003F4F877FFF796FA626868435200B0FB59
:1059F000F2FAFFF78FFA636868435B00B0FBF3F3DA
:105A0000B3FBF9F309FB13A3DB003233B3FBF9F368
:105A100003F0070343443B44B360BDE8F087FFF75E
:105A200061FA192505FB00F360684FF06409400036
:105A3000B3FBF0F3B3FBF9F34FEA0318FFF752FAA5
:105A4000636868435B00B0FBF3F7FFF74BFA6368EA
:105A500068435B00B0FBF3F3B3FBF9F309FB13738B
:105A6000DB003233B3FBF9F35B0003F4F877FFF7A5
:105A700039FA626868435200B0FBF2FAFFF732FA73
:105A8000B9E79E4202D03B4B9E4240D1FFF742FA1B
:105A9000676819254FF0640905FB00F3BF00B3FBED
:105AA000F7F3B3FBF9F31F01FFF734FA63686843B8
:105AB0009B00B0FBF3F8FFF72DFA636868439B0087
:105AC000B0FBF3F3B3FBF9F309FB13831B01323390
:105AD000B3FBF9F303F0F008FFF71CFA62686843C0
:105AE0009200B0FBF2FAFFF715FA636868439B0077
:105AF000B0FBF3F3B3FBF9F309FB13A31B01323340
:105B0000B3FBF9F303F00F0343EA080383E7FFF75E
:105B1000E9F9676819254FF0640905FB00F3BF0038
:105B2000B3FBF7F3B3FBF9F31F01FFF7DBF963688E
:105B300068439B00B0FBF3F8FFF7D4F96368684350
:105B40009B00B0FBF3F3B3FBF9F309FB13831B01D9
:105B50003233B3FBF9F303F0F008FFF7C3F96268DF
:105B600068439200B0FBF2FAFFF7BCF9BDE700BF53
:105B70000010014000140140704710B5044640B3C6
:105B800090F8393003F0FF021BB980F83820FFF796
:105B9000F3FF2268242384F83930D36823F40053B8
:105BA000D3602046FFF7CEFE23681A6922F49042A4
:105BB0001A615A6922F02A025A61DA6842F40052E4
:105BC000DA6000202023E06384F8393084F83A302A
:105BD00010BD012010BD00000268136823F04003CF
:105BE00010B513600446FFF788FC10B1044800F0BC
:105BF000BFFE2268136843F04003136010BD00BF6E
:105C00001C4801082DE9F04F0F4687B00446534960
:105C1000BDF94050384690461E4600F061FE50499E
:105C20008146404600F05CFE4E490190304600F04F
:105C300057FE4D498246284600F052FE019B83469E
:105C40001946484600F02EFE59468146504600F05F
:105C500029FE0146484600F025FEE065013004D1EA
:105C60005F224249424800F067FE424BE26D9A4291
:105C70004FF000033ED102933F4B5A6C42F48052E6
:105C80005A645B6C03F480530293029B232384F8D1
:105C900058303249384600F0E7FD3149404600F0BF
:105CA000E3FD3049304600F0DFFD6B1CA4F8608056
:105CB000A4F86270A4F86460A4F866504AD02A4937
:105CC000284600F0D1FDE36D23604FF482736360DA
:105CD0003823E36107220023A36063612361A36289
:105CE000E262E360236263622046FFF775FF07B05C
:105CF000BDE8F08F21498A420CD103931E4B1A6CE8
:105D000042F480421A641B6C03F480430393039BA8
:105D10002423BCE71A498A420CD10493164B1A6C0F
:105D200042F400421A641B6C03F400430493049B86
:105D30003323ACE713498A42ABD105930E4B5A6C1F
:105D400042F400525A645B6C03F400530593059BC4
:105D500054239CE74FF40073A361B4E77443010834
:105D60002C430108BC4301080444010832480108DF
:105D70008B480108003001400038024000380040E4
:105D8000003C00400034014010290CBF4FF400617A
:105D90000021012AC16016D0022A17D0CAB90261B7
:105DA00042618269B2F5007F05D0002B14BF00224A
:105DB0004FF480228261002B14BF00234FF48273C2
:105DC0004360FFF709BF00210161E9E7026100229A
:105DD000E6E7022202610122E2E7000070B5044614
:105DE0000E46FEF7B3FB0023022290FBF2F0B04216
:105DF000DDB203DD0133082B09D10725054B33F84C
:105E00001530E3612046BDE87040FFF7E5BE90FB2A
:105E1000F2F0ECE70C4801087FB506AA002342F82F
:105E2000043DC3680391B3F5006F4FF00A0300937C
:105E300003A90CBF02230123FFF7A1FB18B90598A2
:105E400007B05DF804FB4FF0FF30F9E77FB50F2393
:105E50000193022100234FF4805201A80291039381
:105E600004920593FEF788FFB0FA80F0400907B06E
:105E70005DF804FB174A1849936803F00C03042BE0
:105E800010B50DD0082B0DD0144B0B60114B144ADC
:105E90009B68C3F30313D25C0B68D3400B6010BD47
:105EA000104BF2E75468506852686302C2F38812DC
:105EB00000F03F004CBF0B4B084BB3FBF0F35343D8
:105EC000044A5268C2F3014201325200B3FBF2F3BA
:105ED000DBE700BF00380240A80100200024F400E6
:105EE000A648010800127A0000B58FB01B4B0021B4
:105EF00000911A6C42F080521A641B6C184A03F02D
:105F000080530093009B0191136823F4404343F4B2
:105F100000431360136803F440430193019B012382
:105F20000293B8B90393022308934FF480030993B3
:105F300008230A934FF4A8730B9304230C9302A82D
:105F400007230D93FEF76EFD30B9FFF77FFF0FB00B
:105F50005DF804FB0523E5E70020F8E70038024080
:105F60000070004010B58EB000241A4B00941A6CDB
:105F700042F080521A641B6C174A03F0805300935E
:105F8000009B0194136823F4404343F400431360DF
:105F90001368039403F440430193019B0994032382
:105FA000029301230593102306930A934FF4A873D9
:105FB0000B93042302220C9302A8072308920D934B
:105FC000FEF730FD18B9FFF741FF0EB010BD2046B7
:105FD000FBE700BF003802400070004008B5012018
:105FE000FFF782FF30B9FFF77FFF18B9FFF7BAFF5D
:105FF00000B9FEE708BD0000174AD2F8883010B596
:1060000043F47003154CC2F888302368002143F034
:1060100001032360A160236823F0847323F4803399
:1060200023600F4B6360236823F4802323604FF0C9
:106030000063E16093600B4B0B4A1A60FEF7C6FAEF
:10604000FFF7CCFF236A43F008032362236A23F09F
:106050000803236210BD00BF00ED00E000380240DD
:1060600010300024A80100200024F400054B18681B
:1060700030B901221A60044B044A1A60FDF7D8BCFB
:10608000704700BF10190020A41A0020000C004027
:1060900008B5044B1B680BB9FFF7E8FF024B586AC1
:1060A00008BD00BF10190020000C0040044B054A39
:1060B00013605863DA6842F00202DA60704700BF8A
:1060C000000C0040A41A0020034B044A1360DA6855
:1060D00022F00202DA607047000C0040A41A00208F
:1060E000034A044B13606FF002021A61704700BF4D
:1060F000A41A0020000C004010B5044600F05EFD1C
:1061000023682BB9E06800F0DFFA012360602360A8
:10611000BDE8104000F07EBD38B5054600F04EFDEC
:106120002C6824B1E86800F0CFFA6C68041B00F01A
:1061300071FD204638BD10B5044600F03FFD2046F5
:10614000FFF7EAFFA36818440023A0602360BDE8BE
:10615000104000F05FBD38B5054600F02FFD284621
:10616000AC68FFF7D9FF044400F054FD204638BD69
:1061700008B5FFF7F0FF4FF47A7390FBF3F008BD1A
:1061800010B5044600F01AFDE06800F09DFA002307
:106190006060A360BDE8104000F03CBD002310B576
:1061A000036043608360044600F0D8FBE060204653
:1061B000FFF7E6FF204610BD10B5002303604360E3
:1061C0000A782F2A04460DD14A785AB1481C20601B
:1061D000194623681A782F2A06D10133236000F06C
:1061E00099F86060204610BD002AF8D001330131D3
:1061F0002360EEE7406808B520B100F03BF8B0FA44
:1062000080F0400908BD10B50446FFF7F3FF00B168
:10621000606810BD4068003018BF012070470368F7
:106220009B681847074B10B50360002343608360E9
:10623000C360044600F092FB0349206100F0D7F9E7
:10624000204610BDC04801081F62000803460A46E8
:10625000011D006900F0F7B9011D006900F014BAD2
:1062600010B5034B03600446FFF7F6FF204610BD50
:10627000C0480108007B704738B504460A4B0360EC
:10628000002343600D46A16002730848FCF732FD0D
:1062900045B1074B1A6862601C600448FCF72AFD90
:1062A000204638BD6560F8E7D44801082019002071
:1062B0001C19002010B50F4B036004460E48FCF774
:1062C00019FDA3682BB10D4A13689C420CD1636879
:1062D00013600948FCF70EFD237B13B92046FDF738
:1062E000BBFD204610BD13465A689442FBD162683C
:1062F0005A60EEE7D4480108201900201C1900203C
:1063000010B50446FFF7D6FF2046FDF7A3FD204653
:1063100010BD000070B506460C480D46FCF7EAFCBF
:106320000B4B1C685CB1A06870B12A46314603F083
:1063300035FE48B9A06803F0C3FD854204D1034887
:10634000FCF7D8FC204670BD6468EBE720190020FC
:106350001C1900200368DB69184703685B6918474C
:1063600003689B6A184770477047F8B503689B6BD2
:106370000E4604468F1898473546BD4207D023681D
:1063800015F8011B1B6C204698470130F5D1236896
:106390002046DB6B9847A81BF8BDF8B503689B6BDC
:1063A0000E4604468F1898473546BD4208D02368EC
:1063B00020465B6C9847431C02D005F8010BF4E7BC
:1063C00023682046DB6B9847A81BF8BD0020704768
:1063D0000020704770470020704700207047000081
:1063E0001FB504460022FFF747FF094B2360002337
:1063F00023612246074901A803F060FA064901A873
:1064000001F09EF82061FDF7FEFC204604B010BDAF
:10641000304901083F4601082449010810B5064BE0
:1064200003600446006900F08DFE044B23602046A3
:10643000FFF740FF204610BD30490108E44801083D
:106440000EB477B5036807AD044655F8046B9B6B33
:1064500098472069019500F037FF019A206931467D
:1064600007F0A2FF23680546DB6B204698472846C5
:1064700003B0BDE8704003B0704700004369416855
:1064800070B504461944FFF7E1FE636A04F118058C
:106490002BB940F21F220549054800F04DFA636A06
:1064A00028461B68BDE87040184700BF78490108BE
:1064B000CF49010838B504460D4600F07FFB204661
:1064C000FFF7CAFE6561206900F0FEF82918204632
:1064D000FFF7BCFEBDE8384000F09CBB7FB5064628
:1064E00006F1180400F06AFB6D463046FFF7B4FE73
:1064F0000023AC4203930BD02046FCF712FD3CB1C5
:10650000039B1BB15B68694620469847039B7362F7
:106510002846FCF706FD00F07DFB04B070BD704717
:10652000A0F1BC00FFF7FBBFA0F1BC00FFF7F7BF75
:1065300000F018BCA0F1BC00FFF7FABF00F015BCDA
:10654000A0F1BC00FFF7FABF38B504461D46049B16
:1065500000F024FC294604F1BC00FFF741FF044B86
:1065600003F1080228332260C4F8BC30204638BD4D
:10657000E849010870B50E4604461546FDF7DEF9F8
:10658000013609D020460021FDF7FCF929462046B6
:10659000BDE87040FDF7F2B970BD38B504460D4650
:1065A00003685AB18268136020460121FDF7EAF9B9
:1065B00029462046BDE83840FDF7E0B9C2681B0413
:1065C000F1E70022FFF7D6BF70B50E460446154628
:1065D000FDF7B4F9013606D02A4620460021BDE871
:1065E0007040FFF7DABF70BD0022FFF7EDBF38B58E
:1065F000036804461B680D46984763681D6038BDF4
:10660000036870B5DB680446984763685A68236876
:106610001AB99B68BDE8704018475B6815689847D1
:106620006368281A00285A6807DC916859601B685B
:10663000002BEAD050689847E7E7236810681B6989
:10664000BDE870401847F8B506460C461F4615468B
:1066500000F0B4FA706884E8A0004368002153B9E0
:10666000A36079B9336844601B6928469847BDE840
:10667000F84000F0CFBA1A68AA1A002AF0DB1946CF
:106680009B68ECE78C60F2E738B505460C4600F0F5
:1066900095FA6A685368A3420ED19B6853602A68D2
:1066A0002BB993689847BDE8384000F0B3BA126937
:1066B00018689047F7E71346002BF4D09A68944285
:1066C000F9D1A2689A60EEE703685B6818477047E3
:1066D00070B50446074B44F8043B054600F14406F8
:1066E00054F8040B08B1FDF7B5FBB442F8D12846C5
:1066F00070BD00BF604A010810B50446FFF7E8FF0F
:106700002046FDF7A7FB204610BD00002DE9F04113
:1067100088B00546ADF80430BDF93830ADF8063024
:10672000BDF93C30ADF80830BDF94030ADF80A3065
:10673000BDF94430ADF80C30BDF94830ADF80E303D
:10674000BDF94C30ADF81030BDF95030ADF8123015
:10675000BDF95430ADF81430BDF95830ADF81630ED
:10676000BDF95C30ADF81830BDF96030ADF81A30C5
:10677000BDF964301948ADF81C300024BDF968300B
:106780002860ADF80010ADF80220ADF81E306C6442
:106790002F1D3DF91480B8F1FF3F1DD01C20FDF7DF
:1067A00049FB002106461C2202F082F94146304690
:1067B000FFF71AFFB8F1FF3F47F8046B05D001233C
:1067C00003FA04F26B6C13436B640134102CE0D1B8
:1067D000284608B0BDE8F0810026EBE7604A0108D2
:1067E00070B50446054654F8043B9B680E4698472E
:1067F000002354F8040B48B146FA03F212F0010FDB
:10680000026812BF8168C16812040A600133102B4C
:10681000EFD12B682846DB68BDE87040184770B59B
:106820000446064654F8043B9B68984700231D46DF
:1068300054F8042B42B1516812680968114214BF20
:10684000012200229A4015430133102BF0D1336806
:106850003046DB689847284670BD10B50446FFF700
:10686000BFFF204610BD000010B5044601300DD119
:1068700010BD9C4209D120468968FDF79DFB20464A
:106880000021BDE81040FDF72FBC0C31B1F90030FC
:106890005A1CEED10248BDE8104000F069B800BFB4
:1068A000BF4A0108884208B508D0431C06D0013110
:1068B00006D0044800F05CF84FF0FF31084608BDF0
:1068C0000146FBE78E4A0108B1F900305A1C01D19C
:1068D00018467047834201D1486870470C31F3E78E
:1068E000421C10B5044607D0FFF7EEFF431C0446D8
:1068F00002D1024800F03CF8204610BD9F4A010832
:10690000B1F900305A1C01D118467047834201D1B9
:10691000886870470C31F3E7421C10B5044607D075
:10692000FFF7EEFF431C044602D1024800F020F8B6
:10693000204610BD704A010870B504460D46164643
:1069400000F03CF933462A4621460348FDF710F98A
:10695000BDE87040FDF7CCB8D04A01080048704748
:10696000044B01080148FFF74BBE00BF044B010870
:106970000FB407B504A951F8040B0191FDF7CEF847
:106980000120FDF73BFA10B480B1146853680CB9CC
:10699000DA070BD513F0010F4FEA63031CBFC2588F
:1069A0001459184423465DF8044B18475DF8044B0E
:1069B00070470000064B19681A1D01B91A601B6860
:1069C000934204D0592203490348FFF7B5BF7047EB
:1069D00094190020204B0108AA400108036870B5F3
:1069E0000D4E5B680446984733689C420ED0251DC7
:1069F0000023D4F8D020D4F8CC102846FFF7C4F9EF
:106A0000D4F8D4102846FFF7E9F93460236820460B
:106A10009B68BDE8704018479C190020036870B55A
:106A20005B6804460E4615469847084BC4F8CC6090
:106A30002046C4F8D05000221A60FFF7CFFF236829
:106A400020469B68BDE87040184700BF9C19002095
:106A5000036870B55B6804460D469847064BC4F85A
:106A6000D450204600221A60FFF7B8FF2368204662
:106A70009B68BDE8704018479C19002038B5036832
:106A800004465B680D4698472046FFF7A7FF294656
:106A9000201DFFF7C1F9236805469B6820469847EB
:106AA000284638BD2DE9F04305469946224B45F866
:106AB000043B044685B00F469046002190222846AC
:106AC00001F0F6FF002204AB0292039213E90300E7
:106AD00004F19806194B86E80300C4F8A03048F288
:106AE0000703C4F8A430164BC4F8AC20C4F8A8407F
:106AF000C4F8B060C4F8B430BFF36F8FBFF34F8FEA
:106B00000823C4F8CC300F4BC4F8D430BDF9303072
:106B1000C4F8C42084F8C820C4F8D02000934246AA
:106B20004B4639462846FFF76DF82046FFF756FFDB
:106B3000204605B0BDE8F083844B010801A090E831
:106B40008769000840420F0038B5044648B1583004
:106B5000A04206D0A0F12C051438FCF7C5F9284650
:106B6000F6E7204638BD000070B50E4C20460025E3
:106B700028263246294640F8045B01F099FF324648
:106B8000294604F13000E56201F092FFA565204638
:106B9000E565054A84F860500449BDE87040FDF79A
:106BA0002BB900BF3019002098010020496B000864
:106BB000EFF31080C04300F00100704738B5FFF7D5
:106BC000F7FF054672B60E4C236823B980F0010327
:106BD0000C4ADBB213702368013304D135220A4911
:106BE0000A48FFF7A9FE23682BB125B139220649CF
:106BF0000748FFF7A1FE23680133236038BD00BFBB
:106C0000A4190020A0190020984B0108E94B0108A5
:106C10000F4C010810B50A4C236883B1FFF7C8FF79
:106C200020B14A2207490848FFF786FE2368013B46
:106C3000236023681BB9054B1B7803B962B610BDEE
:106C4000A4190020984B01080F4C0108A01900203E
:106C500038B50446FFF71CFA0546FFF719FA401B42
:106C6000A042FAD338BD000007EE100ADFED047A27
:106C700067EE277AFDEEE77A17EE900AFFF7E8BF96
:106C8000002474494FF47A735843FFF7E1BF0000C2
:106C900010B504460748FCF72DF8074B1B6803B1F5
:106CA0009847064B1B680BB1204698470148FCF7F4
:106CB00021F810BDA8190020B4010020AC0100206B
:106CC00038B505460A48FCF715F80A4B1B681BB196
:106CD000984708B9FFF7DCFF074B1C680CB1A047C9
:106CE000044605B12C600248FCF704F8204638BD84
:106CF000A8190020B0010020B8010020704770479B
:106D0000704710B480B1146853680CB9DA070BD51A
:106D100013F0010F4FEA63031CBFC2581459184403
:106D200023465DF8044B18475DF8044B704700009C
:106D3000090170B5441801F19805D4F8A430054450
:106D40002BB940F21F2205490548FFF7F5FDD4F89D
:106D5000A43028461B68BDE87040184778490108F0
:106D6000CF4901084C30FDF7C3BB10B54C300C4681
:106D7000FDF7DAFB204610BD884238B504460D46C3
:106D80000AD0FCF7CEF83CB1EB681BB15B68294632
:106D900020469847EB68E360204638BD2DE9F04374
:106DA00087B0002591460095024601950446884625
:106DB0001F469DE80300274B42F8083B264B82E81C
:106DC0000300236148F207036361244BE561A4617A
:106DD00022626362BFF36F8FBFF34F8F04F14C06E3
:106DE0004C226563656484F8485084F84950304605
:106DF00001F05EFE02A9C4F8A450C4F8B450C4F86F
:106E0000B870174D174F029704F198000595FFF7DA
:106E1000B3FF02A8FCF785F802A904F1A8000297C5
:106E20000595FFF7A9FF02A8FCF77BF84A46414603
:106E30003046FDF799FAD4F8B8103046FDF73EFB1E
:106E4000304622460849FDF73DFB204607B0BDE825
:106E5000F08300BF2C4C010801A090E8036D0008EE
:106E6000C0400108FD6C0008316D00082DE9F04FAD
:106E70008BB004460D4600F055F8284B93F900A05E
:106E8000BAF1FF3F06460F4612D022462B46204657
:106E900029460CF0B9FC834650B94FF000084FF07A
:106EA00000092046294642464B460CF085FC20B995
:106EB000304639460BB0BDE8F08F194BCDF820B005
:106EC0000122CDE90445CDE902458DE80C00BAF177
:106ED000000F15D042464B46404649460CF024FB75
:106EE000BAF1020FCDE906010CD100F0E3F821233D
:106EF0000360089B63B9DDE906010BB0BDE8F08FC4
:106F0000CDE90689684600F0CFF80028F1D1ECE71A
:106F100000F0D0F8089B0360EDE700BFBC01002043
:106F20003C4C01082DE9F0415E4EB6460E407645D8
:106F300004460D4600F0948000290B46024672DD9F
:106F40000F157DD0A7F2FF37C3F31303F80743F4FF
:106F5000801363D403EBD27100260B447F105200E0
:106F6000B64616204FF400110EEB01049C424FEA86
:106F7000D2754FEA420203DC1B1B04EB010E0E44E8
:106F8000013805EB43034FEA5101EDD1844620243B
:106F90004FF0004109E020D003EBD275013C4FEAED
:106FA00051012B444FEA420220D09E4501EB0C05D3
:106FB000F1DA002D05EB010C09DBF0469542CEEB32
:106FC000030300D9013B521B0844C646E4E7BCF169
:106FD000000FF2DB0EF10108F0E795421CD8002DFE
:106FE00005EB010C48DB98460023ECE7134304D083
:106FF000411C45D000F00104204444087310F207FE
:1070000003F17F5303F5001348BF44F0004403EB42
:1070100007512046BDE8F0817346BDE75B0003EBF6
:10702000D273520096E721F00046064322D071BB8E
:107030000F46D30A153F5205002BFAD0DD0221D4AA
:10704000002100E001465B00DC0201F10100F9D5FE
:10705000C0F1200422FA04F423437F1A824071E72E
:1070600002460B460CF036F922462B460BF080FF09
:10707000BDE8F081BDE8F081BCF1000FAADAB2E70B
:107080000136BBE720244FF0FF310020E2E7024643
:107090000B460BF06BFF02460B460CF045FABDE8C1
:1070A000F08100BF0000F07F002070470A2200211D
:1070B00003F0A6B8014B1868704700BFE805002030
:1070C00000293DD070B505460C4608B1836B7BB3F3
:1070D000B4F90C300BB9002070BD2146284600F0F1
:1070E00039F8E36A064633B1E16928469847002833
:1070F000B8BF4FF0FF36A3891B061CD4216B41B1EA
:1071000004F14003994202D0284600F083FA00239C
:107110002363616C21B1284600F07CFA002363648C
:1071200000F0C4F90023A38100F0C2F9304670BD1D
:1071300000F0B6F9CCE72169284600F06BFADDE7EC
:1071400000207047024B01461868FFF7B9BF00BF27
:10715000E8050020B1F90C309AB22DE9F0410D4656
:10716000110780463CD46A6843F40063002AAB816F
:1071700073DDAC6A002C4BD09BB203F4805200212B
:1071800092B2D8F80060C8F80010002A69D02A6DC1
:107190005F0705D569682B6B521A0BB1EB6BD21ADE
:1071A0000023E9694046A047441C3CD0B5F90C30A7
:1071B0002A692A6023F400630022AB81DB046A6041
:1071C00049D4296BC8F8006011B305F14003994216
:1071D00002D0404600F01EFA00202863BDE8F0818E
:1071E0002E69AEB12C682E6090070CBF6B6900232E
:1071F000A41BAB600AE0234632466F6AE969404649
:10720000B8470028A4EB0004064404DD002CF2DC9F
:107210000020BDE8F081AB8943F04003AB814FF023
:10722000FF30BDE8F081D8F800201D2AF3D81A4BB2
:10723000D34003F0010383F00104002BEBD0B5F938
:107240000C302969296023F40063D9046C60AB8198
:10725000B7D5002AB5D12865B3E7EA6B002A88DCE8
:10726000D6E70123E9694046A047431C024602D005
:10727000AB89AC6A8CE7D8F80030002BF8D01D2B16
:1072800001D0162B02D1C8F80060C1E7AB8943F0EA
:107290004003AB81BDE8F0810100402010B50446F9
:1072A00082B008B1836B53B1B1F90C0008B902B0D8
:1072B00010BD204602B0BDE81040FFF74BBF019162
:1072C00000F0EEF80199EFE720B1054B0146186890
:1072D000FFF7E4BF034B0449186800F0A1BD00BFED
:1072E000E8050020444C01089D720008014900F0A7
:1072F00097BD00BFC17000082DE9F04F354B4568C0
:10730000C3630024074600F53B7204230321C0F841
:10731000E412C0F8E822C0F8E04283B02C606C6050
:10732000AC606C66EC812C616C61AC61AB81214618
:1073300005F15C00082201F0BBFBBE68DFF898B0E5
:10734000DFF898A0DFF89890DFF89880C5F820B0B3
:1073500001230922C5F824A0C5F82890C5F82C807F
:10736000ED612146F381B28106F15C003460746006
:10737000B460746634617461B4610822019301F0F1
:1073800097FBFD68F66112200222C6F820B0C6F80D
:1073900024A0C6F82890C6F82C802146A881EA814E
:1073A0002C606C60AC606C662C616C61AC6105F14A
:1073B0005C00082201F07CFB019BED61C5F820B068
:1073C000C5F824A0C5F82890C5F82C80BB6303B08D
:1073D000BDE8F08FED7200086199000889990008F6
:1073E000C5990008E599000870B568234D1E03FB98
:1073F00005F50E4605F1740100F01CFF044640B18E
:1074000000210C30666005F168022160A06001F087
:107410004FFB204670BD00BF204B70B51D68AB6BA5
:10742000064613B92846FFF767FF05F538756B6800
:10743000AC68013B05D521E0013B5A1C04F168040E
:107440001CD0B4F90C20002AF6D1002501234FF6F8
:10745000FF72E281A38165662560A5606560256194
:107460006561A5612946082204F15C0001F020FB5A
:10747000256365636564A564204670BD2B680BB108
:107480001D46D4E704213046FFF7AEFF286008B15F
:107490000546CCE70C23336070BD00BF444C0108A7
:1074A000836B03B17047FFF727BF00BF704700BF72
:1074B000704700BFF0B5134683B00F4601AA1946C6
:1074C000064608F0ABF8F0B105463046FFF7A4FFDA
:1074D0000446C0B139464FF4DB73019A304601F0DF
:1074E0000FFE00281BDB124B124F1349134AE362B5
:1074F000EB05E081A581E46127626162A26205D4A7
:10750000204603B0F0BD002003B0F0BD304602239A
:107510000022214600F066F9204603B0F0BD0025A8
:10752000FFF7C4FFA581FFF7C3FF2846E9E700BFC7
:10753000E59900086199000889990008C599000833
:10754000024B0A4601461868FFF7B4BFE805002061
:107550000EB410B583B005AB064C53F8042B019361
:107560000146206805F084FB03B0BDE8104003B07D
:10757000704700BFE8050020F8B5234F0C460646CB
:10758000FCF748FCBB685D6825F00305291B01F684
:10759000EF7121F47F6121F00F01A1F58054B4F562
:1075A000805F07DB0021304602F078F8BB682B448F
:1075B000984204D03046FCF731FC0020F8BD61420F
:1075C000304602F06BF801300DD0104BBA681968E4
:1075D0002D1B45F001053046091B55601960FCF76D
:1075E0001DFC0120F8BD0021304602F057F8BA68B2
:1075F000831A0F2BDEDD064C0449246843F0010397
:10760000001B53600860D5E7EC050020BC19002082
:10761000F8090020002945D02DE9F0410D468046AB
:10762000FCF7F8FB55F8047C6A4927F00103A5F143
:107630000804E2188E685068B24220F0030062D05D
:10764000FE0750600BD455F8087CE41B01F1080ECE
:10765000A56875453B446FD0E768EF60BD601518BD
:107660006D68ED0742D543F001026260E350B3F567
:10767000007F18D2DB085A1C4D6851F83270A760A1
:1076800001209B1000FA03F301EBC2001D430838F0
:10769000E0604D6041F83240FC604046BDE8F0419A
:1076A000FCF7BCBB70475A0A042A53D89A0902F166
:1076B00039077F0002F1380501EB870051F82720D8
:1076C0004449083890424DD0516821F003018B4263
:1076D00002D292689042F7D1D068E060A2608460E4
:1076E000D4604046BDE8F041FCF798BB95683A4F3E
:1076F000BD4203443FD0D068E86043F0010285609A
:107700006260E350B3E7FF07034407D455F8082C41
:10771000A41A1344A068E268C26090602F4A1268FD
:1077200043F00100934260608C60B6D32C4B40461E
:107730001968FFF721FFB0E711184968C90744D459
:107740009168D268CA60034443F0010091606060B0
:10775000E350A2E7142A17D802F15C077F0002F178
:107760005B05A9E7AA104B68012505FA02F213434D
:107770004B600246B1E743F001024C610C61E560E9
:10778000A5606260E35088E7542A06D81A0B02F11C
:107790006F077F0002F16E058EE7B2F5AA7F06D86B
:1077A000DA0B02F178077F0002F1770584E740F2F7
:1077B0005450824206D89A0C02F17D077F0002F1F4
:1077C0007C0579E7FE277E2576E743F001026260BB
:1077D000E35062E7EC050020F4050020F4090020E6
:1077E000B819002000F000B82DE9F04F0C4691B018
:1077F00091461E46054610B1836B002B74D0A389B9
:1078000003F48473B3F5847F76D0D4F82880B8F17C
:10781000000F00F04181012E4BD0022E08D03EB166
:1078200016232B604FF0FF37384611B0BDE8F08FBC
:107830004FF0000A23695746002B00F01881B4F975
:107840000C2040F61A0391B20B4043B949055FD4AE
:10785000944B984500F0F78042F40062A2812146E3
:107860002846FFF71BFD07460028DBD133464A4672
:10787000E1692846C0470130D4D0216B41B104F101
:107880004003994202D02846FFF7C4FE0023236339
:10789000A3892269226023F402630021A38161602D
:1078A00004F15C00082201F003F9384611B0BDE88C
:1078B000F08F21462846FFF7F1FCA38903F480529C
:1078C00092B2002A00F0B580276D5E075DD41807DC
:1078D00040F1AD80226823690AB1D21A1744B94435
:1078E0004FF0010A0026A7E7FFF7DAFDA38903F4AA
:1078F0008473B3F5847F88D121462846FFF7CEFCF8
:1079000083E7A3894FF4806243F48063A381E26438
:10791000002E43D1CB46BAF1000F4ED1A389DA0431
:1079200040F1AA80206D6368216BC71A002900F01E
:10793000AC80E26BBF1A1F442069A36B1B1AFF1AAD
:107940001344BB453FDBFA185A453CD9C7EB0B073C
:107950003844DB1B84E8090041B104F1400399423B
:1079600002D02846FFF756FE00232363A38923F0A5
:107970002003A38104F15C000822002101F098F8A3
:107980000027384611B0BDE8F08F6268236BBF1A3C
:10799000002B4CD0E26B2369BF1AA0E701AAB4F90F
:1079A0000E10284600F080F800287FF458AF059BA1
:1079B00009EB030BBAF1000FB0D0216B636800290B
:1079C00063D0E26BB7E7E76CE1697F4207EA0B0738
:1079D0003A4600232846C04701303FF440AF2369B0
:1079E000216B23600023636041B104F1400399429D
:1079F00002D02846FFF70EFE00232363A389BBEBCA
:107A0000070B23F02003A381B4D02146284601F0C0
:107A1000BBFD00287FF423AF626893453FF61FAF9C
:107A20002368CBEB02025B4462602360A2E7236918
:107A300055E73346E1692846C047431C07463FF4F3
:107A4000F1AEA38941E7B4F90E100029FFF604AFA7
:107A500001AA284600F028F830B9029B03F47043CD
:107A6000B3F5004F3FF44DAFB4F90C20F4E62146D6
:107A7000284600F08BFBE2E601235246E1692846E6
:107A8000C047431C7FF44FAFE9E622682069121A11
:107A9000BF1A1344002154E71D232B604FF0FF371A
:107AA000C2E600BFC599000838B50B46074C05462D
:107AB0001146184600232360FCF748F9431C00D008
:107AC00038BD2368002BFBD02B6038BDE01A0020A6
:107AD0009368002B76D02DE9F04F8B8985B00C464A
:107AE00019070190164629D522693AB303F0020816
:107AF0001FFA88F0356800282FD04FF00009B44FE6
:107B0000C846B246B84543464A4628BF3B46019858
:107B1000B8F1000F50D0E169666AB047002871DD06
:107B2000DAF808301B1A8144C0EB0808CAF808309C
:107B3000002BE7D1002005B0BDE8F08F2146019869
:107B400006F02AFD002840F03A81A389356803F049
:107B500002081FFA88F00028CFD113F001095BD189
:107B60004F4602961FB39A05D4F808802CD5474596
:107B7000C246C0F0A48013F4906F40F0B18020683A
:107B80005246494600F030FFA0682368C8EB000069
:107B90005344A06023603846029A93681B1A8144BC
:107BA0003F1A9360002BC5D0A389002FDBD1D5F8F5
:107BB00000906F680835D5E7D5F80090D5F80480B7
:107BC00008359FE70020704720682369984203D852
:107BD00061698F4280F0B780B84528BFB8464246F9
:107BE000494600F001FFA3682268C8EB0303424442
:107BF000A3602260002B49D121460198FFF74EFB7C
:107C0000002843D0B4F90C3043F040034FF0FF306C
:107C1000A38105B0BDE8F08F804602908246814680
:107C2000B9F1000F2AD0029B002B4CD020682369A9
:107C30006269C845C34628BFCB4698425F4604D90F
:107C4000A36813449B4500F39080934520DB1346C3
:107C5000676AE16901985246B847071ED2DDB8EB62
:107C6000070823D0B368DB1BBA44C7EB0909B3602C
:107C7000002B3FF45FAFB9F1000FD4D10023D5F84A
:107C800000A0D5F8049002930835C9E7404683E781
:107C90005A46514600F0A8FEA2682368CBEB0202C8
:107CA0005B44B8EB0708A2602360DBD12146019852
:107CB000FFF7F4FA0028A5D1CDF80880D2E72068B4
:107CC000B846BA465CE74A460A21504600F070FDC5
:107CD00000286FD001300123CAEB00080293A5E70A
:107CE00062692068216902EB4208C1EB000A08EBD7
:107CF000D8780AF101004FEA680838444045424606
:107D000084BF804642465B0542D51146019800F08B
:107D100091FA8346002855D05246216900F0CAFDE9
:107D2000A38923F4906343F08003A381CAEB080383
:107D30000BEB0A00C4F81480C4F810B02060A360F4
:107D4000B846BA461CE76FF00043BB4228BF3B462B
:107D50004A4693FBF1F30198666A01FB03F3E1697C
:107D6000B04700283FF718AF4CE71A465146039337
:107D700000F03AFE2268039B01981A4422602146D3
:107D8000FFF78CFA039B00287FF43CAF1F4666E7A1
:107D9000019801F0FFF983460028C7D1019D2169B0
:107DA0002846FFF737FCB4F90C300C2223F080038F
:107DB0002A6029E7012309F10108029336E74FF011
:107DC000FF30B8E6019A0C231360B4F90C301BE7BE
:107DD00000FCFF7F2DE9F04110F538771BD0884675
:107DE00000267D68BC68013D0FD4A389012B05F1F5
:107DF000FF3506D9B4F90E300133204601D0C04713
:107E000006436B1C04F16804EFD13F68002FE8D1F2
:107E10003046BDE8F0813E463046BDE8F08100BF07
:107E20002DE9F84310F538771FD0884606464FF005
:107E300000097D68BC68013D11D4A389012B05F1BF
:107E4000FF3508D9B4F90E3001332146304602D04F
:107E5000C04749EA00096B1C04F16804EDD13F6892
:107E6000002FE6D14846BDE8F883B9464846BDE84C
:107E7000F88300BF70B50F4E0F4D761BB61018BFBC
:107E8000002405D0013455F8043B9847A642F9D1A7
:107E90000A4E0B4D761B0BF0F1FEB61018BF0024F6
:107EA00006D0013455F8043B9847A642F9D170BD7D
:107EB00070BD00BFB40B0020B40B0020C40B002029
:107EC000B40B0020024B19687C3100F003B800BFEE
:107ED000E80500202DE9F8430C46064607F01EFC95
:107EE00021468046304607F01DFC476907F26C7753
:107EF000B907044600F0C880FA17874B83FB0713C5
:107F0000C2EBE3124FF4C87303FB1273B3FA83F3AB
:107F10005B095A00814D134405EB031504F00CFD79
:107F200004F00EFD7E4B1B6843B3D8F804309F422B
:107F300005D0384604F036FC002800F0B380D8F8AD
:107F4000003083B93368D8F81C20934280F2AE80A9
:107F5000D8F838209342B4BF0123002323620EDAFD
:107F6000D8F83C000DE03368D8F81C20934204DBBD
:107F7000D8F838209342C0F2998000232362D8F8C1
:107F80002000684A684EA76880FB0289C11700EB91
:107F900009034FF4616EC1EBE3230EFB130383FB74
:107FA000068982FB00E24FEAE37C03EB090E024400
:107FB000CCEB6E1E86FB0306C1EBE222CEEB0E1E5F
:107FC00021681E44A3EB8E03CB1A61682360CCEBBF
:107FD0006616BA1A891B3B2BA26061604DDD013128
:107FE0003C3B616023603B2940DD01323C39A260AB
:107FF0006160172A1DDDA369E1690133062BC8BF43
:108000000023A361E3680131E161183A013321697A
:10801000A260E36055F82120934205DD01319B1AEF
:108020000C29E36045D0216104F088FC2046BDE8BE
:10803000F883002AF8DAA369E169013B48BF062307
:10804000A361E36801391832013BE161A260E3609A
:10805000002BE9D12369013B32D423619B00EB580B
:10806000E36004F06BFC2046BDE8F8830029C0DA29
:10807000013A3C31A2606160BBE7002BB3DA013901
:108080003C3361602360AEE7234BFA1783FB071391
:10809000C2EB6313642101FB1373002B3FF42DAF7C
:1080A000012336E74FF0FF33236268E701232362A1
:1080B00056E763690022013363612261E261B3E73D
:1080C00063695A1E0B2162619207216113D003F28A
:1080D0006B71CA17104B83FB0103C2EBE3124FF421
:1080E000C87303FB1213B3FA83F35B0903F5B6738A
:1080F000E3612C23B3E7084A03F26B7182FB01238F
:10810000CA17C2EB6313642000FB1313002BE1D0EA
:1081100040F26D13ECE700BF1F85EB51A84C01083E
:10812000001A0020C5B3A2918988888870B50D46D1
:10813000B1F90E10002990B014461E4614DB01AAB6
:10814000FFF7B2FC00280FDB029A02F47042A2F59E
:108150000052B2FA82F252094FF480634FF4006089
:108160003260236010B070BDA88900F0800082B238
:10817000002030601AB14023236010B070BD4FF46E
:1081800080631046236010B070BD00BF8A899207DB
:108190000B4606D501F1430201211A601A615961AB
:1081A0007047F0B583B001AB6A460C460546FFF751
:1081B000BDFF00990646284600F03CF8B4F90C30A3
:1081C000D0B1019A124F0099EF6343F08003A3816D
:1081D0002060206161611AB93343A38103B0F0BD0F
:1081E0002846B4F90E1007F083FBB4F90C300028D0
:1081F000F2D043F00103EFE79A05EFD404F1430214
:1082000043F002030121A381226022616161E5E75D
:10821000ED720008024B0146186800F00BB800BF71
:10822000E8050020024B01461868FFF7F3B900BFCC
:10823000E80500202DE9F04F01F10B05162D83B064
:10824000064640F29F8035F0070500F1BF80A94245
:1082500000F2BC80FBF7DEFDB5F5FC7FC0F09C8230
:108260006B0A00F0BA80042B00F28381A80900F1A8
:10827000390E4FEA4E033830C44F07EB8303A3F1A6
:1082800008015C68A14207D1ACE0002A80F2AC8012
:10829000E468A14200F0A680636823F003035A1B40
:1082A0000F2AF2DDB9493C6901F1080E744500F06E
:1082B000B381636823F003035A1B0F2A00F39981EB
:1082C000002AC1F814E0C1F810E080F29E80B3F5F6
:1082D000007F80F06781DB0803F1010C01229B1015
:1082E00002FA03F34A6851F83C80C4F8088001EBB5
:1082F000CC091A43A9F10803E3604A6041F83C4005
:10830000C8F80C40831001249C40944200F28A80FB
:10831000144206D120F003006400144200F104006E
:10832000FAD007EBC009CC468046DCF80C108C452F
:1083300007D173E1002A80F28181C9688C4500F081
:108340006D814B6823F003035A1B0F2AF2DD0C46A4
:10835000D1F80CC054F8088F4B1945F001054D6059
:1083600042F00101C8F80CC03046CCF808807B61AF
:108370003B61C3F80CE0C3F808E059609A50FBF782
:108380004DFD1FE0102921D8FBF744FD10250623E1
:1083900002207E4F07EB8303A3F108025C6894423E
:1083A00000F045816368E168A56823F00303234476
:1083B00030465A68E96042F001028D605A60FBF76E
:1083C0002DFD0834204603B0BDE8F08F00240C23B7
:1083D0002046336003B0BDE8F08F80234FF0400E9D
:1083E0003F2049E770465DE72344E1685A68A56885
:1083F00042F00102E96030468D605A60FBF70EFDE5
:108400000834204603B0BDE8F08F234430465A6854
:1084100042F001025A60FBF701FD0834204603B028
:10842000BDE8F08FBC68636823F00308A84504D357
:10843000C5EB08030F2B00F38C80554BDFF86091E0
:108440001A68D9F8003001332A4404EB080A00F016
:10845000608102F580520F3222F47F6222F00F0217
:1084600011463046019201F019F9B0F1FF3F834601
:10847000019A00F05881824500F2FC80454B196852
:10848000DA451144196000F05381D9F80000DFF893
:1084900010E101301BBFCAEB0B0A5144CEF800B00B
:1084A00019601BF0070100F01781C1F10800C1F548
:1084B0008051834408315A44C2F30B02C2EB0109D4
:1084C00049463046019301F0E9F8431C019B00F056
:1084D0003F81CBEB00024A4442F001021968C7F821
:1084E00008B04944BC42CBF804201960DFF8A490DE
:1084F00016D0B8F10F0F40F2FD806268A8F10C03AE
:1085000023F00703E01802F001024FF0050E1A43B2
:108510000F2B6260C0F804E0C0F808E000F21C8194
:108520001D4BBC681A68914288BF19601B4B1A68C2
:108530009142626888BF196022F003029542A2EB63
:10854000050301D80F2B04DC3046FBF767FC002441
:1085500038E7621943F0010345F0010565603046D4
:10856000BA605360FBF75AFC0834204603B0BDE8FC
:10857000F08F142B71D9542B00F2A480280B00F13A
:108580006F0E4FEA4E036E3076E600BFEC0500201A
:10859000B8190020BC190020B4190020B01900201F
:1085A000F80900205A0A042A5ED9142A00F2B3807E
:1085B00002F15C0149005B3207EB810C57F8211096
:1085C000DFF8DC81ACF1080C8C4500F088804A684B
:1085D00022F00302934202D289688C45F7D1D1F888
:1085E0000CC07A68C4F80CC0A160CCF80840CC601C
:1085F00088E6631942F0010745F0010565603046E1
:108600004B610B61C3F80CE0C3F808E05F609A505F
:108610000834FBF703FCD5E64A6873E608F1010865
:1086200018F0030F0CF1080C7FF47FAE30E0DC682B
:10863000A34208BF02303FF435AEB3E60B440C460C
:108640005A68C96854F8085F42F001025A6030461F
:10865000E9608D60FBF7E2FBB4E603F15C0E03F129
:108660005B004FEA4E0307E69A0902F1390149001F
:108670003832A1E7BC424A4B3FF400AF9C686268C5
:1086800022F003025AE759F80839994540F08280F0
:1086900010F0030F00F1FF30F5D17B6823EA0403EB
:1086A0007B6064009C423FF6BDAE002C3FF4BAAE46
:1086B0001C4240467FF435AE64001C4200F10400C9
:1086C000FAD02EE6B3F5AA7F18D8E80B00F1780EA1
:1086D0004FEA4E037730CFE54FF48051EBE60121AE
:1086E000D8F80430921001FA02F21A43C8F80420B4
:1086F000614677E70123CBF8043025E740F2545276
:10870000934220D8A80C00F17D0E4FEA4E037C3036
:10871000B2E51032A4E6542A26D81A0B02F16F01F2
:1087200049006E3248E7BC68626822F0030205E740
:10873000CAF30B0000287FF4A8AE4244BB6842F0A5
:1087400001025A60ECE6FE234FF07F0E7E2093E597
:1087500001224FF00009C1E604F108013046FEF79E
:1087600059FFD9F80010DBE6B2F5AA7F05D8DA0B7D
:1087700002F17801490077321EE740F254518A42F3
:1087800005D89A0C02F17D0149007C3214E7FE21E4
:108790007E2211E77B6884E7E808431C5B00F8E56C
:1087A000EC050020000000000000000000000000B8
:1087B00001F0FF01102A2BDB10F0070F08D010F892
:1087C000013B013A8B422DD010F0070F42B3F6D196
:1087D000F0B441EA012141EA014122F007047FF0AF
:1087E00000070023F0E80256083C85EA010586EA06
:1087F000010685FA47F5A3FA87F586FA47F6A5FA42
:1088000087F68EB9EED1F0BC01F0FF0102F007024D
:1088100032B110F8013B013A83EA010313B1F8D1F8
:108820000020704701387047002D06BF35460338D9
:10883000073815F0010F07D1013015F4807F02BF12
:10884000013015F4C03F0130F0BC0138704700BF63
:10885000032A70B426D940EA01039B0711D004789B
:108860000D78AC4222D10244431C05E013F8014BC1
:1088700011F8015FAC4219D19342F7D1002070BCCE
:1088800070470C4603461E682568AE4218462146CE
:1088900003F1040304F10404E1D1043A032A184665
:1088A0002146F0D8002ADAD11046E8E7601B70BCF8
:1088B000704700BF844641EA000313F003036DD103
:1088C000403A41D351F8043B40F8043B51F8043B93
:1088D00040F8043B51F8043B40F8043B51F8043B9A
:1088E00040F8043B51F8043B40F8043B51F8043B8A
:1088F00040F8043B51F8043B40F8043B51F8043B7A
:1089000040F8043B51F8043B40F8043B51F8043B69
:1089100040F8043B51F8043B40F8043B51F8043B59
:1089200040F8043B51F8043B40F8043B51F8043B49
:1089300040F8043B51F8043B40F8043B51F8043B39
:1089400040F8043B403ABDD2303211D351F8043BD9
:1089500040F8043B51F8043B40F8043B51F8043B19
:1089600040F8043B51F8043B40F8043B103AEDD288
:108970000C3205D351F8043B40F8043B043AF9D2D9
:10898000043208D0D2071CBF11F8013B00F8013BAC
:1089900001D30B8803806046704700BF082A13D3B9
:1089A0008B078DD010F003038AD0C3F10403D21AD1
:1089B000DB071CBF11F8013B00F8013B80D331F805
:1089C000023B20F8023B7BE7043AD9D3013A11F885
:1089D000013B00F8013BF9D20B7803704B784370F0
:1089E0008B788370604670478842F0B50DD98B183C
:1089F00098420AD28118002A51D09A1A13F8014DD0
:108A000001F8014D9342F9D1F0BD0F2A48D941EA4E
:108A100000039B0746D100F1100401F11003154635
:108A200053F8106C44F8106C53F80C6C44F80C6C50
:108A300053F8086C44F8086C103D53F8046C44F883
:108A4000046C0F2D03F1100304F11004E8D8A2F117
:108A5000100323F00F0302F00F0E1033BEF1030FCB
:108A60001944034421D91E1F0D467446043C55F891
:108A7000047B46F8047F032CF8D8AEF1040424F0FC
:108A8000030404342344214402F0030262B1013B95
:108A90000A4411F8014B03F8014F8A42F9D1F0BDA5
:108AA0000346F3E70346F2E7F0BD7246EEE700BF88
:108AB00070B4840746D0541E002A41D0CDB203467C
:108AC00002E0621EE4B3144603F8015B9A07F8D192
:108AD000032C2ED9CDB245EA05250F2C45EA0545D4
:108AE00019D903F110022646103E0F2E42F8105CF1
:108AF00042F80C5C42F8085C42F8045C02F1100297
:108B0000F2D8A4F1100222F00F0204F00F04103288
:108B1000032C13440DD91E462246043A032A46F874
:108B2000045BFAD8221F22F003020432134404F03B
:108B300003042CB1C9B21C4403F8011BA342FBD1AE
:108B400070BC704714460346C2E700BF2DE9F043EE
:108B500001683B2983B0044600F2BB8041683B2991
:108B600000F2AA80A168172900F2998021690B29D7
:108B700000F2888063699F073ED17448DA1780FB52
:108B80000365C2EB6512642505FB1232002A73D11E
:108B900003F26C7380FB0320DA17C2EBE0104FF492
:108BA000C87202FB1033002B0CBF1D261C26E36885
:108BB000002B26DD664FDFF894C14FF0000E4FF01A
:108BC00064084FF4C8794A1C07EB81000BE0056884
:108BD0009D42A3EB050337DA0C2AE360226136D00D
:108BE0000131013204300129F1D19E42A3EB060389
:108BF0002ADAE3602261F3E7E368002B4FF01C06FA
:108C0000D8DC5348514D64274FF4C87E07E0012952
:108C100014BF50F8212032461344002B12DC11F10E
:108C2000FF31F4D261694A1E9607626126D185FB45
:108C3000026CD617C6EB6C1607FB1622002A55D01D
:108C40001D261CE0E360216103B0BDE8F08361698B
:108C5000C4F810E04A1C9007626102D01C26002173
:108C6000B1E78CFB0205D017C0EB651008FB1022A2
:108C7000002A49D01D26F2E71D2698E71C260B2165
:108C80001F22C9E70C22684605F0FCFC6269009BC4
:108C9000019913440029636153DB21616BE71822BA
:108CA000684605F0EFFCE168009B019A0B44002A3E
:108CB000E36041DBA26059E73C22684605F0E2FC34
:108CC000A3680099019A1944002AA1602FDB626011
:108CD00049E73C22684605F0D5FC6168009B019A93
:108CE0001944002A61601DDB226038E701F26B71D4
:108CF00085FB0126CA17C2EBE6120EFB12110029F2
:108D000014BF1C261D26BAE701F26D718CFB0120F1
:108D1000CA17C2EBE01209FB1211002914BF1C266E
:108D20001D269CE73C3201392260616017E73C3226
:108D300001396260A16016E71832013BA260E3606E
:108D400014E70C31013B2161636114E71F85EB518E
:108D5000784C01082DE9F84F064606F0DFFC804606
:108D60003046FFF7F3FEC64C356973683068F26829
:108D700054F82540B168C3EB031300EB83034FF4B1
:108D8000616E013A012D0EFB013E1444756902DD4E
:108D9000AB0700F0C18005F51C53103344F6206288
:108DA0009342F46100F26381462D00F38C8053D02E
:108DB000452D00F03481B348452340F26D196427F6
:108DC0004FF4C87C16E003F26C7B80FB0BA14FEAEA
:108DD000EB7ACAEBE1110CFB11B1002A40F0C7801D
:108DE000002914BF4A464FF4B772013BAB42A4EBD3
:108DF000020410D080FB0312D917C1EB621213F0EA
:108E0000030F07FB1232DED0013B40F26D12AB4282
:108E1000A4EB0204EED1AF0740F00181994AEB17B1
:108E200082FB0501C3EB6113642101FB1353002B8B
:108E300040F0078105F26C7182FB0132CB17C3EB66
:108E4000E2124FF4C87303FB1213002B40F26D13B0
:108E500008BF4FF4B773E41A8B4800FB04E903F032
:108E60006BFD03F06DFD894B1F68002F00F08280C1
:108E7000376A7069D8F80430012F00F26C70A8BF0F
:108E80000127984257D003F08DFC002853D1012FC1
:108E900040F0D380D8F83C1009EB0105012703F01E
:108EA0004DFD7B4A3762043484FB0223E218E3174A
:108EB000C3EBA203C3EBC303E31A48BF0733B36199
:108EC0002846BDE8F88F6F48462340F26D196427A5
:108ED0004FF4C87C13E003F26C7B80FB0BA14FEADC
:108EE000EB7ACAEBE1110CFB11B10ABB002914BFEC
:108EF0004A464FF4B7720133AB421444ACD080FB06
:108F00000312D917C1EB621213F0030F07FB1232E1
:108F1000E1D040F26D12EEE75A4AEB1782FB0501F1
:108F2000C3EB6113642101FB135343B3013432E7F4
:108F30004FF4B772DFE7D8F82020D8F83830D8F8E7
:108F40003C10C2EB030CE145104602DB5B1A99456D
:108F50009DDBD8F81C30C1EB030ED8F80030EBB124
:108F6000F1455FDA002F80F2C180002704E04FF462
:108F7000B7723AE7D8F8200009EB00058FE705F251
:108F80006C7182FB0132CB17C3EBE2124FF4C87352
:108F900003FB1212002A7FF4FEAEC7E7F14541DB66
:108FA000002FFFF679AF7FF477AF511A3268F76878
:108FB0000A44326030468944FFF7C8FDF368DB1B82
:108FC0003FF468AF0127012B40F383804FF0FF335C
:108FD000F2691C449B185DD4AA074ED12949EA17AF
:108FE00081FB05E0C2EB6012642000FB1252002AF4
:108FF00073D105F26C7581FB0512E917C1EBE21123
:109000004FF4C87202FB1152002A40F26D1208BFE1
:109010004FF4B7729A42D8BF9B1AF36137E740F218
:109020006D1318E7E145ACBF00230123002F02DBDD
:109030005F40012F08D01F4629E7D8F820201046AE
:109040009AE74FF4B77306E7511A002BAED1326896
:10905000F768521A32603046C1EB0909FFF776FD16
:10906000F368DB1B07D1D8F820001F4684E74FF0D8
:10907000FF30BDE8F88F0027A5E740F26D12C9E781
:10908000484C01081F85EB5180510100001A002057
:1090900093244992681E810722D11849C21781FB87
:1090A00000E3C2EB6312642303FB1203DBB905F296
:1090B0006B7581FB0531EA17C2EBE1124FF4C873FF
:1090C00003FB1253002B40F26D1318BF4FF4B6731D
:1090D000A3E7981CD8BF01237AE74FF4B77299E74A
:1090E0004FF4B67399E740F26D1396E7012F02D063
:1090F0000027104640E7511AA9E700BF1F85EB5132
:1091000070B50D46084C114606461A4628460023FF
:109110002360FAF7BBFE431C00D070BD2368002B10
:10912000FBD0336070BD00BFE01A00200FB400B563
:10913000074983B004AB086853F8042B8168019396
:1091400003F096FD03B05DF804EB04B0704700BF78
:10915000E805002010B40C4B0C4C19680C4AD1F8EF
:10916000A830D1F8AC0004FB03F402FB0040A3FBE1
:1091700002230344013243F10003C1E92A2323F00F
:1091800000405DF8044B7047E80500202DF451586D
:109190002D7F954C2DE9F04F174683B0002900F044
:1091A000C1800E46814607F10B05FAF733FE56F8EB
:1091B00004EC162D2EF00304A6F1080840D8102266
:1091C0001546AF4241D8944275DAC94B996808EB0D
:1091D00004008842416800F0D98021F00103034473
:1091E0005B68DB077DD51EF0010F35D03946484658
:1091F000FFF720F80746E0B156F8043C23F00103DE
:109200004344A0F108029A4200F04481221F242A1C
:1092100000F23181132A00F20481034632461168BC
:1092200019605168596092689A6031464846FEF765
:10923000F1F94846FAF7F2FD384603B0BDE8F08F81
:1092400025F00705002D2A46BBDA0C230020C9F8BB
:10925000003003B0BDE8F08F56F8083CC3EB080AB5
:10926000DAF8043023F0030C04EB0C039342BDDB6B
:109270005746DAF80C1057F8080F221F242AC1604D
:10928000886000F21781132A40F212813168CAF80F
:1092900008107168CAF80C101B2A00F22B810836DE
:1092A0000AF110023168116071685160B168916013
:1092B0003E461C46D046631B0F2B1DD8D8F8043001
:1092C00003F0010323434444C8F80430636843F0C7
:1092D000010363604846FAF7A1FD304603B0BDE8DC
:1092E000F08F21F003012144914221DBC3688268A1
:1092F0000C46D3609A60DEE7D8F8042008EB05013D
:1093000002F00102154343F001020B44C8F8045077
:109310004A605A6842F0010208315A604846FEF736
:1093200079F9D7E7114603B0BDE8F04FFEF782BFE9
:109330001EF0010F7FF45AAF56F8083CC3EB080A41
:10934000DAF8043023F0030C01EB0C0E96458BDBAE
:10935000C36882685746D3609A6057F8081FDAF8E6
:109360000C30CB60221F242A996000F29980132AC6
:1093700062D93368CAF808307368CAF80C301B2AFF
:1093800000F2A08008360AF1100356E021F0030B2A
:10939000A34405F11000834559DA1EF0010F7FF454
:1093A00025AF56F8081CC1EB080ADAF8041021F0C2
:1093B000030CE34458453FF757AF5746DAF80C1013
:1093C00057F8080F221F242AC160886000F2B48079
:1093D000132A40F2A5803168CAF808107168CAF8EB
:1093E0000C101B2A00F2AF8008360AF11002316817
:1093F000116071685160B16891600AEB0501C5EBBD
:109400000B0242F0010299604A60DAF8043003F07E
:1094100001031D434846CAF80450FAF7FFFC3846DA
:109420005CE733680360736843601B2A27D800F148
:10943000080306F10802F2E63B4632681A607268D9
:109440005A60B2689A603E467446D04633E708EBED
:109450000501C5EB0B0B4BF0010299604A6056F811
:10946000043C03F001031D43484646F8045CFAF748
:10947000D5FC304632E73146FFF7B6FAD5E6B36899
:109480008360F368C360242A28D000F1100306F13A
:109490001002C4E650F8043C23F003031C440AE71E
:1094A000314638467446D046FFF79EFA3E4602E7FC
:1094B0003A46F7E6314638461C46D046FFF794FA5E
:1094C0003E46F8E6B368CAF81030F368CAF81430BC
:1094D000242A1BD010360AF11803AEE73369036162
:1094E0007369436106F1180200F1180397E600BFA3
:1094F000EC050020B168CAF81010F168CAF8141021
:10950000242A0FD010360AF11802CBE63369CAF8C4
:1095100018307369CAF81C3018360AF120038CE73A
:109520003A4664E73269CAF818207269CAF81C2002
:1095300018360AF12002B5E6314638460193FFF7A6
:1095400053FA019B59E7B168CAF81010F168CAF8DC
:109550001410242A03D010360AF1180247E73269A2
:10956000CAF818207269CAF81C2018360AF12002BD
:109570003DE700BF838903F00903092B01D00020D8
:109580007047FDF7A1BE00BFF8B50C46054610B107
:10959000836B002B45D0B4F90C309AB2970407D4F2
:1095A000626E43F4005322F400526266A3819AB2C1
:1095B00000219606616031D4500722D5216B61B13C
:1095C00004F14003994202D02846FEF723F8E36BEA
:1095D000636000202063002B3FD12369002B4CD017
:1095E000B4F90C70BEB2B3071ED1226922602846BE
:1095F0006369256AE169A8470028606009DD0020E9
:10960000F8BDD1063ED512072AD443F00403A38146
:10961000E3E7A38919D143F02003A3814FF0FF3082
:10962000F8BDFDF73DFFB6E71A4B1B49186801234B
:10963000A38106F00906FEF7CDFB092EA781D4D140
:1096400021462846FDF786FDCFE7002243F0400380
:10965000A38162604FF0FF30F8BDA36B2360F8BDBB
:1096600021462846FDF71AFE0028D7D1B4F90C3060
:10967000A060A06123F00803C7E721462846FEF753
:1096800085FDADE743F0400309222A604FF0FF302B
:10969000A381F8BD444C01087595000838B5074C06
:1096A0000023054608462360FAF772FB431C00D0EE
:1096B00038BD2368002BFBD02B6038BDE01A00209A
:1096C00000290CBF022200224FF4806300F000B892
:1096D0002DE9F043514C256883B004460F4690466F
:1096E0001E4615B1AB6B002B79D0B8F1020F04D038
:1096F000B8F1010F7FD8002E7DDB21462846FDF70B
:10970000CDFD216B41B104F14003994202D02846BE
:10971000FDF780FF00232363B4F90C300022A2611F
:1097200062601A0654D423F44A6323F00303B8F1A9
:10973000020FA38139D001AB6A4621462846FEF7C5
:10974000F5FCA3891843A08126B327B3AB6B002B8C
:109750004DD0009BB4F90C0027609E421CBF40F422
:109760000060A081B8F1010F08BF40F0010083B292
:1097700008BFA08103F0080080B22761666118B3BA
:1097800013F001002FD000207642A661A06003B044
:10979000BDE8F083009E3046FEF73CFD074668B307
:1097A000A38943F08003A381D0E7002004F14302A2
:1097B00043F0020300250121A381A56022602261FC
:1097C000616103B0BDE8F083A06003B0BDE8F08341
:1097D00021692846FDF71EFFB4F90C30A3E728469F
:1097E000FDF75EFE81E7A66003B0BDE8F083284682
:1097F000FDF756FEADE74FF0FF30E2E7DDF80090F1
:10980000B14506D04846FEF705FD074608B14E466D
:10981000C6E7B4F90C304FF0FF30C7E7E805002089
:109820000CB4F0B5244B00299DB01D683EDB4FF40D
:1098300002730C4602900690ADF8143023AE17D098
:109840004C1E229A049433464FF6FF7702A928460D
:1098500007940196ADF8167000F0EAFC421C1BDB81
:10986000029B00221A701DB0BDE8F04002B07047A4
:1098700033464FF6FF77229A049402A928460794AC
:109880000196ADF8167000F0D3FC431C07DB1DB049
:10989000BDE8F04002B070478B232B60E0E78B23DC
:1098A0002B601DB0BDE8F04002B070478B232B60E9
:1098B0004FF0FF30EBE700BFE80500200EB4F0B535
:1098C0009CB021AB0F4953F8042B019305466FF070
:1098D0000044086802954FF402774FF6FF7602A91C
:1098E0000695ADF8147004940794ADF8166000F076
:1098F0009FFC029B00221A701CB0BDE8F04003B030
:10990000704700BFE80500200EB4F0B59CB021AC54
:109910004FF4017254F8046BADF8142002900690D5
:1099200000F0CEFA0C4B0194054632460B4F1868F6
:10993000039523464FF6FF76002402A907950A9760
:109940000E941394ADF8166001F0ECFF1CB0BDE866
:10995000F04003B0704700BFE8050020859900087B
:1099600010B50C46B1F90E1006F0DAFC002803DB46
:10997000236D0344236510BDA38923F48053A38181
:1099800010BD00BF002070472DE9F0411646B1F927
:109990000C201F46D3050C46054607D5002202239E
:1099A000B1F90E1005F0FCFFB4F90C20B4F90E105B
:1099B00022F48052A2813B4632462846BDE8F0415F
:1099C00004F0D4BD10B50C46B1F90E1005F0E8FF57
:1099D000A389421C0EBF23F4805343F480532065B7
:1099E000A38110BDB1F90E1004F03ABE830710B583
:1099F000044610D10268A2F1013323EA020313F0F6
:109A0000803F08D150F8042FA2F1013323EA02036A
:109A100013F0803FF6D003781BB110F8013F002B04
:109A2000FBD100F0DBF9204610BD00BF70B411F08F
:109A3000FF0434D085070FD00378002B5AD09C4206
:109A40002BD0431C05E013F8012B002A4FD0944281
:109A500023D09A071846F6D10E0206F47F46264315
:109A6000036846EA064601E050F8043F86EA03052B
:109A7000A5F10132A3F1013122EA050221EA030333
:109A8000134313F0803FEFD0037823B932E010F88E
:109A9000013F002B2ED09C42F9D170BC7047840747
:109AA0000BD00378002BF8D0431C03E0027801337D
:109AB000002AF2D099071846F8D10268A2F10133C2
:109AC00023EA020313F0803F08D150F8042FA2F1DB
:109AD000013323EA020313F0803FF6D00378002B12
:109AE000DBD010F8013F002BFBD170BC7047104653
:109AF00070BC7047184670BC704700BF0000000083
:109B0000A2EB0300704700BF02780B78012A28BF40
:109B10009A42F5D16DE9044540EA0104CDE90267B6
:109B20006FF0000C4FEA447212B380EA010414F0A3
:109B3000070F6AD100F0070420F0070004F00305C6
:109B400021F007014FEAC505F0E8042314F0040FE3
:109B5000F1E804670CFA05F462EA040266EA040616
:109B60000AD063EA0403624667EA0407664603E034
:109B7000F0E80423F1E8046782FA4CF582EA06046F
:109B8000A4FA8CF46CBB83FA4CF583EA0705A5FABA
:109B90008CF595B950E9022351E9026782FA4CF538
:109BA00082EA0604A4FA8CF483FA4CF583EA0705EA
:109BB000A5FA8CF52543DBD09CB92DBAB5FA85F40E
:109BC00024F0070427FA04F1DDE9026723FA04F31D
:109BD00003F0FF0001F0FF01FDE80445A0EB0100E8
:109BE000704724BAB4FA84F424F0070426FA04F186
:109BF000DDE9026722FA04F202F0FF0001F0FF0142
:109C0000FDE80445A0EB0100704714F0030F3CD1C0
:109C100010F0030428D150F8082B51F8083B82FAC1
:109C20004CF582EA0305A5FA8CF55DB950F8042CD1
:109C300051F8043C82FA4CF582EA0305A5FA8CF54A
:109C4000002DE8D02DBAB5FA85F424F0070423FAE4
:109C500004F122FA04F202F0FF0001F0FF01FDE836
:109C60000445A0EB010070474FEAC40420F0030054
:109C700050F8082B21F0030151F8083B0CFA04F4CA
:109C800062EA040263EA0403C9E710F003041AD08D
:109C9000A1EB040120F00300E40750F8042B06D0E8
:109CA0000FD28B785FFAA2F4E41A06D12BB1CB78ED
:109CB0005FFAB2F4E41A00D11BB920465DF8104BEC
:109CC000704701F1040150F8042BCC0721F0030187
:109CD00051F8043B48D824D222F07F4482FA4CF554
:109CE00094EA1325A5FA8CF50AD165B951F8043B1D
:109CF00084EA0204B4EB036F0ED150F8042BEBE7B7
:109D00004FEA132355E035F07F454DD10878FDE843
:109D10000445C0F1000070474FEA126203F0FF03F0
:109D200047E002EA1C4482FA4CF594EA1345A5FA8E
:109D30008CF50AD165B951F8043B84EA0204B4EB0E
:109D4000034F0CD150F8042BEBE74FEA134330E0FC
:109D500015EA1C4528D10B884FEA124229E04FEA48
:109D6000124203EA1C4324E002F0FF0482FA4CF59D
:109D700094EA1365A5FA8CF50AD165B951F8043B4C
:109D800084EA0204B4EB032F09D150F8042BEBE76B
:109D90004FEA13630DE015F0FF0F05D10B684FEA92
:109DA000122223F07F4304E04FF00000FDE8044559
:109DB000704712BA1BBA82FA4CF482EA0304A4FA7E
:109DC0008CF5B5FA85F402FA04F203FA04F34FEACB
:109DD0001260FDE80445A0EB1360704780EA0102C1
:109DE000844612F0030F4FD111F0030F32D14DF81A
:109DF000044D11F0040F51F8043B0BD0A3F10132D4
:109E00009A4312F0803F04BF4CF8043B51F8043BE6
:109E100016D100BF51F8044BA3F101329A4312F05E
:109E2000803FA4F101320BD14CF8043BA24312F065
:109E3000803F04BF51F8043B4CF8044BEAD0234662
:109E40000CF8013B13F0FF0F4FEA3323F8D15DF814
:109E5000044B704711F0010F06D011F8012B0CF8DC
:109E6000012B002A08BF704711F0020FBFD031F854
:109E7000022B12F0FF0F16BF2CF8022B8CF80020DB
:109E800012F47F4FB3D1704711F8012B0CF8012B5E
:109E9000002AF9D1704700BF000000000000000058
:109EA00000000000000000000000000000000000B2
:109EB00000000000000000000000000000000000A2
:109EC00090F800F06DE9024520F007016FF0000CFA
:109ED00010F0070491F820F040F049804FF00004A2
:109EE0006FF00700D1E9002391F840F000F108007D
:109EF00082FA4CF2A4FA8CF283FA4CF3A2FA8CF3B5
:109F00004BBBD1E9022382FA4CF200F10800A4FA1B
:109F10008CF283FA4CF3A2FA8CF3E3B9D1E904236F
:109F200082FA4CF200F10800A4FA8CF283FA4CF3A6
:109F3000A2FA8CF37BB9D1E9062301F1200182FA60
:109F40004CF200F10800A4FA8CF283FA4CF3A2FA66
:109F50008CF3002BC6D0002A04BF04301A4612BA74
:109F6000B2FA82F2FDE8024500EBD2007047D1E977
:109F7000002304F00305C4F100004FEAC50514F006
:109F8000040F91F840F00CFA05F562EA05021CBFD7
:109F900063EA050362464FF00004A9E7002A41D0B6
:109FA00040EA010313F00303F0B425D1032A23D9B7
:109FB00004680D68AC421FD1043A35D0A4F10135D4
:109FC00025EA040414F0803F31D1071D0D1D0DE07A
:109FD00057F8043B0E68A3F10134B34224EA0304AA
:109FE0000AD1043A20D014F0803F23D1032A294615
:109FF000384605F10405EBD803780C789C4202F151
:10A00000FF320CD182B114B916E06AB17BB110F8FD
:10A01000013F11F8014FA34202F1FF32F5D0181BA6
:10A02000F0BC7047104670471046F0BC70471846A9
:10A03000F0BC70470020F3E72046F1E740EA010357
:10A040009B0770B42BD1032A29D90C46034621461D
:10A0500054F8046BA6F1013525EA060515F0803F9A
:10A0600006D1043A032A43F8046B2146EFD8A2B183
:10A070000C781C70013A013301313CB16AB111F81E
:10A08000014B03F8014B013A002CF7D12AB11A44D5
:10A09000002103F8011B9A42FBD170BC70470346B4
:10A0A000E5E700BF2DE9F84FDDF828900F46804620
:10A0B00016461D468B4600E0A3465C46484614F80B
:10A0C00001AB05F04FFC5044417801F0080101F06C
:10A0D000FF0C0029F0D152462D2A61D02B2A04BF53
:10A0E0009BF801200BF10204002D43D0102D65D008
:10A0F000A946BCF1000F0CBF6FF0004A4FF0004AB8
:10A100000021BAFBF9FE084609FB1EAA05E029D08A
:10A1100009FB0030012114F8012BA2F13003092BB7
:10A1200005D9A2F14103192B0AD8A2F137039D42A8
:10A130000EDD4A1CEFD08645E9D24FF0FF31EAE749
:10A14000A2F16103192B03D8A2F157039D42F0DC61
:10A150004B1C15D0BCF1000F10D14EB1E1B93760E6
:10A16000BDE8F88F9A45D3DA70464FF0FF31D2E759
:10A17000BDE8F88F302A1AD00A25B9E74042ECE74B
:10A18000BCF1000F4FF022030CBF6FF000404FF006
:10A190000040C8F80030F6B1671E3760BDE8F88FA0
:10A1A0000BF102049BF801204FF0010C9CE723788F
:10A1B00003F0DF03582B08D0082599E7302A97D100
:10A1C000237803F0DF03582B92D14FF01009627807
:10A1D0004D4602348DE7BDE8F88F00BF30B5064C20
:10A1E000064D2468646B83B0002C08BF2C46009495
:10A1F000FFF758FF03B030BDE8050020440A0020F7
:10A2000030B5084C084B25686C6B83B0002C08BF38
:10A210001C46009413460A4601462846FFF742FFB3
:10A2200003B030BDE8050020440A00200000000013
:10A230002DE9F04FC5B00C46099115460E930A90D2
:10A2400005F0A0FB036817931846FFF739FEA389B2
:10A2500016901E0603D52369002B01F033819FED74
:10A26000A67B00238DED147B1293299328931993D9
:10A270000B93DFF890A234AB27939946A84698F841
:10A2800000304446EBB1252B02D11AE0252B03D038
:10A2900014F8013F002BF9D1C8EB04058DB1289BC0
:10A2A000299AC9F8008001332A44072BC9F80450C1
:10A2B0002992289300F3A68009F108090B9B2B44EF
:10A2C0000B932378002B00F0A68000231A468DF80C
:10A2D0007F3019460C9307934FF0FF3B637804F1EE
:10A2E00001085D4608F10108A3F12000582800F29A
:10A2F0003484DFE810F0A00332043204A8033204EF
:10A3000032043204320432043204AF03BD03320497
:10A310005D00E2003204090110011001100110017A
:10A320001001100110011001100132043204320436
:10A330003204320432043204320432043204200182
:10A340008602320486023204320432043204D40219
:10A3500032043204E502320432043204320432049C
:10A360000F03320432043D03320432043204320457
:10A370003204320432043204320432047E03910384
:10A38000860286028602990391033204320407048E
:10A3900032041204A3006400C2033204C90332046D
:10A3A000EA0332043204F2030C980E9340420C90FC
:10A3B000079B43F00403079398F8003092E70E9848
:10A3C000AB46002104688DF87F10071D07983023E5
:10A3D00078228B458DF880304FF000058DF8812074
:10A3E00040F00203C0F2D68320F0800343F0020362
:10A3F000079354EA05030E9700F0A2830F461192CB
:10A400003F48E6E227AA09990A9807F06BFA48B98B
:10A410000DF1D00952E7299B23B10A98099927AA7F
:10A4200007F060FA099B9B8913F0400F0B9B18BF44
:10A430004FF0FF33184645B0BDE8F08F1193AB469F
:10A44000002A41F03B82079A12F0200300F0468276
:10A450000E9F073727F00703002703F10801BB45CC
:10A460000E91D3E900458DF87F70C0F2648722F029
:10A470008003079354EA050300F0848334AEE208B6
:10A4800042EA4572E90804F007030D4614463033EA
:10A4900054EA050206F8013DF1D1079AD10740F1CF
:10A4A0008F80302B00F08C803022731E06F8012C38
:10A4B00034AAD21A0D921E4685E098F800302A2B55
:10A4C00008F1010401F0EC81A3F13000092898BFE4
:10A4D000002501F28E8114F8013B05EB850500EBA8
:10A4E0004505A3F130000928F5D945EAE575A046F0
:10A4F000FAE600BFAFF3008000000000000000009B
:10A500003C4D0108084D0108079B43F08003079369
:10A5100098F80030E6E6A3F1300000231C4618F856
:10A52000013B04EB840400EB4404A3F13000092850
:10A53000F5D90C94D8E61193AB46002A41F0CC81B2
:10A54000079B43F010030793079B9C0640F1378558
:10A550000E9F073727F00707D7E9002307F1080107
:10A560000E9114461D46002A73F10003C0F2628565
:10A57000BBF1000F9DF87F70C0F23F85079B23F071
:10A580008003079354EA050300F0E881002D08BF1B
:10A590000A2CC0F0E88134AE204629460A22002366
:10A5A00009F0E0F9303206F8012D20462946002353
:10A5B0000A2209F0D7F904460D4654EA0503EBD107
:10A5C00034AB9B1B0D930D9B5B45B8BF5B4608935B
:10A5D0000023139317B1089B01330893079B13F0D3
:10A5E00002030F9302D0089B02330893079B13F0DA
:10A5F0008403109340F0DB820C9B089A9D1A002D77
:10A6000040F3D582102D2999289AA84F27DD189656
:10A6100048461024B946099E2F460A9D04E0103F83
:10A62000102F00F1080016DD0132A04B28921031E6
:10A63000072A299180E81800F1DD27AA314628462B
:10A6400007F050F900287FF4EDAE103F102F299944
:10A65000289A34A8E8DC189E3D464F4681460132D0
:10A660006C18072A29942892C9F80070C9F8045078
:10A6700000F32D849DF87F7009F1080977B1289BBC
:10A68000013301340DF17F010122072B2994289316
:10A6900089E8060000F3A58309F108090F9B6BB157
:10A6A000289B0133023420A90222072B29942893E6
:10A6B00089E8060000F3A18309F10809109B802BAB
:10A6C00000F0E1820D9BC3EB0B07002F33DD784ACE
:10A6D000289B0F92102F22DD22464FF0100B0A9D6F
:10A6E000099C04E0103F102F09F1080916DD013321
:10A6F0001032072B2992289389E8000CF2DD27AA53
:10A700002146284607F0EEF800287FF48BAE103F74
:10A71000102F299A289B0DF1D009E8DC144601334B
:10A720000F9A28933C44072B299489E8840000F36E
:10A730004C8309F10809079BDA0500F13A82289B4E
:10A740000D99C9F8006001330C44072B2994C9F80E
:10A750000410289300F3238309F10809079B590784
:10A760003FD50C9B089A9D1A002D3ADD102D289B91
:10A770004E4F23DD22461026DDF828B0099C04E068
:10A78000103D102D09F1080917DD013347492893C1
:10A790001032072B299289E84200F1DD27AA2146D1
:10A7A000584607F09FF800287FF43CAE103D102D6E
:10A7B000299A289B0DF1D009E7DC144601332C447B
:10A7C000072B29942893C9F80070C9F8045008DDB4
:10A7D00027AA09990A9807F085F800287FF422AE85
:10A7E000299C0B9B0C9A08998A42ACBF9B185B185A
:10A7F0000B93002C40F0DF82002328930DF1D00949
:10A800003DE51193AB46002A41F06A80079B0E9FFD
:10A810001A0707F1070740F1768527F0070393ED44
:10A82000007B8DED147B03F108020E92DDE914121A
:10A8300022F000431A911B93DDE91A454FF0FF32D5
:10A84000204629461B4B08F0DFFF002840F0DA8441
:10A850004FF0FF32174B2046294608F0B7FF00287B
:10A8600040F0D08400220023DDE9140108F0A4FFA9
:10A87000002840F05A879DF87F700F4E0F4B0799C4
:10A8800021F080010791119903224FF0000B0892EB
:10A890004729D8BF1E460D92CDF84CB09AE6079BCB
:10A8A00043F00803079398F800301BE55C4D01085E
:10A8B000084D0108FFFFEF7F1C4D0108184D0108EE
:10A8C0001193AB46002A41F01780079B43F0100319
:10A8D0000793079A12F020037FF4BAAD079911F09D
:10A8E000100200F05B840E988DF87F30BBF1000FF2
:10A8F000046800F104074FF00005C0F21B850A460A
:10A9000022F08002079254EA05020E9700F03A8185
:10A910001F46B3E51193AB46002A40F0E987079B39
:10A9200043F010030793079A12F0200300F02C83E2
:10A930000E9F073727F00703002703F10801BB45E7
:10A940000E91D3E900458DF87F70C0F2568322F056
:10A950008003079354EA05037FF418AEBBF1000FA0
:10A9600000F0F580002444AE303406F8414D27E66F
:10A970001193AB46002A40F0B787079BAF489D066E
:10A9800040F1B5800E9F073727F00703D3E9004554
:10A9900003F108020E92079A12F0010700F03982C3
:10A9A00054EA050300F004859DF844208DF88120C9
:10A9B0000027079A8DF87F703023BB458DF88030D3
:10A9C00042F00203C0F2B68622F0800343F0020395
:10A9D000079334AE230904F00F0143EA05732A09F3
:10A9E0001C461546435C06F8013D54EA0503F1D1C7
:10A9F000E6E50E9911930A688DF8A82000230A460F
:10AA00001F468DF87F30043201230893BB4613970D
:10AA10000E920D932AAEE1E51193AB46002A3FF466
:10AA200093AD8DF87F108FE5079B43F040030793AC
:10AA300098F8003056E498F8003000297FF452ACC2
:10AA4000012220214EE4079B43F00103079398F86D
:10AA5000003047E40E9C23680C93184600282346D8
:10AA600003F10403FFF6A0AC0E9398F8003039E42C
:10AA700098F8003001222B2134E4079B43F0200397
:10AA8000079398F800302DE40E9A1193166800246D
:10AA90008DF87F40171D002E00F02186002DC0F29A
:10AAA00066852A4621463046FDF782FE002800F0E2
:10AAB0006B86831B0D93A34623EAE3730E970893DB
:10AAC000CDF84CB09DF87F7084E51193AB46002A19
:10AAD0003FF429AF8DF87F1025E71193AB46002A8C
:10AAE00040F01687079B56489D063FF54BAF079BE6
:10AAF000DC0640F140840E9A1346043314680E932A
:10AB0000002548E798F800306C2B00F0C4840798C3
:10AB100040F010000790FFF7E5BB002A40F0F486F4
:10AB2000079B9B0640F157830E9A0B991368CD172C
:10AB30000846043229460E92C3E90001FFF79FBB85
:10AB40003F481192BBF1000F40F074815F464FF017
:10AB5000000BCDF834B034AE35E51193002A40F047
:10AB6000CF86119A002A3FF456AC002301211F46DC
:10AB700008918DF8A8208DF87F309B4613930D9196
:10AB80002AAE2BE5BBF1000F00F01686002700244B
:10AB9000002573E42A480793119254EA05030E979F
:10ABA0004FF000077FF415AF0024002511E7299C22
:10ABB00064E5119B652B40F3AA8000220023DDE9A8
:10ABC000140108F0EFFD002800F03681289B1D4A93
:10ABD000C9F80020013301340122072B299428935E
:10ABE000C9F8042000F3F08309F10809219B129AA7
:10ABF000934203DB079BDB077FF5B0AD289B1699DB
:10AC0000179AC9F8002001330C44072B2994C9F87E
:10AC10000410289300F3498409F10809129B5D1E72
:10AC2000002D7FF79BAD084A289B0F92102D40F313
:10AC3000E98110260A9FDDF824B00DE0284D0108B7
:10AC40003C4D0108584D0108084D010809F108095B
:10AC5000103D102D40F3D68101331034072B299479
:10AC60002893C9F800A0C9F80460EFDD27AA594667
:10AC7000384606F037FE00287FF4D4AB299C289B89
:10AC80000DF1D009E4E70C9B089A9F1A002F7FF77B
:10AC900019ADBC4A289B0F92102F2BDD4A46214646
:10ACA000B946102537460A9C099E06E0A9F110090D
:10ACB000B9F1100F02F1080218DD01331031072B32
:10ACC00029912893C2F800A05560EFDD27AA3146EC
:10ACD000204606F007FE00287FF4A4ABA9F1100976
:10ACE000B9F1100F2999289B34AAE6DC3E460C46A0
:10ACF0004F46914601330F9A28933C44072B2994E1
:10AD000089E8840000F33D8209F10809DAE4129B26
:10AD1000289D012B40F30A82013501340123072DC0
:10AD200029942895C9F80060C9F8043000F30F820F
:10AD300009F10809169A179BC9F800300135144427
:10AD4000072D29942895C9F8042000F30D8209F1F4
:10AD5000080900230022DDE9140108F023FD129BFD
:10AD6000002840F0C380013B013501361C44072D0B
:10AD700028952994C9F80060C9F8043000F3F580DB
:10AD800009F10809199AC9F804200135144423ABC4
:10AD9000072D29942895C9F800307FF7DDAC27AA44
:10ADA00009990A9806F09EFD00287FF43BAB299C88
:10ADB0000DF1D009D2E427AA09990A9806F092FD6C
:10ADC00000283FF419ADFFF72DBB27AA09990A986F
:10ADD00006F088FD00287FF425AB299C0DF1D009F1
:10ADE000A9E427AA09990A9806F07CFD00287FF4B7
:10ADF00019AB299C0DF1D00950E427AA09990A98AA
:10AE000006F070FD00287FF40DAB299C0DF1D009F0
:10AE100054E4BBF1000F8DF87F70C0F2E18222F0A4
:10AE20008003079354EA05037FF4D3ADBBF1000F11
:10AE30003FF48CAE0027B7E6219D002D40F3D3826E
:10AE4000139B129A9342A8BF1346002B1D460DDD9B
:10AE5000289BC9F8006001332C44072B2994C9F8BA
:10AE60000450289300F3AE8309F10809139B002DC9
:10AE7000A8BF5B1B002B1D4640F3F880414A289B6E
:10AE80000F92102D40F3858222461027DDF828B05E
:10AE9000099C05E009F10809103D102D40F3788266
:10AEA00001331032072B29922893C9F800A0C9F862
:10AEB0000470EFDD27AA2146584606F013FD00284E
:10AEC0007FF4B0AA299A289B0DF1D009E4E727AABC
:10AED00009990A9806F006FD00287FF4A3AA9DF8B8
:10AEE0007F70299C0DF1D009FFF7C8BB5E1E002EB4
:10AEF0007FF748AF234B0F93102E2CDDCDF8348015
:10AF00001027B046DDF828B0099E06E0A8F1100829
:10AF1000B8F1100F09F108091ADD01351034072DB9
:10AF200029942895C9F800A0C9F80470EEDD27AA75
:10AF30003146584606F0D6FC00287FF473AAA8F1E3
:10AF40001008B8F1100F299C289D0DF1D009E4DC00
:10AF50004646DDF834800F9B01353444072D299493
:10AF6000289589E848007FF70BAF27AA09990A9826
:10AF700006F0B8FC00287FF455AA299C289D0DF105
:10AF8000D009FFE6084D0108079911F0100200F002
:10AF9000D5810E988DF87F30BBF1000F046800F169
:10AFA00004074FF0000526DB0A4622F080020792D4
:10AFB00054EA05020E971F467FF4E8AACEE4079BE9
:10AFC000D8062AD4079B590627D50E99B1F9004017
:10AFD0000431E51722462B460E91FFF7C4BA0E99AD
:10AFE0008DF87F30BBF1000F0C6801F104074FF0C2
:10AFF000000580F24E820E971F4654EA05037FF447
:10B00000C5AAB0E401330F9A28932C44072B299446
:10B0100089E824007FF7A0ABC1E60E9A14681346B6
:10B020000433E51722460E93002A2B4673F10003E2
:10B03000BFF69EAA64424FF02D0765EB4505BBF1B4
:10B04000000F8DF87F70FFF6A1AA079B23F0800305
:10B050000793FFF79BBA27AA09990A9806F042FCC2
:10B0600000287FF4DFA9299C0DF1D009139A219BB8
:10B0700032441746129A934247DB079AD50744D4C5
:10B0800012990E44F51BCB1A9D42A8BF1D46002DF8
:10B090002E460DDD289AC9F8007001322C44072A8B
:10B0A0002994C9F80450289200F30A8309F1080989
:10B0B000002EACBF9D1B1D46002D7FF74FABBB4A3A
:10B0C000289B0F92102D9DDD10260A9FDDF824B0DD
:10B0D00004E009F10809103D102D93DD013310340F
:10B0E000072B29942893C9F800A0C9F80460F0DD63
:10B0F00027AA5946384606F0F5FB00287FF492A9A6
:10B10000299C289B0DF1D009E5E7289A16981799F4
:10B11000C9F8001001320444072A2994C9F8040030
:10B12000289200F3B98209F10809A9E7079BD8071B
:10B130003FF5F2AD013501340123072D29942895FF
:10B14000C9F80060C9F804307FF71AAE0DE727AAE6
:10B1500009990A9806F0C6FB00287FF463A9299C88
:10B16000289D0DF1D009E5E527AA09990A9806F06E
:10B17000B9FB00287FF456A9299C289D0DF1D00920
:10B18000E7E527AA09990A9806F0ACFB00287FF4A6
:10B1900049A9299C0DF1D009FFF794BA079911F03C
:10B1A000400300F0BB800E988DF87F200346BBF172
:10B1B000000F03F1040304884FF00005C0F2C581BD
:10B1C00021F08001079154EA05010E933FF4DAACB7
:10B1D0001746FFF753B9079BDF060BD4079B5E06A4
:10B1E00008D50E9A136804320E92BDF82C201A80EE
:10B1F000FFF745B80E9A136804320E920B9A1A6044
:10B20000FFF73DB8DDE9140102460B4608F0FCFAF1
:10B21000002840F00583119BBBF1FF3F23F020077E
:10B2200000F06C82472F00F08781159B079A002B56
:10B2300042F480720F92C0F280829DED147B8DEDFE
:10B240001C7B00230893119B662B00F05A82462B2F
:10B2500000F04781452F0CBF0BF101055D4625A885
:10B2600022A921AA02230490029200930195DDE90C
:10B270001C2303910A9803F0BBFA119B672B064627
:10B2800040F07182079BDA0740F1BF8274190022F7
:10B290000023DDE91C0108F085FA002840F09081C8
:10B2A000259B9C4206D930215A1C25921970259B5A
:10B2B0009C42F9D89B1B472F129300F07A81119B77
:10B2C000652B40F35F82119B662B219B139300F04B
:10B2D0006682139A12998A42C0F23882079BD90774
:10B2E00000F1958222EAE2730D9267221192089A88
:10B2F000002A40F0328108930F9B079393469DF8F4
:10B300007F70FFF767B927F0070797ED007B07F11C
:10B3100008038DED147B0E93FFF788BA0E998DF814
:10B320007F30BBF1000F0C6801F104074FF00005FE
:10B3300080F2AC800E970027FFF7A0B8079911F0B4
:10B3400040033FF44CAE0E988DF87F200346BBF1CE
:10B35000000F03F1040304884FF00005C0F2F280EF
:10B3600021F08001079154EA05010E9317467FF4FE
:10B370000DA9FFF7F3BA079B0E9A13F0400F13467F
:10B3800000F0E580043314880E930025FFF703BB1B
:10B39000144601330F9A28932C44072B299489E8EB
:10B3A00024003FF758AE09F108095FE6084D01088F
:10B3B0000027BB458DF87F70FFF6F6AB079B23F0A7
:10B3C00080030793FFF7BEBB27AA09990A9806F0E6
:10B3D00089FA00287FF426A8299C0DF1D00905E4FC
:10B3E0000E9FFFF7DABB289BB24AC9F80020013351
:10B3F00001340122072B29942893C9F8042000F373
:10B400008E8009F108092DB9129B1BB9079BDF0734
:10B410007FF5A4A9289B1699179AC9F80020013333
:10B420000C44072B2994C9F80410289300F3D38106
:10B4300009F108096D42002D40F3AD809E4A0F923C
:10B44000102D40F3CC8022461027DDF828B0099C4F
:10B4500005E009F10809103D102D40F3BF800133CC
:10B460001032072B29922893C9F800A0C9F804705C
:10B47000EFDD27AA2146584606F034FA00287EF46C
:10B48000D1AF299A289B0DF1D009E4E7079AFFF77D
:10B4900037BA079A89E5079B43F02003079308F121
:10B4A000010898F80030FEF71DBF27AA09990A98ED
:10B4B00006F018FA00287EF4B5AF299C0DF1D009EA
:10B4C000FFF7ACBB40210A98FCF7B4FE099A106064
:10B4D0001061002800F0F981099A40235361FEF7BA
:10B4E000BEBE25A822A921AA03230490029200939C
:10B4F000CDF804B00391DDE91C230A9803F078F934
:10B500005D460646119B462B06EB05047FF4BFAE55
:10B510003378302B00F08A81219D2C44B7E627AA8E
:10B5200009990A9806F0DEF900287EF47BAF219D88
:10B53000299C0DF1D00966E7BBF1000F08BF4FF061
:10B54000010B72E60E93174657E50E93F3E60433AC
:10B5500014680E930025FFF71EBA2D2708930F9B42
:10B5600007938DF87F704FF0000BFFF734B830462B
:10B57000FEF7A6FCA34603460D90FFF79DBA27AA47
:10B5800009990A9806F0AEF900287EF44BAF299C81
:10B59000289B0DF1D0091299C9F8006001330C44C1
:10B5A000072B29942893C9F804107FF7D5A8FFF733
:10B5B000F6BB219BDD1C1EDB9B451CDB139388E641
:10B5C000234677E627AA09990A9806F08BF90028FE
:10B5D0007EF428AF299C0DF1D00947E414460133CD
:10B5E0000F9A28932C44072B299489E82400C6DC61
:10B5F00009F10809CFE7119A023A1192013B002B99
:10B600009DF844202193B8BF5B428DF88C20B4BFD5
:10B610002D222B22092B8DF88D2040F3EE800DF189
:10B620009B000446254A82FB0321DA17C2EBA102E4
:10B6300002EB8201A3EB410303F13001092A134617
:10B6400004F8011DEEDC21463033DAB201F8012D99
:10B65000884240F237810DF18E01234601E013F854
:10B66000012B01F8012B9842F9D1431C1B1B0DF152
:10B670008E02134423AA9B1A129A1993012A134487
:10B680000D9340F3EA800D9B169A134400220D930C
:10B69000139223EAE3732AE627AA09990A9806F087
:10B6A00021F900287EF4BEAE219B299C0DF1D00922
:10B6B000E6E400BF584D0108084D0108676666665C
:10B6C00027AA09990A9806F00DF900287EF4AAAE77
:10B6D000219B129A299CD31A0DF1D009E8E4062D7A
:10B6E0002B4628BF06230D9323EAE373B3460E9738
:10B6F000139637460893884EFEF76CBF4FF0060B43
:10B7000093E525A822A921AA03230490029200937D
:10B71000CDF804B00391DDE91C230A9803F068F822
:10B720005D46064600EB0B04F2E62D278DF87F7090
:10B73000FFF7A3B80793FFF74CB9DDE9141202F144
:10B7400000431D932D231C9108937CE5169A129BB0
:10B750001344139A0D93002A40F38980672223EA49
:10B76000E3731192C3E5119B472B7FF48FAD079BC9
:10B77000DB073FF5C7AE259B472FA3EB06031293CC
:10B780003FF417AF219B39E725EAE5730E9708933D
:10B790000D95834613909DF87F70FEF71BBF002B1D
:10B7A0006DDDBBF1000F4FD1079AD4074CD41A4678
:10B7B0000D9223EAE3739AE5079BDB075F4605D505
:10B7C00044AE302306F8413DFEF7FABECDF834B062
:10B7D00034AEFEF7F8BE27AA09990A9806F082F857
:10B7E00000287EF41FAE219D299C289B0DF1D009D5
:10B7F00020E6A0460025FEF777BD303330228DF8D5
:10B800008F308DF88E2024AB34E7259B52E5169AB5
:10B81000139B134467220D93119223EAE37366E5A9
:10B820003E4E3F4B9DF87F70FFF729B80022002362
:10B83000DDE91C0107F0B6FF00287FF46DAEC5F10D
:10B84000010521952C4422E5139B169A9D1805EBC2
:10B850000B030D9323EAE37349E5079B13F0010300
:10B860007FF411AF13930D9B23EAE3733FE5139B22
:10B870000D9AC3F101031A4413460D926EE7BBF112
:10B88000000F02D1079BD80707D5169B5D1C05EB5F
:10B890000B030D9323EAE37329E501230D9326E5BA
:10B8A0000E9898F8013005680430002D0E90A046DF
:10B8B000BEF618AD4FF0FF35FEF714BD8DF87F10C2
:10B8C000FEF7C1BD0DF18E03D4E60A9A0C23136076
:10B8D0004FF0FF30FEF7AFBD8DF87F10FEF730BEA2
:10B8E0008DF87F10FEF792BF8DF87F10FFF745B8F7
:10B8F0008DF87F10FFF713B88DF87F10FEF7E5BFC6
:10B900008DF87F10FFF72DB98DF87F10FFF708B97C
:10B910008DF87F10FFF7E6B8504D0108244D01085F
:10B92000204D01082DE9F04F8B46B1F90C10ADF513
:10B930002B7D824688041446049309D4DBF86430D6
:10B9400041F4005123F40053ABF80C10CBF86430F1
:10B9500026460023069303931F46059316F8013BE2
:10B960000F936BB304F002F80F9A1044437803F07E
:10B97000080303F0FF0543B3DBF8043011E003F0E4
:10B98000F5FFDBF800301A781044013342781107D4
:10B990000FD5DBF80420CBF80030531E0137CBF86D
:10B9A0000430002BEBDC5946504606F05DF80028C9
:10B9B000E5D03446264616F8013B0F93002BD1D133
:10B9C00005980DF52B7DBDE8F08F252A40F0848089
:10B9D00094F801802C46731CB8F1780F00F2438272
:10B9E000DFE818F0920041024102410241024102A7
:10B9F000410241024102410241024102410241022F
:10BA0000410241024102410241024102410241021E
:10BA1000410241024102410241024102410241020E
:10BA200041024102410241024102410241027900C8
:10BA30004102410241024102D80141024102410258
:10BA400041024102CF01CF01CF01CF01CF01CF0190
:10BA5000CF01CF01CF01CF0141024102410241029A
:10BA6000410241024102410241024102C101B901C8
:10BA70004102B9014102410241024102B3014102C6
:10BA80004102A3014102410241024102410241023D
:10BA9000410241029301410241025101410241022E
:10BAA0004102410241024102410222018801B901E1
:10BAB000B901B9011C01980041024102D5004102BF
:10BAC0000D010101F30041024102EB004102DF00E0
:10BAD0004102410293011E46DBF80430002B40F383
:10BAE0005382DBF8003016F8012C197891427FF46C
:10BAF00067AFDBF804200133013ACBF8003001379F
:10BB0000CBF80420344655E74FF0FF300DF52B7D80
:10BB1000BDE8F08F0293DBF80430002B40F3638222
:10BB2000B84B069300230393032601E0CBF800E013
:10BB300003F01CFFDBF800201178084402F1010E2D
:10BB4000437803F0080303F0FF08002B00F07F8226
:10BB5000DBF80430013B002B07F10107CBF8043080
:10BB6000E4DC5946504605F07FFF0028E0D0059AF6
:10BB7000002AC9D0BBF80C3013F0400F134618BF91
:10BB80004FF0FF3318460DF52B7DBDE8F08F96F88A
:10BB90000180B8F16C0F00F0028245F001051E46ED
:10BBA00019E70293DBF80430002B40F34882964BF0
:10BBB00006930A2303930326BAE70293DBF80430C3
:10BBC000002B40F334820226B2E70293DBF8043004
:10BBD000002B45F4087540F3A0808B4B069310238F
:10BBE00003930326A4E70293DBF80430002B40F311
:10BBF000A480854B069308230393032698E7EA065F
:10BC00001E46029300F1F2806B0740F1D481049943
:10BC10000B681F800B1D04933446CBE696F8018019
:10BC200045F004051E46D6E60293DBF80430002BEF
:10BC300040F3ED81002C08BF012415F0010340F012
:10BC40002281EA0640F18B811D4609E01344CBF8BE
:10BC500000301544A41A05F007FF002840F07B814E
:10BC6000DBF80420DBF80030A24259465046EDDBF9
:10BC7000121B2344CBF804202544CBF80030029E4D
:10BC80002F44344696E60DF148091946484604F01B
:10BC90005DFBDBF80430002B064640F3B081002C3E
:10BCA000DBF8002008BF4FF0FF34EB06117840F1BD
:10BCB000A080A046002500E0117819F8013001327B
:10BCC000002B00F04381DBF80430CBF80020013575
:10BCD000013BA542CBF8043000F03581002BEBDCB2
:10BCE0005946504605F0C0FE002840F02B81DBF895
:10BCF0000020E1E70293DBF80430002B3ADD414BF2
:10BD000006930A230393032612E70293DBF8043019
:10BD1000002B45F400753FF760AF5946504605F0DB
:10BD2000A3FE00283FF459AF21E70293DBF804306B
:10BD3000002B45F001053FF75CAF5946504605F032
:10BD400093FE00283FF455AF11E796F8018045F0C7
:10BD500002051E463FE60293DBF80430002B40F359
:10BD60005E810426E4E60293DBF80430002B45F004
:10BD70000105C4DC5946504605F076FE0028BED0C9
:10BD8000F5E604EB840408EB4404303C96F80180AB
:10BD90001E4620E696F8018045F010051E461AE67C
:10BDA00010AB4146184608220793FCF781FE15F0B8
:10BDB000100940F05D84049A13460433D2F80080E1
:10BDC0000493002603F0D2FDDBF800301B78184402
:10BDD0004378180702D4002C40F0FC83B9F1000F1F
:10BDE00004D1C8F80090059B01330593029E3446A8
:10BDF000E0E5049805680346043305EB0408029364
:10BE00002C4606E0DDA1000885160108DBF80020BD
:10BE1000117819F80130501CC3B1DBF80430CBF8AD
:10BE20000000013BCBF80430137804F8013BA04537
:10BE30000CD0DBF80430002BE8DC5946504605F006
:10BE400013FE0028E2D0A5423FF491AE651B3FF4FB
:10BE5000B7AD059A013200230592029A049223702D
:10BE60002F443446A6E5029303F080FD4044437816
:10BE700003F00303012BDBF8043000F09680002B65
:10BE80003FF73DAF76E710AB184608220021079335
:10BE9000FCF70EFE15F0100308937DD1049A1346AB
:10BEA0000433D2F80090049300250DF5A47803F034
:10BEB0004BFDA8423FF45BAE9BE80C0012F8010B6F
:10BEC000CBF80020013B079A00926E1CCBF804309F
:10BED000494608F8050033464246504603F076FDD1
:10BEE000411C3FF444AEA0B9089B13BBC9F8003015
:10BEF0003744013C09F10409DBF80430002B4FF012
:10BF000000050DDD002CD2D1089B002B3FF46BAF58
:10BF10006CE7023010D1DBF80430002B3546C6DC6C
:10BF20005946504605F0A0FD0028EBD0002DEBD07F
:10BF30001DE63744013CDFE7089B3744013C002BFA
:10BF4000DAD1D7E7A84645462F448AE7002D3FF4CB
:10BF500037AD2F4485E7002D7FF491AE07E6049DB1
:10BF600023462968CDF800B00122504605F09AFD1D
:10BF70002E1D00283FF4FBAD059B0496029E013365
:10BF800007440593344615E55946504605F06CFDC7
:10BF900000283FF4A6ADEAE54FF0000984E796F8E3
:10BFA000028045F00205023615E5002B45F001053B
:10BFB0003FF7A5AEDEE6EC070CD4A8070AD5049A35
:10BFC000029E13683846F91704320492C3E900014F
:10BFD0003446EFE4049A029E13681F60134604334C
:10BFE00004933446E6E45946504605F03DFD0028EA
:10BFF0007FF4BDAD7E4B03900693032698E559462A
:10C00000504605F031FD00283FF449AEAFE55946F2
:10C01000504605F029FD00283FF40CAEA7E559462F
:10C02000504605F021FD00283FF49BAE9FE55946A0
:10C03000504605F019FD00283FF4C5AD97E5594677
:10C04000504605F011FD00283FF4B1AD8FE5032EF9
:10C0500000F09B81042E40F03982504603F092FCA0
:10C06000631E02680A92B3F5AE7F40F263826FF4FA
:10C07000AE7163180C9340F25D1452AB4FF00008A0
:10C080001A46089345F4F0654346CDF83480CDF860
:10C090002C804646CDF824809146DBF800000178DC
:10C0A000A1F12B0EBEF14E0F00F24781DFE81EF02A
:10C0B0007A0045017A00450145016E004F004F00AE
:10C0C0004F004F004F004F004F004F004F00450101
:10C0D0004501450145014501450145014001450135
:10C0E000450145012801210145014501A200450105
:10C0F0004501450145018B004501450145014501CB
:10C100004501850045014501450145017F00450187
:10C1100045014501450145014501450140014501F4
:10C12000450145012801210145014501A2004501C4
:10C130004501450145018B0045014501450145018A
:10C140004501850045014501450145017F0013EB8F
:10C15000080F16D125F4C07589F8001009F10109FE
:10C16000DBF804100139002904F1FF3407F101075D
:10C17000CBF8041040F3EE800130CBF80000002C27
:10C180008BD1002E42D025F480753FE0EA05DED544
:10C190000C9A25F080050136002AE1D0013A0C9274
:10C1A0000134DDE72A06ECD525F08005D4E7B8F1A7
:10C1B000070FE6D14FF00808CEE7B8F1060FE0D13F
:10C1C0004FF00708C8E7002B40F0DA802EB905F4DD
:10C1D000E06EBEF5E06F00F03F82B8F1010F02D0D3
:10C1E000B8F1040FCDD108F101085FFA88F8B3E780
:10C1F000DDA10008B8F1000F40F0B980002EC2D1D7
:10C2000005F4E06EBEF5E06F00F03682013B012BD5
:10C2100040F27D8208F1FF33062B16D8B8F1020FE9
:10C2200040F29C82B8F1030F0FD0A8F10404E4B2ED
:10C230006FEA0408C84419F8011D5A46504605F033
:10C24000D1FBC845F7D1013F3F1BE9051CD56A0565
:10C2500000F16F8219F8011C652909F1FF3407F11B
:10C26000FF380BD0452909D05A46504605F0BAFB95
:10C2700019F8021CA7F10208A9F102045A46504617
:10C2800005F0B0FB4746A14615F010027FF4AEADB5
:10C2900005F4C063B3F5806F89F8002000F0F181E8
:10C2A0000B9B002B40F0FE8108990022504605F0C0
:10C2B0003DF8EB078046894600F13F8115F0020505
:10C2C00040F03B81049C02460B46261D246807F083
:10C2D0009BFA002840F05C824046494607F0F2FA9B
:10C2E00004962060059B029E013305933446FFF7B8
:10C2F00061BBB8F1020F7FF444AF4FF003082BE7A6
:10C3000005F4A06EBEF5806F05D06A057FF539AFE4
:10C31000002E3FF47BAFAA0504D4099ACDF83490DF
:10C32000B21A0B9225F4F06545F4C075002613E7A8
:10C33000012B7FF426AF02230EE70A9A92F800E061
:10C340008E457FF41EAFAA057FF51BAF25F420753F
:10C35000099601E759465046079305F085FB079B70
:10C3600000287FF40EAF002C7FF497AE09E7B8F1F8
:10C37000030F3FF438AFB8F1050F3FF434AF00E7D7
:10C38000022B7FF42AAF0323E6E6631EB3F5AE7FEC
:10C3900086BF6FF4AE7004EB0009C14652AB104685
:10C3A0003A464F46DDF80C90089388BF40F25D1482
:10C3B00045F458651E464FF00008A1F12B034D2BA4
:10C3C00051D8DFE803F07E507E50506F696969698B
:10C3D0006969694A4A50505050505050444444444E
:10C3E0004444505050505050505050505050505065
:10C3F0005050502750505050505050504444444496
:10C400004444505050505050505050505050505044
:10C410005050502705F4C063B3F5007F23D125F4B5
:10C42000007545F4A0654FF0100931700136DBF856
:10C430000430013B002BCBF8043072DD0130CBF827
:10C440000000013C0FD0DBF800000178B5E7B9F13E
:10C450000A0F08DD25F43865E7E7BD4B33F919907D
:10C46000B9F1080FF6DCE9051746CDF80C9007D5B1
:10C47000089B9E4200F2F480089B9E423FF4A0AAD3
:10C4800015F0100400F09280089BF61A46443744D9
:10C49000029E3446FFF78EBAAD4B25F4386533F96A
:10C4A0001990C2E72B05C0D5B9F1000F03D145F4AF
:10C4B00000754FF008096B0540F1C08025F4B065A8
:10C4C000B3E72B06CFD525F08005AEE7002C08BFDB
:10C4D0004FF0FF3415F001037FF462ACE90633D569
:10C4E0001D4603F043FADBF800301A78104401339C
:10C4F000427812073FF5C3ABDBF80420CBF80030DD
:10C500000135531EAC42CBF804303FF4B8AB002BDE
:10C51000E7DC5946504605F0A7FA0028E1D0FFF7BE
:10C52000AEBB59465046039205F09EFA039A002886
:10C5300087D098E7CDF830809FE5049A13680432DD
:10C540000492C3E90089CDE6049A1568161D2C44AF
:10C55000A84603F00BFADBF8002013781844511CAE
:10C5600043781B0715D4DBF80430CBF80010013BEF
:10C57000CBF80430137808F8013B44450AD0DBF8C7
:10C580000430002BE5DC5946504605F06DFA0028D2
:10C59000DFD04446059A0496029E651B00230132B3
:10C5A00023702F4405923446FFF704BA22463470B4
:10C5B000039B0899069C5046A047AA0646D46B07E1
:10C5C0007BD5049A1368043204921880059B0133CA
:10C5D000059359E703F0B8F986423FF4C8AA9BE8EF
:10C5E0000C0012F8010BCBF80020079A009252AA17
:10C5F000751C013B9055CBF8043041462B46504604
:10C6000003F0E4F9461C3FF4B2AA00286BD1C8F845
:10C61000000003F07FF9002800F0AF80002D3FF408
:10C62000DDAB52AB5C19013D5A4614F8011D504672
:10C6300005F0D8F9002DF6D1FFF7D0BB25F46075D1
:10C640000FB1013F013408F10108F0E6049A1368C4
:10C65000043204921860B9E725F4F06501237BE504
:10C6600016F8011C5A46504605F0BCF9013E03E796
:10C670000DF13C08FFF7A5BB25F4F0654FF001086C
:10C680006AE5099BF61A7242002E3FF40DAE0DF2D8
:10C690009B23994528BF0DF29A2948462D49FDF75D
:10C6A0000DF901E60D9C21460A2301315046FDF7A4
:10C6B00095FD0B9BA146C21AE9E715F00102C5D111
:10C6C000AC07C3D5069B1946234B99425046039BA2
:10C6D000089963D004F010FF049A1368043204929E
:10C6E000C3E9000172E7023020D12E46DBF80430A6
:10C6F000002B3FF767AB5946504605F0B5F90028C7
:10C700003FF460AB002E7FF432AAFFF767BB089BB3
:10C7100099457FF655A919F8011D5A46504605F06E
:10C7200061F9089B9945F6D1FFF74AB9D8F800009E
:10C730006FE7089B99457FF643A919F8011D5A46F2
:10C74000504605F04FF9089B9945F6D1FFF738B9E7
:10C750006C4D0108904D010885160108089B99450C
:10C760007FF62EA919F8011D5A46504605F03AF9F0
:10C77000089B9945F6D1FFF723B92F44013CB9F145
:10C78000000F03D108F104084E46AFE70646ADE7B7
:10C79000284603F015FE04962060A3E505F090F806
:10C7A0009AE700BF2DE9F04F83B0044602F0B6FFD0
:10C7B00040F2B1739C4240F39B805B49446081FB33
:10C7C0000437E517A4F26D726FF4F66304EB030C03
:10C7D000C5EBE71681FB02E34FF4C878D2176FF47C
:10C7E000C8694FEAAC0E08FB1646A4F2B27CA2EB75
:10C7F000631240F26D1804EB090308FB0CEC81FB9B
:10C8000003E1DB17C3EBE1136244C5EB67154FF09F
:10C81000640EB6FA86F702EB030C04F003030EFB7A
:10C8200015457F090193044600F1380E237A4A2BFF
:10C8300062D0442B71D0019B002B54D03B464FEA71
:10C84000430AE1689A44394B012903EB0A1A67DD70
:10C8500001F1804102394FEA81090AEB0908AAF186
:10C860000402634652F8041F90450B44FAD109F1C3
:10C8700004012F4A5AF8011003F1040B8BFB0289C3
:10C880000BEB09084FEAEB72C2EBA802C2EBC2083D
:10C890006269C8EB0B0BB2EB0B0B226902F1FF32A2
:10C8A00048BF0BF1070BC2EBC2025A448A4202DBBB
:10C8B000073A8A42FCDA1344226AA16900921D4AAF
:10C8C00002FB0311009B194444F81C1F7445ADD1B1
:10C8D000C369826B9342ACBF002301230360012034
:10C8E00003B0BDE8F08F002D0CBF3B460123A6E747
:10C8F000002003B0BDE8F08F636901990CEB0302DF
:10C9000039B935B13B2BD4BF002301231344013B7C
:10C91000D2E7002EF6D00023F8E763696344CBE743
:10C9200063460021A5E700BF1F85EB51A84C010815
:10C930009324499280510100704700BF704700BFA7
:10C94000014B186800F002B8E80500202DE9F04717
:10C950008AB0064602F0E2FEB949BA4D07463046B3
:10C9600002F0D4FE0446002800F0F480296831B1BA
:10C97000FDF7CAF810B90AB0BDE8F0872968084683
:10C98000FBF750FC2046FDF79BFA411C3046FBF7B5
:10C9900051FC286010B12146FDF720FA2378AA4AFD
:10C9A000AA493A2B08BF013408AD2B46204603F0B4
:10C9B0000BFD0028DFDD089BE25C2D2A1C4400F003
:10C9C000C5802B2A08BF01344FF0010806AB029343
:10C9D0000DF11603002600930395019505AA2B4639
:10C9E0009B49ADF816602046ADF8186003F0ECFCEA
:10C9F000B042C0DDBDF81630BDF81810BDF81420E7
:10CA00000898DFF868A2DFF85492C3EB031301EB38
:10CA100083034FF4616101FB023308FB03F33B62C4
:10CA20000444894BC9F800302046524687492B46BA
:10CA300003F0CAFCB0427FDD0898C9F804A0235C6B
:10CA40002D2B044400F093802B2B08BF01344FF0B2
:10CA5000010806AB02930DF116030026009303951F
:10CA600001952B4605AA7A49ADF814602046ADF829
:10CA70001660ADF81860089603F0A6FCB0427ADDA7
:10CA8000BDF81630BDF81810BDF81420C3EB031321
:10CA900001EB83034FF4616101FB023308FB03F3F5
:10CAA000FB63089BB8461C444FF0000926782C2EE7
:10CAB00004BF667801344D2E62D04A2E08BF01347F
:10CAC0004FF00A0209A920460CBFB2464FF0440AB3
:10CAD00004F0EAFD099EADF81E00B44200F09A8011
:10CAE00080B2C8F8140088F808A000240223ADF82A
:10CAF0001430ADF81640ADF81840089433782F2B59
:10CB00006BD04FF4E15309F10109B9F1020FC8F8F4
:10CB10001830344408F11C08C8D17868FFF742FE89
:10CB20003A6AFB6B4B484C499B1A18BF01230360C0
:10CB30000A600AB0BDE8F0874749464A386AD9F822
:10CB4000003008601660C9F8043014E701344FF073
:10CB5000FF383BE7414B3F493F4E414A286834602C
:10CB60000C601A605A60FBF75DFB2C6003E7013430
:10CB70004FF0FF386DE73B6AA3F56163FB6390E715
:10CB80000DF11E0207AB02920093039501952B460F
:10CB90000DF11A023349204603F016FC03287FF4F6
:10CBA000EAAEBDF81A305A1E0B2A3FF6E4AEBDF8C5
:10CBB0001C20511E04293FF6DEAEBDF81E100629CA
:10CBC0003FF6D9AE88F80860C8F80C30C8F81020D5
:10CBD000C8F81410089E264487E706AB02930DF1AF
:10CBE0001603009305AA2B461F490395019530466D
:10CBF00003F0EAFBBDF81610BDF81830BDF814209C
:10CC0000089CC1EB011103EB81014FF4616303FB4D
:10CC1000021378E7B9F1000F09D04D220B2387F8F2
:10CC20002420BB6201220023FA623B635DE74D23AF
:10CC300003223B720223C7F81490FA603B6154E769
:10CC4000984D0108FC190020F0190020A04D0108A2
:10CC5000B04D0108001A0020041A0020FC09002031
:10CC60009C4D0108C44D0108D84D0108E41900206D
:10CC70002DE9F04FC5B01C460891164605460A90AE
:10CC800002F080FE036817931846FDF719F90E9419
:10CC900016901DB1AB6B002B00F023810898B0F902
:10CCA0000C2093B2990407D4416E42F4005321F44E
:10CCB0000051838141669BB21A0740F1DD80089ADA
:10CCC0001269002A00F0D88003F01A030A2B00F042
:10CCD000E1809FED877B00238DED147B12932993D8
:10CCE000289319930B93DFF814A234AB279399463A
:10CCF000B04698F800304446EBB1252B02D11AE03B
:10CD0000252B03D014F8013F002BF9D1C8EB040503
:10CD10008DB1289B299AC9F8008001332A44072B3A
:10CD2000C9F804502992289300F3C28009F1080938
:10CD30000B9B2B440B932378002B00F0C280002325
:10CD40001A468DF87F3019460C9307934FF0FF3B3E
:10CD5000637804F101085D4608F10108A3F12000A1
:10CD6000582800F25984DFE810F00F0457045704E4
:10CD70001804570457045704570457045704620310
:10CD8000490457045D00090157042501700370032D
:10CD90007003700370037003700370037003570413
:10CDA00057045704570457045704570457045704AB
:10CDB000570480039D0357049D03570457045704E9
:10CDC0005704EB03570457042C0157045704570426
:10CDD00057045704550157045704B4025704570425
:10CDE000570457045704570457045704570457046B
:10CDF000F5020F039D039D039D033F030F0357049B
:10CE00005704460357045003CB0064002004570422
:10CE100028045704F20357045704FA030C980E939E
:10CE200040420C90079B43F00403079398F80030AE
:10CE300092E70E98AB46002104688DF87F10071D1D
:10CE40000798302378228B458DF880304FF000050D
:10CE50008DF8812040F00203C0F2FB8320F08003B4
:10CE600043F00203079354EA05030E9700F0CC83C6
:10CE70000F46119220485DE208990A9801F08CFB58
:10CE8000002841F03F80089B9B8903F01A030A2B7E
:10CE90007FF41FAF0899B1F90E30002BFFF619AFE0
:10CEA000234632460A9801F08BFA45B0BDE8F08F70
:10CEB00027AA08990A9805F0CFFB48B90DF1D009C7
:10CEC00036E7299B23B10A98089927AA05F0C4FBE5
:10CED000089B9B89590601F115800B9845B0BDE868
:10CEE000F08F0A98FAF7DCFAD8E600BFAFF30080BB
:10CEF00000000000000000003C4D0108EC4D01085E
:10CF00001193AB46002A41F03282079A12F02003B7
:10CF100064D00E9F073727F00703002703F10801AD
:10CF2000BB450E91D3E900458DF87F70C0F2BA86FB
:10CF300022F08003079354EA050300F0828334AEA5
:10CF4000E20842EA4572E90804F007030D46144678
:10CF5000303354EA050206F8013DF1D1079AD207B1
:10CF600040F19680302B00F093803022731E06F83B
:10CF7000012C34AAD21A0D921E468CE098F800308B
:10CF80002A2B08F1010401F0D081A3F13000092817
:10CF900098BF002501F26C8114F8013B05EB850573
:10CFA00000EB4505A3F130000928F5D945EAE57500
:10CFB000A046D3E6079B43F08003079398F8003020
:10CFC000CAE61193AB46002A41F0D981079B43F092
:10CFD00010030793079A12F020039AD1079911F0D2
:10CFE000100200F034860E988DF87F30BBF1000FF0
:10CFF000046800F104074FF00005C0F252860A46AB
:10D0000022F08002079254EA05020E9700F019837D
:10D010001F4694E71193AB46002A41F0A081079B7D
:10D0200043F010030793079A12F0200300F0FA84EC
:10D030000E9F073727F00703002703F10801BB45C0
:10D040000E91D3E900458DF87F70C0F2238522F060
:10D050008003079354EA050300F0BC81002D08BF4C
:10D060000A2CC0F01B8534AE204629460A22002334
:10D0700006F078FC303206F8012D204629460023C0
:10D080000A2206F06FFC04460D4654EA0503EBD174
:10D0900034AB9B1B0D930D9B5B45B8BF5B4609935F
:10D0A0000023139317B1099B01330993079B13F0D6
:10D0B00002030F9302D0099B02330993079B13F0DD
:10D0C0008403109340F0D2820C9B099A9D1A002D84
:10D0D00040F3CC82102D2999289AA84F27DD189665
:10D0E00048461024B946089E2F460A9D04E0103F8A
:10D0F000102F00F1080016DD0132A04B28921031EC
:10D10000072A299180E81800F1DD27AA3146284630
:10D1100005F0A2FA00287FF4DBAE103F102F29990A
:10D12000289A34A8E8DC189E3D464F4681460132D5
:10D130006C18072A29942892C9F80070C9F804507D
:10D1400000F328849DF87F7009F1080977B1289BC6
:10D15000013301340DF17F010122072B299428931B
:10D1600089E8060000F3A08309F108090F9B6BB161
:10D17000289B0133023420A90222072B29942893EB
:10D1800089E8060000F39C8309F10809109B802BB5
:10D1900000F0D0820D9BC3EB0B07002F33DD784AE4
:10D1A000289B0F92102F22DD22464FF0100B0A9D74
:10D1B000089C04E0103F102F09F1080916DD013327
:10D1C0001032072B2992289389E8000CF2DD27AA58
:10D1D0002146284605F040FA00287FF479AE103F3A
:10D1E000102F299A289B0DF1D009E8DC1446013351
:10D1F0000F9A28933C44072B299489E8840000F374
:10D20000478309F10809079BDD0500F13182289B5E
:10D210000D99C9F8006001330C44072B2994C9F813
:10D220000410289300F31E8309F10809079B58078F
:10D230003FD50C9B099A9D1A002D3ADD102D289B95
:10D240004E4F23DD22461026DDF828B0089C04E06E
:10D25000103D102D09F1080917DD013347492893C6
:10D260001032072B299289E84200F1DD27AA2146D6
:10D27000584605F0F1F900287FF42AAE103D102D34
:10D28000299A289B0DF1D009E7DC144601332C4480
:10D29000072B29942893C9F80070C9F8045008DDB9
:10D2A00027AA08990A9805F0D7F900287FF410AE4C
:10D2B000299C0B9B0C9A09998A42ACBF9B185B185E
:10D2C0000B93002C40F0DA82002328930DF1D00953
:10D2D0000FE51193AB46002A41F03D80079B29489A
:10D2E0009C0640F146810E9F073727F00703D3E9DC
:10D2F000004503F108020E92079A12F0010700F0B0
:10D30000EB8254EA050300F082859DF844208DF8F5
:10D3100081200027079A8DF87F703023BB458DF858
:10D32000803042F00203C0F23B8722F0800343F0DA
:10D330000203079334AE230904F00F0143EA057397
:10D340002A091C461546435C06F8013D54EA0503CC
:10D35000F1D19DE60E9911930A688DF8A82000235B
:10D360000A461F468DF87F30043201230993BB46DD
:10D3700013970E920D932AAE98E600BFFC4D01085C
:10D38000EC4D0108284D01081193AB46002A40F0EE
:10D39000EA87079B9B0674D50E9F073727F0070780
:10D3A000D7E9002307F108010E9114461D46002A13
:10D3B00073F10003C0F23A84BBF1000F9DF87F7057
:10D3C000C0F26883079B23F08003079354EA0503A8
:10D3D0007FF444AEBBF1000F40F008844FF0000B27
:10D3E000CDF834B034AE56E6079B43F040030793C4
:10D3F00098F80030B0E498F800306C2B00F0D58538
:10D40000079840F010000790A6E4002A40F09F879C
:10D41000079B9F0640F1E4840E9A0B991368CD1781
:10D420000846043229460E92C3E9000161E40E9CCD
:10D4300023680C9318460028234603F10403FFF6E3
:10D44000EDAC0E9398F8003086E4A3F13000002391
:10D450001C4618F8013B04EB840400EB4404A3F1E0
:10D4600030000928F5D90C9478E41193AB46002AD2
:10D4700040F06987079B43F010030793079B9B06C7
:10D480008AD4079BDF0600F19482079B5E0640F179
:10D4900090820E99B1F900400431E51722462B46DF
:10D4A0000E9184E71193AB46002A40F07087079BEA
:10D4B0000E9F1D0707F1070740F1878427F0070338
:10D4C00093ED007B8DED147B03F108020E92DDE9F4
:10D4D000141222F000431A911B93DDE91A454FF014
:10D4E000FF3220462946B54B06F08EF9002840F061
:10D4F000EB834FF0FF32B14B2046294606F066F928
:10D50000002840F0E18300220023DDE9140106F049
:10D5100053F9002840F04A869DF87F70A84EA94B29
:10D52000079921F080010791119903224FF0000B18
:10D5300009924729D8BF1E460D92CDF84CB0B1E5EF
:10D54000079B43F00803079398F8003004E4119315
:10D55000AB46002A3FF467AD8DF87F1063E5119369
:10D56000AB46002A40F00F87079B97489C063FF583
:10D57000BAAE079BD90640F198830E9A134604333E
:10D5800014680E930025B7E698F8003000297FF460
:10D59000E3AB01222021FFF7DFBB079B43F0010330
:10D5A000079398F80030FFF7D7BB079B43F02003A1
:10D5B000079398F80030FFF7CFBB0E9A11931668C7
:10D5C00000248DF87F40171D002E00F0B785002D38
:10D5D000C0F202852A4621463046FBF7E9F80028CA
:10D5E00000F01C86831B0D93A34623EAE3730E977A
:10D5F0000993CDF84CB09DF87F7053E598F8003052
:10D6000001222B21FFF7A8BB6F481192BBF1000F3D
:10D6100040F073815F46E1E61193002A40F0AB864B
:10D62000119A002A3FF44DAC002301211F460991B5
:10D630008DF8A8208DF87F309B4613930D912AAE6C
:10D6400034E5BBF1000F00F0DA8500270024002547
:10D6500075E45D480793119254EA05030E974FF065
:10D6600000077FF467AE0024002563E6299C6DE582
:10D67000119B652B40F3AE8000220023DDE91401ED
:10D6800006F090F8002800F03A81289B4F4AC9F82C
:10D690000020013301340122072B29942893C9F873
:10D6A000042000F3CE8309F10809219B129A9342CA
:10D6B00003DB079BD8077FF5B9AD289B1699179A0E
:10D6C000C9F8002001330C44072B2994C9F8041031
:10D6D000289300F3748409F10809129B5D1E002D44
:10D6E0007FF7A4AD3A4A289B0F92102D40F3B481E6
:10D6F00010260A9FDDF820B005E009F10809103D69
:10D70000102D40F3A98101331034072B299428935D
:10D71000C9F800A0C9F80460EFDD27AA59463846C9
:10D7200004F09AFF00287FF4D3AB299C289B0DF1CD
:10D73000D009E4E70C9B099A9F1A002F7FF72AADC6
:10D74000234A289B0F92102F2BDD4A462146B946CB
:10D75000102537460A9C089E06E0A9F11009B9F188
:10D76000100F02F1080218DD01331031072B299147
:10D770002893C2F800A05560EFDD27AA3146204665
:10D7800004F06AFF00287FF4A3ABA9F11009B9F1F6
:10D79000100F2999289B34AAE6DC3E460C464F46DA
:10D7A000914601330F9A28933C44072B299489E82A
:10D7B000840000F32B8209F10809EBE4FFFFEF7FFF
:10D7C0001C4D0108184D01083C4D0108584D010839
:10D7D000EC4D0108129B289D012B40F3D0810135AF
:10D7E00001340123072D29942895C9F80060C9F850
:10D7F000043000F3E18109F10809169A179BC9F872
:10D80000003001351444072D29942895C9F80420C7
:10D8100000F3DF8109F1080900230022DDE914018A
:10D8200005F0C0FF129B002840F0CC80013B013581
:10D8300001361C44072D28952994C9F80060C9F8C1
:10D84000043000F3AC8109F10809199AC9F80420E1
:10D850000135144423AB072D29942895C9F80030CD
:10D860007FF7E2AC27AA08990A9804F0F5FE002891
:10D870007FF42EAB299C0DF1D009D7E427AA089993
:10D880000A9804F0E9FE00283FF41EADFFF720BB24
:10D8900027AA08990A9804F0DFFE00287FF418AB45
:10D8A000299C0DF1D009AEE427AA08990A9804F042
:10D8B000D3FE00287FF40CAB299C0DF1D00955E470
:10D8C00027AA08990A9804F0C7FE00287FF400AB45
:10D8D000299C0DF1D00959E4BBF1000F8DF87F7040
:10D8E000C0F20D8322F08003079354EA05037FF40E
:10D8F00021ADBBF1000F3FF48DAE0027B3E6219DB3
:10D90000002D40F3AA82139B129A9342A8BF13469C
:10D91000002B1D460DDD289BC9F8006001332C4407
:10D92000072B2994C9F80450289300F3878309F141
:10D930000809139B002DA8BF5B1B002B1D4640F35D
:10D94000BE80B94A289B0F92102D40F36D8222466B
:10D950001027DDF828B0089C05E009F10809103D02
:10D96000102D40F3608201331032072B2992289347
:10D97000C9F800A0C9F80470EFDD27AA214658466F
:10D9800004F06AFE00287FF4A3AA299A289B0DF1CF
:10D99000D009E4E727AA08990A9804F05DFE002858
:10D9A0007FF496AA9DF87F70299C0DF1D009FFF7AE
:10D9B000CDBB0E9A146813460433E5170E93224626
:10D9C0002B46F4E45E1E002E7FF73FAF964B0F937D
:10D9D000102E40F31081CDF834801027B046DDF8CA
:10D9E00028B0089E07E009F10809A8F11008B8F16D
:10D9F000100F40F3FD8001351034072D2994289530
:10DA0000C9F800A0C9F80470EDDD27AA31465846D0
:10DA100004F022FE00287FF45BAA299C289D0DF1CA
:10DA2000D009E2E7079911F0100220D00E988DF886
:10DA30007F30BBF1000F046800F104074FF00005D0
:10DA400026DB0A4622F08002079254EA05020E976E
:10DA50001F467FF403ABBDE401330F9A28932C4497
:10DA6000072B299489E824007FF7DEABFAE60799B3
:10DA700011F0400340F04A820E998DF87F30BBF1DF
:10DA8000000F0C6801F104074FF0000580F21A81C5
:10DA90000E971F4654EA05037FF4E0AA44AE3034E3
:10DAA00006F8414DFFF7F4BA27AA08990A9804F03E
:10DAB000D3FD00287FF40CAA299C0DF1D009139AFC
:10DAC000219B32441746129A934247DB079AD207AA
:10DAD00044D412990E44F51BCB1A9D42A8BF1D4693
:10DAE000002D2E460DDD289AC9F8007001322C4415
:10DAF000072A2994C9F80450289200F32E8309F1CB
:10DB00000809002EACBF9D1B1D46002D7FF78EAB74
:10DB1000454A289B0F92102D9EDD10260A9FDDF8A6
:10DB200020B004E009F10809103D102D94DD013307
:10DB30001034072B29942893C9F800A0C9F8046071
:10DB4000F0DD27AA5946384604F086FD00287FF408
:10DB5000BFA9299C289B0DF1D009E5E7289A1698C2
:10DB60001799C9F8001001320444072A2994C9F80A
:10DB70000400289200F3CF8209F10809A9E7079B66
:10DB8000DF073FF52CAE013501340123072D299421
:10DB90002895C9F80060C9F804307FF754AE27AA69
:10DBA00008990A9804F058FD00287FF491A9299C4F
:10DBB000289D0DF1D00948E627AA08990A9804F093
:10DBC0004BFD00287FF484A9299C289D0DF1D009E4
:10DBD00013E627AA08990A9804F03EFD00287FF46E
:10DBE00077A9299C289D0DF1D00915E6002455E759
:10DBF0004646DDF834800F9B01353444072D2994C7
:10DC0000289589E848007FF71EAEC8E727AA08993B
:10DC10000A9804F021FD00287FF45AA9299C0DF1EF
:10DC2000D009FFF7B7BA00BFEC4D010864424FF0CE
:10DC30002D0765EB4505BBF1000F8DF87F70FFF6F2
:10DC40000DAA079B23F080030793FFF707BA0799F4
:10DC500011F0400317D00E988DF87F200346BBF1DA
:10DC6000000F03F1040304884FF00005C0F21B838A
:10DC700021F08001079154EA05010E933FF4E1ACD5
:10DC80001746FFF75CB90E998DF87F30BBF1000F96
:10DC90000C6801F104074FF0000502DB079AFFF75B
:10DCA000AFB90E970027FFF74AB9079B0E9A13F0FA
:10DCB000400F134600F04281043314880E93002570
:10DCC000FFF71ABB079ABDE6DDE9140102460B46D1
:10DCD00005F09AFD002840F0E882119BBBF1FF3F60
:10DCE00023F0200700F05F82472F00F05881159B3A
:10DCF000079A002B42F480720F92C0F25C829DED75
:10DD0000147B8DED1C7B00230993119B662B00F087
:10DD10003382462B00F02581452F0CBF0BF1010506
:10DD20005D4625A822A921AA02230490029200930D
:10DD30000195DDE91C2303910A9800F059FD119B20
:10DD4000672B064640F07582079BDA0740F1948204
:10DD5000741900220023DDE91C0105F023FD0028D1
:10DD600040F07881259B9C4206D930215A1C25928F
:10DD70001970259B9C42F9D89B1B472F129300F0EA
:10DD80005681119B652B40F36382119B662B219B6F
:10DD9000139300F02682139A12998A42C0F21482D9
:10DDA000079BDB0700F16A8222EAE2730D92672289
:10DDB0001192099A002A40F0178109930F9B07934B
:10DDC00093469DF87F70FFF76DB927F0070797ED31
:10DDD000007B07F108038DED147B0E93FFF777BBF3
:10DDE000079BDE060BD4079B5D0608D50E9A1368C9
:10DDF00004320E92BDF82C201A80FEF77ABF0E9ADC
:10DE0000136804320E920B9A1A60FEF772BF002755
:10DE1000BB458DF87F70FFF626AC079B23F080038F
:10DE20000793FFF7F3BB144601330F9A28932C4452
:10DE3000072B299489E824003FF736AE09F1080939
:10DE40003DE627AA08990A9804F006FC00287FF40A
:10DE50003FA8299C0DF1D00927E4289BB44AC9F8B2
:10DE60000020013301340122072B29942893C9F89B
:10DE7000042069DC09F108092DB9129B1BB9079B25
:10DE8000D9077FF5D3A9289B1699179AC9F80020BE
:10DE900001330C44072B2994C9F80410289300F38C
:10DEA000D98109F108096D42002D40F3B380A14AE0
:10DEB0000F92102D40F3228122461027DDF828B062
:10DEC000089C05E009F10809103D102D40F315816B
:10DED00001331032072B29922893C9F800A0C9F802
:10DEE0000470EFDD27AA2146584604F0B5FB002850
:10DEF0007EF4EEAF299A289B0DF1D009E4E70E9F3E
:10DF0000FFF7AABB4FF0FF30FEF7E8BF0E988DF881
:10DF10007F200346BBF1000F03F1040304884FF098
:10DF20000005C0F2B48121F08001079154EA050197
:10DF30000E9317467FF492A8FFF74CBA0433146887
:10DF40000E930025FFF7D8B927AA08990A9804F07C
:10DF500083FB00287EF4BCAF219D299C0DF1D009E4
:10DF60008AE725A822A921AA0323049002920093FC
:10DF7000CDF804B00391DDE91C230A9800F038FCC9
:10DF80005D460646119B462B06EB05047FF4E1AE89
:10DF90003378302B00F09881219D2C44D9E6BBF1D9
:10DFA000000F08BF4FF0010BA1E6079B43F02003D1
:10DFB000079308F1010898F80030FEF7CDBE27AAB4
:10DFC00008990A9804F048FB00287EF481AF299C48
:10DFD0000DF1D009FFF781BB3046FBF771FFA34677
:10DFE00003460D90FFF701BB2D2709930F9B079365
:10DFF0008DF87F704FF0000BFFF755B827AA0899EE
:10E000000A9804F029FB00287EF462AF299C289B23
:10E010000DF1D0091299C9F8006001330C44072BA7
:10E0200029942893C9F804107FF7FEA81AE4219BCD
:10E03000D81C11DB9B450FDB1393ACE627AA08998C
:10E040000A9804F009FB00287EF442AF299C0DF1E8
:10E05000D0096EE423468FE6119A023A1192013BF1
:10E06000002B9DF844202193B8BF5B428DF88C2093
:10E07000B4BF2D222B22092B8DF88D2040F30B816C
:10E080000DF19B0004462C4A82FB0321DA17C2EBF8
:10E09000A10202EB8201A3EB410303F13001092A43
:10E0A000134604F8011DEEDC21463033DAB201F8E4
:10E0B000012D884240F26F810DF18E01234601E06F
:10E0C00013F8012B01F8012B9842F9D1431C1B1BBB
:10E0D0000DF18E02134423AA9B1A129A1993012A56
:10E0E00013440D9340F3FE800D9B169A13440022B7
:10E0F0000D93139223EAE3735BE6144601330F9A00
:10E1000028932C44072B299489E824003FF776AF05
:10E1100009F108097EE727AA08990A9804F09CFAF1
:10E1200000287EF4D5AE219B299C0DF1D009D0E4C6
:10E13000584D0108EC4D010867666666062D2B46B2
:10E1400028BF06230D9323EAE373B3460E97139675
:10E1500037460993914EFEF7A5BF27AA08990A985A
:10E1600004F07AFA00287EF4B3AE219B129A299C1F
:10E17000D31A0DF1D009C4E425A822A921AA0323AA
:10E18000049002920093CDF804B00391DDE91C23C2
:10E190000A9800F02DFB5D46064600EB0B04F7E6FF
:10E1A0000793FFF7C7B84FF0060BA0E52D278DF8B2
:10E1B0007F70FFF7B3B9DDE9141202F100431D933C
:10E1C0002D231C910993A0E5169A129B1344139AD0
:10E1D0000D93002A40F39080672223EAE3731192A3
:10E1E000E7E5002B40F39080BBF1000F63D1079A65
:10E1F000D10760D41A460D9223EAE373D9E5079B51
:10E20000DB075F4605D544AE302306F8413DFEF7F7
:10E210003FBFCDF834B034AEFEF73DBF25EAE5731D
:10E220000E9709930D95834613909DF87F70FEF726
:10E2300039BF119B472B7FF48BAD079BDC073FF564
:10E24000A1AE259B472FA3EB060312933FF4EFAE3D
:10E25000219B04E727AA08990A9804F0FDF90028F1
:10E260007EF436AE219D299C289B0DF1D0091AE63B
:10E27000A0460025FEF772BD259B7DE5169A139BEF
:10E28000134467220D93119223EAE37391E50E93F1
:10E290001746FFF7FFBB303330228DF88F308DF8F3
:10E2A0008E2024AB17E70E93FCE43D4E3D4B9DF8CA
:10E2B0007F70FFF735B9139B169A9D1805EB0B037A
:10E2C0000D9323EAE37374E500220023DDE91C01CA
:10E2D00005F068FA00287FF45FAEC5F101052195CD
:10E2E0002C4436E5079B13F001037FF4FDAE139336
:10E2F0000D9B23EAE3735CE5139B0D9AC3F10103C5
:10E300001A4413460D9267E7BBF1000F02D1079B39
:10E31000DA0707D5169B5D1C05EB0B030D9323EA6B
:10E32000E37346E501230D9343E50E9898F8013019
:10E3300005680430002D0E90A046BEF60DAD4FF0DE
:10E34000FF35FEF709BD8DF87F10FFF793B88DF804
:10E350007F10FFF75DB88DF87F10FEF7BFBF8DF817
:10E360007F10FEF75CBE8DF87F10FFF712B88DF8B6
:10E370007F10FEF7CABD8DF87F10FFF751B98DF8F9
:10E380007F10FEF723BE8DF87F10FFF7EDB88DF8F4
:10E390007F10FFF78CB80DF18E039CE6504D0108FD
:10E3A000244D0108204D010810B4044C13460A46C0
:10E3B000014620685DF8044BFEF75ABCE8050020D2
:10E3C000F0B50C46ADF26C4D8989666EE5891996FB
:10E3D00021F00201666AADF80E500025E769ADF83C
:10E3E0000C10099606951AAE4FF4806569460096A2
:10E3F00004960295059507970646FEF739FC051E1B
:10E4000007DB30466946F8F749FF002818BF4FF090
:10E41000FF35BDF80C305B0603D5A38943F04003FC
:10E42000A38128460DF26C4DF0BD00BF70B5002AE7
:10E430009AB005462FDB14461A464FF4027300913A
:10E440000491ADF80C3011D0013C4FF6FF761E9BC5
:10E45000029469460594ADF80E60FBF7E9FE421C94
:10E4600012DB009B00221A701AB070BD1E9B029432
:10E470004FF6FF7669460594ADF80E60FBF7D8FEBF
:10E48000431C04DB1AB070BD8B232B60E9E78B23A0
:10E490002B601AB070BD8B2303604FF0FF30F1E7A3
:10E4A00010B582B0054C0093246813460A46014615
:10E4B0002046FFF7BBFF02B010BD00BFE8050020FB
:10E4C000F8B50D461446064610B1836B002B4AD0B2
:10E4D000B4F90C20A369A36091B2080738D5236969
:10E4E000002B35D08904EFB215D522686169D31AA3
:10E4F0008B421CDA0133A168501C0139A1602060F5
:10E50000157062699A421AD0A389DB0701D50A2FD8
:10E5100015D03846F8BD616E42F4005221F4005126
:10E52000A281226861666169D31A8B42E2DB2146CF
:10E530003046F8F7B3FE40B922680123DBE72146F5
:10E540003046F8F7ABFE0028E3D04FF0FF37E0E7A6
:10E550002146304600F020F80028F6D1B4F90C200E
:10E56000236991B2BEE7F8F79BFFB1E770B50D469E
:10E57000084C114606461A46284600232360F5F744
:10E5800041FB431C00D070BD2368002BFBD03360DF
:10E5900070BD00BFE01A002038B5304B1B6805463F
:10E5A0000C4613B19A6B002A38D0B4F90C2093B200
:10E5B00018070CD52069A8B113F001021ED06369B9
:10E5C00000225B42A361A260F0B1002038BDD906F1
:10E5D0003CD5580726D4206942F00803A3819BB29A
:10E5E0000028E9D103F42072B2F5007FE4D0284678
:10E5F0002146F9F7CBFDA3892069DDE7990758BFCC
:10E600006269A2600028E0D1B4F90C301A06DDD5A9
:10E6100043F04003A3814FF0FF3038BD1846F8F7B0
:10E620003FFFC2E7216B51B104F14003994204D08E
:10E630002846F8F7EFFFB4F90C20002323630023EA
:10E640002069636022F024022060C5E742F04002A6
:10E6500009232B604FF0FF30A28138BDE805002070
:10E6600038B5074C0023054608462360F5F7AAFA9B
:10E67000431C00D038BD2368002BFBD02B6038BD75
:10E68000E01A0020002910B491FBF2F402FB1413ED
:10E6900006DB002B0EDB046043605DF8044B704723
:10E6A000002BC4BF04F1FF349B18046043605DF885
:10E6B000044B704701349B1A046043605DF8044BBF
:10E6C000704700BF02690B69934200F38D802DE90A
:10E6D000F04F03F1FF3801F1140700F1140B57F864
:10E6E00028205BF828304FEA880483B00132B3FB5E
:10E6F000F2F90BEB0403009407EB040A0193B9F160
:10E70000000F39D00025BC46DE462B465CF8046B72
:10E71000DEF80020B4B209FB0455360C2C0C09FBC2
:10E720000644ADB25B1BA6B213FA82F3C6EB1246E7
:10E7300006EB23469BB243EA0643E2454EF8043B10
:10E740004FEA14454FEA2643E0D2009B5BF80330C2
:10E7500093B9019C231F9B450CD254F8043C4BB940
:10E76000A4F1080302E01A68043B1AB99B4508F1BA
:10E77000FF38F8D3C0F81080044601F0BFFB002832
:10E780002EDB09F101095D46002357F8041B2868B8
:10E790008AB29A1A090C12FA80F2C1EB104303EB09
:10E7A000224391B241EA0341BA4545F8041B4FEABE
:10E7B0002343EAD25BF828200BEB880382B91A1FA7
:10E7C00093450BD253F8042C42B9083B02E01A6877
:10E7D000043B1AB99B4508F1FF38F8D3C4F8108000
:10E7E000484603B0BDE8F08F0020704700000000ED
:10E7F0002DE9F04F016C99B08146259C92469B46CD
:10E8000049B1426C4A60012393408B6001F048F9A2
:10E810000023C9F84030BBF1000FD84633DB00239A
:10E820002360A34B1A4608EA0303934214D0002244
:10E8300000235046594604F0B5FF054648B3249AD4
:10E8400001231360269B002B00F0C28099481860BA
:10E85000013819B0BDE8F08F249A42F20F731360AB
:10E86000BAF1000F00F09F809348269B002BF0D058
:10E87000C378002B00F0AE8000F10803269A1360E5
:10E8800019B0BDE8F08F01232BF000482360C34688
:10E89000C7E716AA17AB0192009352465B4648465B
:10E8A00001F064FC5FEA1854089040F08580169DE2
:10E8B000179C2C4404F23243202B40F38982C3F18D
:10E8C000400304F2124008FA03F82AFA00F040EA82
:10E8D000080004F089FC0123013CA1F1F8710D93BB
:10E8E0000022764B04F042FB6BA3D3E9002304F033
:10E8F000F1FC6BA3D3E9002304F03AFB0646204663
:10E900000F4604F081FC68A3D3E9002304F0E2FC85
:10E9100002460B463046394604F02AFB06460F46AF
:10E9200004F088FF0022049000233046394604F0AA
:10E9300043FF002840F02782049E162E00F220821A
:10E940005F4B03EBC603D3E9000152465B4604F07C
:10E9500051FF002800F04182731E049300230B93A3
:10E960002C1BB4F1010800F1298200230593049BBC
:10E97000002BC0F21A8298440A9300230293229B30
:10E98000092B29D8052B40F34386043B229300250D
:10E99000229B023B032B00F22286DFE813F02A03BE
:10E9A000230235034F04444B464AC8F313000028A2
:10E9B00014BF1846104658E7CBF3130343F07F51BA
:10E9C0000D955046A4F2FF3441F44011169D87E79F
:10E9D0003D483EE7C31C51E70021C9F844104846B2
:10E9E000229101F037F84FF0FF330693229A0C93EF
:10E9F000012307902392C9F840000993179B002B2D
:10EA0000C0F2D080049A0E2A00F3CC802C4B03EB8A
:10EA1000C20393ED007B239B002B8DED027BC0F2A4
:10EA2000FE8256465F46DDE902AB304652465B4603
:10EA3000394604F079FD04F0FDFE044604F0E4FBE1
:10EA400052465B4604F046FC0B46024639463046C9
:10EA500004F08CFA079D04F130032B70069B012B08
:10EA600006460F4605F1010561D00022174B04F060
:10EA700031FC0022002306460F4604F093FE0028D6
:10EA80007DD1CDF81490DDF818A0DDF81CB0DDE9DB
:10EA9000028928E0AFF3008061436F63A787D23F0C
:10EAA000B3C8608B288AC63FFB799F501344D33F7D
:10EAB0000000F07F594D0108184E01080000F83F92
:10EAC000304E01080C4E0108584D0108000024404A
:10EAD00004F000FC0022002306460F4604F062FE0C
:10EAE000002840F0AE8342464B463046394604F09B
:10EAF0001BFD04F09FFE044604F086FB42464B4695
:10EB000004F0E8FB02460B463046394604F02EFA84
:10EB100004F1300E05F801EBCBEB050ED6450646A9
:10EB20000F464FF00002AE4BD2D1DDF814903246C2
:10EB30003B463046394604F01BFA06460F4602466D
:10EB40000B46DDE9020104F037FE40B932463B4690
:10EB5000DDE9020104F026FE88B1E3070FD515F8C0
:10EB6000014C079A6B1E04E09A4200F0FC8313F8F4
:10EB7000014D392C03F10105F6D001341C700899C0
:10EB8000484600F08DFF0022049B2A70249A01332E
:10EB90001360269B002B00F09B8307981D6019B023
:10EBA000BDE8F08F099A002A00F00E81229A012A0E
:10EBB00040F35782069B029A5F1EBA42C0F28B83D3
:10EBC000D71B069B002BC0F28084059D069B059AEF
:10EBD00001211A4448460592984401F045F806463A
:10EBE00065B1B8F1000F09DD4545059A2B46A8BF70
:10EBF0004346D21A0592ED1AC3EB0808029B002B7C
:10EC000040F3F582099A002A00F00282002F00F0FA
:10EC1000FF8131463A46484601F0C8F8089A014655
:10EC20000646484601F02AF808990446484600F08E
:10EC300037FF029BDB1B029340F0E981012148462C
:10EC400001F012F80A9B0290002B00F01582014699
:10EC50001A46484601F0AAF8229B0290012B40F385
:10EC6000F3820027029A136902EB8303186900F00C
:10EC7000ADFFC0F12000404410F01F0000F0FA8109
:10EC8000C0F12003042B40F3BD84C0F11C00059BA0
:10EC90000344059305448044059B002B05DD214674
:10ECA0001A46484601F0D2F80446B8F1000F05DDD7
:10ECB00042460299484601F0C9F802900B9B002B8E
:10ECC00040F07A82069B002B40F39382099B002B35
:10ECD00040F0F481DDF81CB0069FDDF808805D4649
:10ECE00002E000F0E7FE044641462046FFF7EAFC5A
:10ECF00000F1300A05F801ABCBEB0503BB424FF046
:10ED00000A024FF0000321464846EADB079B069AB9
:10ED1000012AACBF9B1801331D464FF0000B214662
:10ED20000122484601F092F80299089001F0E6F8B5
:10ED3000002840F3058315F8012C07996B1E04E0A9
:10ED40008B4200F0748213F8012D392A03F101057A
:10ED5000F6D001321A700299484600F0A1FE002E4A
:10ED60003FF40DAFBBF1000F05D0B34503D05946BA
:10ED7000484600F095FE3146484600F091FEFEE61A
:10ED800001230B93ECE5DDF81080404604F03CFADB
:10ED900002460B463046394604F004FD00287FF455
:10EDA000CBAD08F1FF330493C6E5059A049BD21A54
:10EDB0005B420293002305920A93E0E5C8F1000349
:10EDC00005934FF00008D2E5029F059D099E07E7D5
:10EDD000C3F120080AFA08F07BE50B90C0E500BFFC
:10EDE0000000244000230993049B239A13440C93AE
:10EDF0000133002B069340F37D82069C26460021BA
:10EE0000172EC9F844100BD9012204235B0003F12B
:10EE10001400B042114602F10102F7D9C9F84410BA
:10EE2000484600F017FE0E2C0790C9F840003FF648
:10EE3000E5AD002D3FF4E2AD04990029CDE90EAB1C
:10EE400040F39A82904B01F00F020E1103EBC203C4
:10EE5000F006D3E9004540F146828C4B50465946B6
:10EE6000D3E9082304F060FBCDE9100106F00F069A
:10EE70004FF0030A86B1854FF10709D52046294690
:10EE8000D7E9002304F026FA0AF1010A04460D46E8
:10EE9000761007F10807EFD122462B46DDE9100175
:10EEA00004F042FB06460F460B9B43B10022784B11
:10EEB0003046394604F080FC002840F01A83504662
:10EEC00004F0A2F932463B4604F004FA714B0022EA
:10EED00004F04EF8069B0446A1F15075002B00F09B
:10EEE000DB81049B1493069B1093099B002B00F07D
:10EEF0009482109A644B684903EBC20353E90223DE
:10EF0000002004F011FB22462B4604F02FF8824625
:10EF10008B463046394604F08DFC044604F074F903
:10EF200002460B463046394604F020F83034079D3F
:10EF3000E4B206460F462C7002460B465046594630
:10EF4000013504F057FC002850D132463B460020E2
:10EF50004F4904F00BF802460B465046594604F060
:10EF600049FC002840F00883109A012A40F3F781F9
:10EF7000109B079ACDF84080134498460DE000207E
:10EF8000434903F0F3FF52465B4604F015FC0028AA
:10EF900040F0F282454500F0E0815046594600229B
:10EFA0003E4B04F097F900223C4B82468B4630469C
:10EFB000394604F08FF90F46064604F03BFC044640
:10EFC00004F022F902460B463046394603F0CEFFE4
:10EFD0003034E4B252465B4605F8014B06460F4614
:10EFE00004F0EAFB32463B460028C8D0149B049349
:10EFF000C5E500230993239B002B40F380811E4627
:10F000001C460C930693FAE601230993F3E7089450
:10F01000029A0899484600F0C9FE04460EE6069B8F
:10F02000002B3FF7FEAC40F04F81DDE902010022EA
:10F030001B4B04F04FF95B46524604F0D1FB069B94
:10F0400002931E46002800F0EA80239B079DDB43C5
:10F0500004930299484600F023FD002E3FF48FAD43
:10F0600089E60D9A002A00F0388203F23343029FAA
:10F07000059DACE51C200AE6229B012B40F3808213
:10F080000A9F0120F7E500BF304E0108F84E010845
:10F090000000F03F00001C400000E03F0000244062
:10F0A00000001440314600230A22484600F002FDC9
:10F0B0000C9B002B064640F38D820693002D05DD48
:10F0C00031462A46484600F0C1FE0646002F40F071
:10F0D0007C81B046069B079A013BD31808930AF03F
:10F0E000010309931746DDF808B020465946FFF79B
:10F0F000E9FA31460546204600F000FF42465946EF
:10F100008246484600F01CFFC268834605F1300382
:10F11000002A49D101462046069300F0EFFE5946E9
:10F120000590484600F0BCFC059A069B2AB9229936
:10F1300019B90999002900F03582BAF1000FC0F21F
:10F14000E38005D1229919B90999002900F0DC80E2
:10F15000002A00F34E81089A3B7007F1010A97429A
:10F16000554600F05281214600230A22484600F00D
:10F17000A1FC4645044631464FF000034FF00A0219
:10F1800048460BD000F096FC4146064600230A2272
:10F19000484600F08FFC57468046A4E700F08AFC02
:10F1A0005746064680469EE701464846059300F0CE
:10F1B00077FC0122059BC0E70299204600F09EFEE5
:10F1C0000028BFF67FAD2146049C0023013C0A22A3
:10F1D0004846049400F06EFC099B0446002B7FF423
:10F1E00061AF0C9B002B40F3ED81069372E5089C08
:10F1F00024E5229B022B7FF769AD069B002B40F094
:10F200009D8102990522484600F054FC0146029077
:10F21000204600F073FE002808947FF716AF049A8A
:10F2200007993123013204920B704D1C11E7049AA7
:10F2300001320492079A312313708CE5012309935C
:10F24000D2E5DDF814909AE4BAF1000F7FF409AD2D
:10F25000CBF31303002B40F03E812BF000473F0D12
:10F260003F052FB1059B0133059308F101080127E4
:10F270000A9B0120002B3FF4FEACF3E4504603F060
:10F28000C3FF32463B4604F025F80022BF4B03F093
:10F290006FFE0446A1F15075304639460022BC4B42
:10F2A00003F064FE22462B4606460F4604F0A2FAFF
:10F2B000002840F0AE80224605F100433046394632
:10F2C00004F07AFA00284AD0002302931E46BCE6D6
:10F2D0000798FFF7BEBA029B0A9A0297FB1A1A44D4
:10F2E0000A9200276DE49DED0E7B4FF0020A8DED32
:10F2F000107BBFE51C460021C9F8441090E50124AD
:10F3000023940C940694F6E7002A9A4611DD2146D0
:10F310000122484600F09AFD0299044600F0EEFDF5
:10F32000002840F34881BAF1390F00F0098105F156
:10F33000310AB34687F800A07D1C464608940AE5CA
:10F3400004D11AF0010F01D0F5E4154615F8013C7F
:10F35000302B05F1FF32F8D0FDE4DDF84080DDE927
:10F360000EABFFF74BBB079930220A70049A15F8D1
:10F37000014C0132049200E4049B5C42002C00F03A
:10F38000B380844B04F00F0203EBC203D3E90023E4
:10F39000DDE90E0103F09EFF241106460F4600F042
:10F3A00016817D4D4FF0020AE20709D530463946F5
:10F3B000D5E9002303F08EFF0AF1010A06460F4645
:10F3C000641005F10805EFD16EE57168484600F05C
:10F3D00041FB33699A1C0546920006F10C010C3082
:10F3E000F9F768FA29460122484600F02FFD8046C9
:10F3F00070E6392B00F0A48003F1010AB34687F8C8
:10F4000000A07D1C46460894A5E4B3469A464646AD
:10F4100085E4002302931E4601E7109B5D495A1EB6
:10F4200001EBC2012B461592D1E90001224603F0FF
:10F4300051FFCDE912013946304604F0FBF904468C
:10F4400003F0E2FE0B4602463946304603F08EFDDD
:10F45000109B0F4607993034012B06460C7001F1C2
:10F46000010520D0109B079A13449A46AB46002210
:10F470004A4B3046394603F02DFF0F46064604F04E
:10F48000D9F9044603F0C0FE303402460B4630463C
:10F49000394603F06BFD0BF8014BDA4506460F4683
:10F4A000E5D1159B1D4400223D4BDDE9120103F01F
:10F4B0005FFD32463B4604F07FF9002848D0149B9C
:10F4C000049315F8014CFFF74CBB059B069A9D1A57
:10F4D0000023FFF77CBB0027CAE6169B029F059D11
:10F4E000C3F13603FFF773BBDDE90E674FF0020A85
:10F4F000DAE4069B002B3FF4C1AE0C9B002B7FF798
:10F500002EAF0022254B3046394603F0E3FE064677
:10F510000F460AF1010003F077FE32463B4603F046
:10F52000D9FE0022194B03F023FD049A0C9B109383
:10F53000013A0446A1F150751492D6E4089484E58A
:10F540003922B346089446463A707D1CFFF7F5BB56
:10F55000DDE912230020124903F008FD32463B4644
:10F5600004F048F908B9FAE6154615F8013C302BC5
:10F5700005F1FF32F8D039E5149B0493FFF7F1BA97
:10F58000BAF1000F7FF47CAD62E600BF00001C40C2
:10F5900000001440304E0108F84E010800002440DD
:10F5A0000000E03F392BD3469A46C9D0BBF1000F8B
:10F5B0003FF7BDAEBDE67FF4BCAE1AF0010F3FF4DD
:10F5C000B8AEB0E6229B022B25DC0C9B0DE64FF07B
:10F5D000020A69E4229B022B1DDC0C9B6DE50024D2
:10F5E000C9F844402146484600F034FA4FF0FF3352
:10F5F00006930C93012307902394C9F840000993C4
:10F60000FFF7FCB93FF448ABC0F13C00FFF73FBB4C
:10F610000125FFF7BDB90C9B0693EEE50B78722B25
:10F6200030B431D0772B2AD0612B04D0162303605D
:10F6300030BC002070474FF4027501244FF48470F1
:10F6400011F8013F8BB1622B16D0782B11D02B2BE8
:10F65000F6D111F8013F20F01C0024F0030440F023
:10F66000100044F00204002BEDD12C43146030BC98
:10F67000704744F40064E3E744F48034E0E74FF477
:10F68000C06501240820DBE700252C460420D7E7CD
:10F690002DE9F0471C4F0E4691468046F4F7C2FB19
:10F6A0003D68F5B134785CB13D2C18BF344602D1C9
:10F6B00017E03D2B15D014F8013F002BF9D1A41B06
:10F6C000286870B122463146FAF768FC28B92868E4
:10F6D000035D3D2B00EB040A09D055F8040F002808
:10F6E000F0D14046F4F7A2FB0020BDE8F0873B686C
:10F6F000ED1AAD104046C9F80050F4F797FB0AF137
:10F700000100BDE8F08700BFB00B002000B583B05A
:10F7100001AAFFF7BDFF03B05DF804FB0048704786
:10F72000040A00200268634B63482DE9F04383FB21
:10F7300002431344D417C4EB234400FB14200028D5
:10F74000C0F2AE8004F52F2404F66C245B4E5C4DB1
:10F750005C4ADFF884E1DFF884C15B4F86FB043646
:10F76000E317C3EBE63605FB0645AB08A2FB0382B5
:10F7700005EBD222AEFB0383A2EBD3122B09ACFB29
:10F7800003C3A2EB1313DFF858C1504AACFB038C40
:10F79000A2FB038205EBDC3C9D1A9B0802EB55059E
:10F7A000AEFB03232D0A4A4AACEBD31340F26D1E85
:10F7B0000EFB1533DFF82CC182FB002E03EB830216
:10F7C00002328644ACFB02C24FEAE07CCCEBEE2C6A
:10F7D0004FF4616E0EFB1C000334DFF80CE1C1F83E
:10F7E00008C084FB078904EB090C8EFB007EE71739
:10F7F000C7EBAC07C7EBC707D209092AA4EB07047C
:10F800004FEAE078864402EBC20C8CBF6FF0090728
:10F810000227C8EB6E1E0CEB0C1CDFF8D0808C614D
:10F820004FF4C87404FB06563A440CF1020CCEEBBC
:10F830000E17A8FB0C4CA0EB87005C1C012A98BF9C
:10F840000136B3F5997FA4EB9C0481E8014024D2F2
:10F85000A80717D01F48A0FB0570C0094FF4C87750
:10F8600007FB1055B5FA85F56D093B332B44A6F21D
:10F870006C76002008624E61CB610A61CC6008465C
:10F88000BDE8F0831348A0FB05704009642707FB1F
:10F8900010500028DED00125E7E7A3F59973E6E7CD
:10F8A00000F5A83004F52F2400F5C07004F66B2491
:10F8B0004CE700BF07452EC280510100BD066B39E1
:10F8C0004FC5FDFF7F206B399324499261F319677F
:10F8D000C5B3A2911F85EB51D97CC65941D67200A0
:10F8E0001F2BD3E5D7802BD689888888CDCCCCCC6C
:10F8F00038B5074C0023054608462360F4F7E8F9BD
:10F90000431C00D038BD2368002BFBD02B6038BDD2
:10F91000E01A0020FF2801D90020704710B50446E6
:10F9200000F024F82044407800F00800C0B210BD78
:10F93000034A044B1268506B002808BF18467047F2
:10F94000E8050020440A0020044B054A1B685B6B55
:10F95000002B08BF134693F828017047E8050020E4
:10F96000440A0020D0F8EC00704700BF08B5034BF4
:10F970001868FFF7DDFFD0F8EC0008BDE8050020AF
:10F98000F0307047044A054B1268506B002808BFDE
:10F990001846F030704700BFE8050020440A0020F8
:10F9A00070B50D46084C114606461A4628460023F7
:10F9B0002360F4F7ADF9431C00D070BD2368002B21
:10F9C000FBD0336070BD00BFE01A0020F0B583B0FB
:10F9D0000746089D92B1114C114E2468646B009546
:10F9E000002C08BF3446D4F8E440A047431C03D1A0
:10F9F00000228A232A603B6003B0F0BD074B084910
:10FA00001B685B6B0095002B08BF0B461446214614
:10FA1000044AD3F8E4400123A047E7E7E8050020C3
:10FA2000440A0020384D010882B049B15AB16BB187
:10FA300013780B601278101C18BF012002B07047B9
:10FA400001A9002AF3D1104602B070476FF00100FF
:10FA5000F4E700BFC36C70B505460C464BB153F8D4
:10FA6000240080B1026843F8242000230361C360AE
:10FA700070BD2122042102F007FEE864034600283D
:10FA8000EDD1002070BD012101FA04F6721D284657
:10FA9000920002F0F9FD0028F3D044608660E4E7AC
:10FAA00031B1C36C4A6853F82200086043F8221051
:10FAB000704700BFF0B50C6983B00D46064601F1F2
:10FAC000140E0027DEF8000081B202FB01310B0C9E
:10FAD000000C02FB003389B2013701EB0341BC4249
:10FAE0004EF8041B4FEA1343ECDC3BB1AA68944286
:10FAF00007DA05EB8402013453612C61284603B018
:10FB0000F0BD6968019301313046FFF7A3FF2A6910
:10FB1000023205F10C01074692000C30F8F7CAFEDC
:10FB2000F26C6968019B52F82100286042F821506C
:10FB30003D46DEE72DE9F843234C089D1F46083378
:10FB400084FB034EDB17C3EB6E0EBEF1010F0646BE
:10FB50000C46904635DD012300215B009E4501F1F6
:10FB60000101FADC3046FFF775FF0123B8F1090FF8
:10FB70004561036121DD04F109094D46444415F84E
:10FB8000013B0146303B0A223046FFF793FFA54276
:10FB9000F5D109EB0804083C47450CDDC8EB070725
:10FBA000274414F8013B0146303B0A223046FFF758
:10FBB00081FFA742F5D1BDE8F8830A344FF0090868
:10FBC000EAE70021CEE700BF398EE338030C1B04BF
:10FBD000B3B90004102310F07F4F04BF00020833B4
:10FBE00010F0704F04BF0001043310F0404F04BF09
:10FBF00080000233002807DB420003D42020704736
:10FC00000023E8E7581C704718467047036813F054
:10FC1000070207D0D90720D49A0720D49B08036095
:10FC20000220704799B209B91B0C102213F0FF0F84
:10FC300004BF1B0A0832190704BF1B0904329907C5
:10FC400004BF9B080232D90704D45B0801D12020ED
:10FC500070470132036010467047002070475B0810
:10FC600003600120704700BF10B50C460121FFF76B
:10FC7000F1FE01224461026110BD00BF2DE9F04F89
:10FC80000D691769BD4283B00C46164604DA2A4650
:10FC900034463D460E461746A368616805EB0708E3
:10FCA0009845C8BF0131FFF7D5FE00F1140C0CEBED
:10FCB0008809CC45009005D26346002143F8041B17
:10FCC0009945FBD806F1140202EB870A04F11403EC
:10FCD000524503EB850E54D2CDF80490994652F864
:10FCE000043B1FFA83FBBBF1000F20D000204F46DE
:10FCF0006646054600E01E4657F8044B3068A1B240
:10FD000083B20BFB0131240C000C4B190BFB0400DC
:10FD100000EB134099B2334641EA0041BE454FEA39
:10FD2000104543F8041BE6D8756052F8043C5FEABE
:10FD3000134B20D0DCF80030674618464D460021B2
:10FD400000E037462C88000C0BFB040001449CB2F9
:10FD50003E4644EA014346F8043B786855F8044BB4
:10FD600083B2240C0BFB043404EB1143AE454FEA81
:10FD70001341E6D87B6092450CF1040CAFD8DDF856
:10FD80000490B8F1000F0BDD59F8043CA9F1040907
:10FD90001BB105E059F8043D13B9B8F10108F9D1D8
:10FDA0000098C0F8108003B0BDE8F08F12F0030394
:10FDB0002DE9F041144607462ED10E46A4101CD062
:10FDC000BD6C95B3E3074FF0000806D4641014D05F
:10FDD0002868A8B10546E307F8D52A4631463846D3
:10FDE000FFF74CFFB6B17268FB6C641053F8221039
:10FDF000316043F822600646EAD13046BDE8F08122
:10FE00002A4629463846FFF739FF2860C0F80080A7
:10FE10000546E0E70646D9E75A1E0B4D002355F884
:10FE20002220FFF747FE0646C8E701213846FFF7C4
:10FE300011FE40F271210122002341610261054659
:10FE4000B8640360BEE700BF204F01082DE9F0470A
:10FE500091460A698B684FEA691404EB020808F1BD
:10FE600001059D420E468246496804DD5B009D42C5
:10FE700001F10101FADC5046FFF7ECFD002C00F126
:10FE8000140238DD02EB8403002142F8041B934284
:10FE9000FBD1346906F1140119F01F0901EB840E3E
:10FEA00021D0C9F1200200240F6807FA09FC4CEAAE
:10FEB00004049C4643F8044B51F8044B8E4524FA45
:10FEC00002F4F1D8CCF804400CB108F10205DAF8DC
:10FED0004C307268013D53F822100561316043F8DF
:10FEE0002260BDE8F087043B51F8042B43F8042F4F
:10FEF0008E45F9D8EBE71346CBE700BF02690B69E3
:10FF0000D21A13D19B0014301431194410B4034495
:10FF100001E098420CD253F8044D51F8042D94425C
:10FF2000F7D009D301205DF8044B704710467047A5
:10FF300000205DF8044B70474FF0FF30F3E700BF3F
:10FF40002DE9F8430B690F4611695B1A002B9046A7
:10FF500017D1890007F1140208F114055318294438
:10FF600001E09A425ED253F8046D51F8044DA64266
:10FF7000F7D060D23B46144647464FF001099846F9
:10FF800006E05DDB07F1140502F114044FF00009EF
:10FF90007968FFF75FFDD8F810303E69C0F80C9023
:10FFA00004EB830CA64605EB860700F1140400233E
:10FFB0005EF8041B55F8048B8AB213FA88F3090C17
:10FFC0009A1AC1EB184303EB224392B242EA03426E
:10FFD000F44544F8042B4FEA2343E9D8AF4217D93C
:10FFE000A446294651F804EB13FA8EF2131403EBDE
:10FFF0001E4392B242EA03428F424CF8042B4FEA6E
:020000040801F1
:100000002343EFD8ED433D4425F0030504352C444C
:10001000043C22B954F8043D013E002BFAD006619D
:10002000BDE8F8830021FFF715FD012200230261DE
:100030004361BDE8F8832C464FF000091546A7E759
:100040003B4607F1140408F1140547464FF0010937
:1000500098469DE70F4B0B40A3F15073002B02DD38
:100060000020194670475B421B15132B0BDD143B18
:100070001E2BDDBFC3F11F03012202FA03F301238C
:100080000021184670474FF40022002042FA03F185
:10009000704700BF0000F07F2DE9F041066900F1D4
:1000A000140808EB860656F8047C3846FFF78EFDE8
:1000B000C0F120030A280B60A6F104031ADC98455E
:1000C00038BF56F8083CC0F10B0227FA02F138BFDE
:1000D00023FA02F200F1150341F07F5528BF0022F8
:1000E00007FA03F345F4401543EA02042046294683
:1000F000BDE8F081984520D2B0F10B0256F8081CFB
:100100001ED007FA02F040F07F50C2F12007A6F19E
:10011000080340F4401021FA07FE984540EA0E0516
:1001200020D256F80C3C01FA02F023FA07F20243FF
:10013000144620462946BDE8F0810B3809D1014616
:1001400047F07F550C4645F4401520462946BDE84A
:10015000F08107FA00F040F07F55002245F4401589
:100160001446E6E701FA02F21446E2E72DE9F0430D
:1001700083B001211C46C3F30A5517460A9EFFF7B8
:1001800069FCC4F3130481460DB144F48014019456
:100190001FB302A840F8087DFFF738FD002835D1CD
:1001A0009DE80C00C9F81420002B0CBF012102218E
:1001B000C9F81830C9F81010DDB909EB8103A0F2B5
:1001C000324030601869FFF701FD0B9BC0EB411016
:1001D0001860484603B0BDE8F08301A8FFF716FD9C
:1001E000019BC9F8143001212030C9F81010002DEE
:1001F000E3D0A5F2334808EB000333600B9BC0F15A
:1002000035001860484603B0BDE8F0839DE80C0057
:10021000C0F1200103FA01F10A43C3400193C9F878
:100220001420C1E72DE9F04383B00E466946074626
:10023000FFF732FF04460D46304601A9FFF72CFFB9
:1002400089469DE80A003A693669C91A961B01EB8E
:100250004613002B80460BDD05EB03510D4642464D
:100260004B462046294603F05FF903B0BDE8F08312
:10027000A9EB0357B946F2E770B4146902F114030D
:1002800001394E1103EB84040136A34200EB8606CC
:100290000CD2011F53F8045B41F8045F9C42F9D86B
:1002A000A31A153B23F0030304331844864204D9F0
:1002B000002340F8043B8642FBD870BC704700BF67
:1002C00003694A11934210B400F1140410DA04EBEC
:1002D00083039C4221D253F8040C043B18B115E06F
:1002E00053F8042D92B99C42FAD35DF8044B704741
:1002F00010DD11F01F010DD054F8220020FA01F397
:1003000003FA01F1884204EB8203E2D001205DF898
:10031000044B704704EB8203DBE70020E5E700BFF6
:1003200070B50D46084C114606461A46284600236D
:100330002360F3F79DFC431C00D070BD2368002BA5
:10034000FBD0336070BD00BFE01A002070B40D78A0
:100350005E2D2FD0002201311646431E00F1FF040E
:1003600003F8012FA342FBD185B186F0010242556B
:100370004C1C14F8013C2D2B0ED05D2B09D013B171
:100380001D462146F3E7084670BC7047481E70BC06
:100390007047204670BC70474E785D2EF0D0B54255
:1003A000EEDC023143190135AE4203F8012FFADCCD
:1003B0000234DEE701224D7816460231CDE700BF58
:1003C000004870470000C07F0EB4F0B59CB021AC6F
:1003D0004FF4017254F8046BADF8142002900690AB
:1003E000F9F76EFD0C4B0194054632460B4F186829
:1003F000039523464FF6FF76002402A907950A9736
:100400000E941394ADF8166001F08EFB1CB0BDE89D
:10041000F04003B0704700BFE80500208599000850
:100420002DE9F0410F469046FFF714FE04460D46B5
:10043000B8F1000F11D0C7F30A53C3F16B03002BBF
:100440000BDD1B0503F17F55002405F54015224601
:100450002B4602F03FFFBDE8F08120462946BDE86B
:10046000F08100BF000000002DE9F04F1D46A1B053
:100470000023834628460E4606921C93FFF780FA17
:100480000024002382460068CDE90434F9F718FD02
:100490001B9681463246144612F8017B2D2F00F23E
:1004A000AF80DFE807F017ADADADADADADADAD815F
:1004B00081818181ADADADADADADADADADADADAD1C
:1004C000ADADADADADAD81ADADADADADADADADAD88
:1004D000AD2BAD7E069B4FF000094FF0000A43B1F3
:1004E00000230793069B1E60079B13B10AF100438C
:1004F0009A464846514621B0BDE8F08F0023079345
:10050000621C1B926778002FE4D0302F14467BD0FA
:10051000002308940A93A7F13003092B00F2E78324
:100520004FF00008204645464446082CC8BF08EB5B
:10053000880805EB850300F1010007EB43031B90DE
:10054000C4BF07EB4807A7F130080778D8BFA3F16D
:100550003005A7F13003092B04F10104E5D9DAF8DD
:1005600000104A46F9F71AFD00B300203B468146C9
:100570000746A246652B00F0B280452B00F0AF8005
:100580000022002C52D118B90A9A002A00F0D38216
:100590004FF000094FF0000A069B002BA4D01B9ED1
:1005A000A0E701230793ABE71B9274E71B9B03EBC8
:1005B00009021B9213F809300746A246A3F1300244
:1005C000092A00F27B82411C1346002A00F087862C
:1005D00001290F4418BF001905D100F07CBE4D0061
:1005E000844200F0C0840134611E082905EB8501B6
:1005F000F5DD102CDCBF08EB88084FEA4808EFE770
:100600000023302F079383D16378582B00F0538356
:10061000782B00F0508301341B942778302FFAD0C8
:10062000002FB5D0012308940A9374E7102CA2EB95
:1006300007032846A1460B93A8BF4FF0100902F00C
:10064000D3FDBAF1000F08BFA246B9F1090FCDE9F9
:10065000040113DD494B03EBC90353E9122302F0F4
:1006600039FE064640460F4602F0BEFD02460B46E6
:100670003046394602F07CFCCDE904010F2C00F332
:1006800085800B9B002B27D040F307850B9B162BF7
:1006900000F38384394F07EBC307D7E90001DDE995
:1006A000042302F017FE81468A4675E71BA83449E9
:1006B00002F056FB00283FF40DAF1B9B3149013B74
:1006C0001BA81B9302F04CFB10B91B9B01331B931F
:1006D0002D4B059300230493DDE9049A5CE7002C7D
:1006E00000F0E0811B9E731C1B9373782B2B00F092
:1006F000DF822D2B00F017824FF0000CA3F13002A7
:10070000092A00F2D282302B05D11B9A01321B92AA
:100710001378302BFAD0A3F13102082A3FF630AF1C
:100720001B9A0C92511C303B1B910B935378A3F1F5
:10073000300EBEF1090F0FD80B9A01311B9102EB5D
:10074000820203EB42020B78A3F1300EBEF1090FD7
:10075000A2F13002F1D90B920C9A891A082900F300
:1007600013840B9A44F61F618A42A8BF0A46BCF163
:10077000000F3FF406AF524203E700BF304E0108BE
:10078000404F0108444F01080000F07F0B9BC9EB6C
:1007900004099944B9F1000F40F38C8319F00F015B
:1007A0000AD0B94B03EBC101D1E90001DDE9042313
:1007B00002F090FDCDE9040139F00F0640F01282FD
:1007C00000230A9300952346524608995846FFF79E
:1007D000B1F91290002800F0E5820B9A0021002A5E
:1007E000C2F10003A8BF0B460C9322EAE2730B93FD
:1007F0000F468A46129C58466168FFF72BF9064659
:10080000002800F0378322699DED047B02329200BC
:1008100004F10C010C308DED087BF8F74BF81EA8A5
:100820001DA90190DDE9082300915846FFF79EFCC1
:100830001C90002800F0438401215846FFF714FA69
:100840000746002800F016831D9A002AC0F2328164
:100850000C9B0B9C9D180A981E9B8C49121A1A44DB
:10086000013A8A42C3F1360380F2EB80891A1F29CC
:10087000A3EB010300F3258101228A400E9200229E
:10088000139205EB03081C440A9B45452A461C4469
:10089000A8BF4246A242A8BF2246002A03DDC2EBFF
:1008A0000808A41AAD1A0C9BBBB139461A46584623
:1008B000FFF77CFA0746002800F0DC8201461C9A0C
:1008C0005846FFF7DBF9002800F0D4820D901C9900
:1008D0005846FFF7E5F80D9A1C92B8F1000F08DDB5
:1008E00042461C995846FFF7B1FA1C90002800F0C8
:1008F000E6830B9B43B131460B9A5846FFF756FAF5
:100900000646002800F0B682002C08DD314622465B
:100910005846FFF79BFA0646002800F0AB82002DF0
:1009200008DD39462A465846FFF790FA0746002860
:1009300000F0A08232461C995846FFF701FB824620
:10094000002800F097820023C268C36039460D92E8
:10095000FFF7D4FA0028C0F2CD8300F01D84394699
:100960005046FFF75FFC00224FF0804304460D46DF
:1009700002F02CFF002869D00D9B002B00F0A9800D
:100980009FED3D7B059B424D8DED0E7B00249946EE
:10099000DFF804813F4B09EA0808984500F0D88148
:1009A0000A9B2BB3B8F1D46F22D835A3D3E9002327
:1009B000DDE90E0102F00AFFB0B1DDE90E0102F03F
:1009C00061FF002800F0458302F00EFCCDE90E0126
:1009D0000D9B002B40F03883DDE90E1202F100433D
:1009E00014911593DDE9144505F1D663C8EB0305B1
:1009F000DDE90801FFF72EFB02460B46204629469B
:100A000002F068FCDDE9082302F0B2FACDE9040146
:100A10000C460A9B23B9204B2340984500F0EC81FB
:100A20001C995846FFF73CF831465846FFF738F80E
:100A300039465846FFF734F851465846FFF730F824
:100A4000D8E60022139201220E921AE7134B204699
:100A50002946002202F03EFC0D9BCDE90E01002B41
:100A60005CD101F1004310901193059BDDE9104525
:100A700099468DE7AFF30080000000000000F03FD2
:100A80000000C0FFFFFFDF41304E010802FCFFFF06
:100A90000000F03F0000E07F0000F07F0000E03F3A
:100AA0004FF00109002844D10A9B002B3FF412ADFE
:100AB000044617E60B9B0C9D9C1ACCE64FF00109EF
:100AC00058E5C149891A012202FA01F113910E92E7
:100AD000D7E6DDE90412002940F0C980C2F3130310
:100AE0009146002B40F0C9800022B84B2046294691
:100AF00002F062FE002840F071830022B44B2046D1
:100B0000294602F0E7FB0A460146CDE90E1202F142
:100B1000004318901993DDE9184539E79DED0E7BE8
:100B20008DED107BA1E74FF0010CB31C1B93B37844
:100B3000E4E50024D6E5B9F1000F7FF4CBAC493BE6
:100B4000252B3FF6C7AC01A252F823F0AD060108F1
:100B5000D5040108D5040108D5040108D50401080D
:100B6000890C0108D5040108D5040108D504010841
:100B7000D5040108D5040108D5040108D5040108ED
:100B8000D5040108D5040108D5040108D5040108DD
:100B9000D5040108D5040108D5040108D5040108CD
:100BA000D5040108D5040108D5040108D5040108BD
:100BB000D5040108D5040108D5040108D5040108AD
:100BC000D5040108D5040108D5040108AD060108C3
:100BD000D5040108D5040108D5040108D50401088D
:100BE000890C0108B6F59A7F00F3DC803611012EDE
:100BF000DFF8009240F30F83DDE9040100234F4644
:100C0000984616F0010F08F101084FEA660604D075
:100C1000D7E9002302F05EFB0123012E07F108074C
:100C2000EFD1002B40F06983059BA3F1547305932A
:100C300009EBC808DDE90423D8E9000102F04AFB0A
:100C400021F000431B0D634A1B059342CDE90401CB
:100C500000F2A880A2F58012934240F2C8825E4B57
:100C6000059300230A934FF0FF330493AAE5DDE9CF
:100C70000412012900F0F28191469FED517B00247E
:100C8000564D8DED0E7B83E61BA8554902F068F8A2
:100C900000283FF41FAC1B9B1B78282B00F0098316
:100CA000504B05930023049316E51B96002268E43D
:100CB0004FF0000C39E7079A02951CAB01920093A4
:100CC000494A1DAB1BA9584601F0C2FD10F00706AA
:100CD00005463FF45DAC062E40F07B8101340023D5
:100CE0001B944FF000094FF0000A079354E4DAF820
:100CF000001020464A46F9F751F948B14FF0000A72
:100D00003B46D0465546504657465446D14631E4B8
:100D10001B9B03EB09021B9213F80930302B06D101
:100D200001321B921378302B00F10100F8D0A3F1AF
:100D30003102082A40F2A2814FF0000A652BD0460A
:100D4000554657463FF4ACAE54464FF0010914E403
:100D5000A9F1547305939DED047B51EC170BFFF73C
:100D600079F902460B462046294602F0B3FADDE93E
:100D7000042302F0FDF821F00043CDE904011B0D2E
:100D80001A4ADDE908011B059342CDE9160140F23C
:100D9000FF80114B99426AD00F4B05934FF0FF3300
:100DA00004933DE6124B0593002222230492DDE9D1
:100DB000049ACBF80030FFF7EFBB00BFAFF3008021
:100DC000000000000000F03FE2FBFFFF0000F03FEA
:100DD0000000E03F0000A07CFFFFEF7F0000F0BFBD
:100DE0004C4F01080000F8FF2C4F0108FFFF9F7CCB
:100DF0000000F07FF84E0108DDE90E8949464046C3
:100E000002F018FD02F000FA0B4602464946404641
:100E100002F0ACF80D9B80468946002B36D1049B2E
:100E2000002B33D1C4F3130484BBB0A3D3E9002354
:100E300002F0C2FC00283FF4F3ADD046DDE9049A8D
:100E40001C9801465846FEF72BFE31465846FEF7E1
:100E500027FE39465846FEF723FE12995846FEF7FC
:100E60001FFE41465846FEF71BFEFFF795BB169B3B
:100E7000013391D1D0461C98994B0593002222232F
:100E80000492DDE9049ACBF80030DAE78EA3D3E9C7
:100E900000234046494602F08FFC0028CDD1404651
:100EA00049468BA3D3E9002302F0A4FC00283FF4B9
:100EB000B7ADC2E73FF484ACC9F1000616F00F02EB
:100EC0000AD0884B03EBC203DDE90401D3E9002318
:100ED00002F02AFBCDE9040136113FF471AC1F2E5C
:100EE00038DC16F0100300F0C9816A23002E0A9343
:100EF00013DDDDE904017C4F0023F20704D5D7E9B7
:100F0000002302F0E7F90123761007F10807F4D176
:100F1000002B40F0F5810A9B9BB1DDE90412C2F37E
:100F20000A53C3F16B03002B11460ADD1F2B40F35C
:100F3000AD810022342B049240F3D7814FF05C73D3
:100F4000059300220023DDE9040102F02BFC0028B8
:100F50003FF438AC2223CBF800304FF000094FF0BB
:100F6000000AFFF719BB1B990134082840F38F8052
:100F7000102CDCBF08EB880802EB480800204B1C53
:100F80001B934B78FFF71ABB44F61F62FFF7EFBBCA
:100F9000059B03F1547405943BE50B9EC4F12503B6
:100FA0009E423FF7F3AB4F4DC4F10F0405EBC40174
:100FB000341BDDE90423D1E9000105EBC40502F08F
:100FC00089F9D5E9002302F085F981468A46FFF7C1
:100FD000E3BA1C9A3AB135211EA8FFF74DF95846DD
:100FE0001C99FEF75DFD062E0BD8DFE806F0291DE3
:100FF0001813041D29006FF0004305934FF0FF33D1
:10100000049329077FF568AB059B43F000430593E4
:10101000FFF762BB324B059300230493F1E71E9B5D
:1010200004931F9B0593ECE71D9A1F9B1E99049147
:1010300002F2334223F4801343EA02530593E0E7BC
:10104000002305930493DCE79DED0E7B8DED147B6F
:10105000C8E49FED217B8DED0E7BB9E4DDE9041240
:101060009146002A7FF409AED0462223CBF8003007
:101070001C984FF000094FF0000AE2E61B9A089214
:101080000025303B471C1146AA46A846012405EB23
:10109000850503EB4505002071E70B9911F1160F4B
:1010A000FFF674AB0F4AA2EBC102D2E90023DDE9DF
:1010B000040102F039FA81468A46FFF76DBAD0463C
:1010C000DAE600BFAFF300809535A094FFFFDF3F65
:1010D00035E5AF350000E03F000000000000F03FC4
:1010E0000000F07F304E0108684F01089535A0944C
:1010F000FFFFCF3F0D9A5546D046DDE9089A7ABBEF
:10110000DDE9040160BBC1F313030C4643BB21F0CE
:1011100000431B0D1B05B3F1D66F21D96B6913B9C1
:101120002B69012B1CDD414601225846FEF78EFE3D
:1011300039468046FEF7E2FE002811DD0A9B002BAF
:1011400040F0AC80744B2340A3F580136FEA135337
:101150006FEA035305934FF0FF330493DDE9049ADC
:101160000A9BBBB16D4B179300231693DDE9162341
:101170004846514602F0AEF803460C4681468A4680
:10118000CDE9043431B9049B23B922231C98CBF850
:10119000003056E61C9854E60D9BD046DDE9089ACF
:1011A00053B3DDE904455E4BC5F3130199422A466A
:1011B00046D0139B53B3059A1342D1D00D9B0A9A84
:1011C000DDE9040153B3FFF72BF902460B4648460D
:1011D000514601F0CDFE81468A46C1E79FED4A7B2C
:1011E0008DED187B9FED4A7B8DED0E7B93E401F135
:1011F00054730593FFF7E4BADDE90412C2F3130355
:101200001446002BD5D10029D3D197E70E9B049A21
:101210001342A5D0D2E74FF0000805E5FFF700F92B
:1012200002460B464846514601F0A0FE002200232C
:1012300081468A4602F0B6FA00287FF416AF8FE79F
:101240000A9B0499FBB1344B2B40B3F1D46F1AD8ED
:101250001B0DC3F16B034FF0FF3000FA03F38B4219
:10126000A7D130498A423DD02B4B134003F5801360
:10127000059300230493DDE9049A71E7002E0A9395
:101280003FF737AE5DE64FF0FF33E8E74FF0FF3250
:1012900002FA03F3049A1A40049252E61E4B2340CA
:1012A000B3F1D66F3FF750AFB3F15C7F3FF75AAF62
:1012B000DBE61BA81EAA1C4901F06AFD05287FF485
:1012C000EFAC1F9B43F0FF4343F4E00305931E9BE9
:1012D0000493FFF701BA20461B99013445E60846FE
:1012E0001B994CE60133BFD1C5E5203B4FF0FF32DF
:1012F00002FA03F30B40059323E6CDE9040193E4DE
:10130000CDE9040107E600BF000000000000E0BFD7
:10131000000000000000E03F0000F07F00005039B6
:10132000FFFF0F00FFFFEF7F504F0108054B1B68C9
:1013300010B45B6B044C002B08BF23465DF8044BD4
:10134000FFF792B8E8050020440A00202DE9F04F8D
:1013500085B09A460291039001920F460E9E00E0DE
:101360002F463D46304615F8014BFEF7FBFA204468
:10137000437803F0080303F0FF02002BF0D12D2C7B
:1013800000F083802B2C08BF7C78009208BFBD1C26
:10139000BAF1000F0CD0BAF1100F00F09580009B4D
:1013A0005646F7176BB94FF0FF386FF000490CE065
:1013B000302C7FD00A2600274FF00A0A009B002B12
:1013C000F1D04FF000084FF0004932463B4640460E
:1013D000494602F0C7FA3B469346404632464946E4
:1013E00002F0C0FA4FF0000E002200230FE045D0BB
:1013F00002FB07F406FB0344A2FB0623234412EB83
:101400000C0243EBEC734FF0010E15F8014BA4F105
:10141000300CBCF1090F06D9A4F1410CBCF1190F35
:101420000DD8A4F1370CE24512DDBEF1FF3FECD040
:10143000994208BF9042DAD24FF0FF3EE5E7A4F1AF
:10144000610CBCF1190F03D8A4F1570CE245ECDC98
:10145000BEF1FF3F1ED0009911B1524263EB43032E
:101460000199002942D0BEF1000F1FD1029D104604
:101470001946019B1D6005B0BDE8F08FE345B7DA62
:1014800002460B464FF0FF3EBFE70123BD1C7C78B0
:1014900000937DE7009B2BBB4FF0FF306FF00041C6
:1014A000039A22231360019B13B9E4E710461946FF
:1014B000013DDEE72B7803F0DF03582B0BD0082625
:1014C00000274FF0080A79E7302C12D12B7803F06F
:1014D000DF03582B0DD16C781026002702354FF012
:1014E000100A6BE700204FF00041D9E7104619467B
:1014F000C1E71026002761E730B5064C064D246889
:10150000646B83B0002C08BF2C460094FFF71EFFCD
:1015100003B030BDE8050020440A00202DE9F84F53
:10152000DDF828900E460746154698468B4600E0A3
:10153000A3465C46484614F801ABFEF713FA504444
:10154000407800F0080000F0FF0C0028F0D1514670
:101550002D2961D02B2904BF9BF801100BF1020447
:10156000B8F1000F0CD0B8F1100F5CD04FF0FF3382
:10157000B3FBF8F308FB03FA6FEA0A0AC14607E077
:10158000302961D04FF00A083D4BC1464FF0050AA3
:101590004FF0000E704606E02FD009FB00204FF000
:1015A000010E14F8011BA1F13002092A05D9A1F19D
:1015B0004102192A0BD8A1F1370290450FDDBEF187
:1015C000FF3FEED09842E7D94FF0FF3EE9E7A1F1A7
:1015D0006102192A03D8A1F157029045EFDCBEF150
:1015E000FF3F11D0BCF1000F00D0404255B1BEF119
:1015F000000F0DD12E60BDE8F88F5245CDDD4FF0C4
:10160000FF3ECEE7BDE8F88F22233B60704645B32E
:10161000661E2E60BDE8F88F0BF102049BF80110E6
:101620004FF0010C9CE730291DD1237803F0DF0334
:10163000582B1ED14FF010096178C8464FF00F0AA1
:1016400002346FF07043A3E7237803F0DF03582BD5
:10165000F0D04FF00808C1464FF0070A6FF0604322
:1016600096E7BDE8F88F4FF00F0A6FF07043C14660
:101670008EE7C1464FF00F0A6FF0704388E700BF56
:101680009999991930B5064C064D2468646B83B05E
:10169000002C08BF2C460094FFF740FF03B030BD7C
:1016A000E8050020440A002030B5084C084B2568A6
:1016B0006C6B83B0002C08BF1C46009413460A468E
:1016C00001462846FFF72AFF03B030BDE805002099
:1016D000440A00202DE9F04F85B08B460290174652
:1016E0001E4688460E9C00E0A8464546204615F852
:1016F000019BFEF737F94844437803F0080303F0F1
:10170000FF02002BF0D14C462D2C00F08C802B2CAE
:1017100008BF98F80140019208BF08F10205DEB148
:10172000102E00F087804FEAE67932464B464FF0A4
:10173000FF304FF0FF3102F015F9324603908A4630
:101740004B464FF0FF304FF0FF3102F00BF9B0463F
:101750009646039A53460CE0302C00F08180574B9C
:101760004FF0050E4FF099324FF00A084FF0000984
:101770000A264FF0000C0020002112E0994208BF19
:10178000904240D000FB09F408FB0144A0FB080193
:10179000214410EB0A0041EBEA714FF0010C15F8FF
:1017A000014BA4F1300ABAF1090F06D9A4F1410A9C
:1017B000BAF1190F0DD8A4F1370A564512DDBCF164
:1017C000FF3FECD08B4208BF8242D7D24FF0FF3CA4
:1017D000E5E7A4F1610ABAF1190F03D8A4F1570A99
:1017E0005645ECDCBCF1FF3F12D0019B13B14042E7
:1017F00061EB410127B1BCF1000F12D15D463D60A4
:1018000005B0BDE8F08FF245BCDD4FF0FF3CC6E708
:10181000029A222313604FF0FF304FF0FF31002F68
:10182000EED0013DEBE7012308F1020598F80140F5
:10183000019374E7302C24D12B7803F0DF03582B6D
:101840002AD14FF0FF336C7803934FF00F0E02351F
:101850006FF0704A4FF010084FF00009102678E73B
:101860002B7803F0DF03582BEBD04FF0070E4FF02F
:10187000FF326FF060434FF008084FF00009082670
:1018800077E74FF00F0E4FF0FF326FF070434FF0DD
:1018900010084FF000096CE74FF010084FF00009F6
:1018A00042464B464FF0FF304FF0FF3102F05AF8FE
:1018B0006FF0704396464FF0FF325AE799999919A5
:1018C00030B5064C064D2468646B83B0002C08BF0D
:1018D0002C460094FFF7FEFE03B030BDE805002063
:1018E000440A00202DE9F04F936883B09046002B06
:1018F00072D083464FF00009166808688B680D4661
:101900004C46002C45D09C421F469A4646D3AB8994
:1019100013F4906F2DD06F69296907EB4707C1EB6E
:10192000000A07EBD777601C7F105044B8423A4654
:1019300084BF07463A465B0533D511465846F6F74D
:1019400079FC002837D0524629690190F6F7B2FF9A
:10195000AA89019B22F4906242F08002AA81CAEB1C
:10196000070203EB0A006F612B612860AA6027461B
:10197000A24652464946F7F737F8D8F80820AB6830
:101980002868DB1B5044141BAB602860C8F8084073
:1019900014B3D6F8009074680836B2E72746A2461A
:1019A000E7E75846F7F7F6FB03460028D7D1296941
:1019B0005846F5F72FFE0C23CBF80030AB890022F8
:1019C00043F040034FF0FF30AB81C8F80820C8F85F
:1019D000042003B0BDE8F08F0020C8F8040003B075
:1019E000BDE8F08F4B1C70B51BD09389146B23F0AE
:1019F00020039381CDB2BCB114465268636B9A4206
:101A00000E4609DA23685A1E226003F8016C6368E7
:101A100001336360284670BD214600F0A5FD002813
:101A2000F0D04FF0FF35F5E71069136828B1984200
:101A300003D213F8010C85420FD093631346566806
:101A4000D66302F1400403205063146303F8421F7D
:101A5000012113605160284670BD5168013B01317E
:101A600013605160D6E700BF10B50C46096B69B131
:101A700004F14003994201D0F5F7CCFDE36B6360BC
:101A80000020206313B1A36B236010BDA3892269DA
:101A9000226043F020030022A38162604FF0FF30F8
:101AA00010BD00BF2DE9F04F83B002FB03F9019296
:101AB0009A460C9CB9F1000F29D007460E464D46B8
:101AC0004FF000080FE02168F6F7F4FE2268C4F832
:101AD00004805A442260214638465E44CBEB05051B
:101AE000FFF7C2FFB8B9D4F804B05D4530465A4696
:101AF000E9D82A462168F6F7DDFE62682368521BA2
:101B00002B4450466260236003B0BDE8F08F484626
:101B100003B0BDE8F08F019BC5EB0909B9FBF3F0F9
:101B200003B0BDE8F08F00BF2DE9F04F8B46B1F94F
:101B30000C10D9B08F0481461446069309D4DBF803
:101B4000643041F4005123F40053ABF80C10CBF88F
:101B5000643025460023059303931F46079315F829
:101B6000013B0B936BB3FDF701FF0B9A10444378D5
:101B700003F0080303F0FF063BB3DBF8043011E089
:101B8000FDF7F4FEDBF800301A7810440133427898
:101B900016070FD5DBF80420CBF80030531E0137B1
:101BA000CBF80430002BEBDC59464846FFF75CFFCE
:101BB0000028E5D02C46254615F8013B0B93002B59
:101BC000D1D1079859B0BDE8F08F252A40F0848024
:101BD00094F8018034466B1CB8F1780F00F2D08184
:101BE000DFE818F0CD00CE01CE01CE01CE01CE014E
:101BF000CE01CE01CE01CE01CE01CE01CE01CE016D
